:100000000C946E0D0C949F0D0C949F0D0C949F0DF1
:100010000C949F0D0C94F6870C94BD520C94A64C36
:100020000C949F0D0C949F0D0C949F0D0C949F0DA0
:100030000C949F0D0C949F0D0C949F0D0C949F0D90
:100040000C949F0D0C94B97D0C947A870C949F0DA1
:100050000C949F0D0C949F0D0C949F0D0C94974A3B
:100060000C949F0D0C94DF8D0C94B68D0C949F0D09
:100070000C949F0D0C949F0D0C949F0D0C949F0D50
:100080000C94CA910C949F0D0C949F0D0C949F0D91
:100090000C948D8D0C94648D0C949F0D0C949F0D7D
:1000A0000C949F0D0C949F0D0C949F0D0C949F0D20
:1000B0000C949F0D0C9425610C949F0D0C949F0D36
:1000C0000C949F0D0C949F0D0C949F0D0C943B8DE4
:1000D0000C94128D0C949F0D0C94E98C0C94C08C94
:1000E0000C949F0D66186918701873187618791893
:1000F000801887188A18911898189F18611E8F1EEB
:10010000C61EFD1ED81F0F203D206B20312131213E
:10011000312131213121312131213121312131214F
:10012000312131213121312131213121312131213F
:10013000312131213121312131213121312131212F
:10014000312131213121341F6C1FA31F9920D1206F
:10015000082129232F2335233B23412347234D23E4
:10016000532359235F2365236B237D238323892313
:10017000A123A723AD23B323B923BF23C523CB23B7
:10018000D123D723DD23E323E923EF23FB23072414
:100190000D2413241924312437243D2443244924D5
:1001A0004F2439253F25452557255D256325752590
:1001B0007B25812587258D259325A525AB25D5254F
:1001C000DB25E125E725FF2505260B261126A6269A
:1001D000A626A626A626A626A626A626A62627263E
:1001E0002B262F26352639263D264126452649260B
:1001F0004D265326712677267D261F2455245B2401
:10020000612467246D247324ED25F325F925172631
:100210001D262326832689268F2699259F25792426
:100220007F2485248B24912497244B256925012440
:100230007123772325242B2495269B26A126F5239D
:10024000B125B725BD25C325C925CF259D24A324C8
:10025000A924AF24B524BB24C124C724CD24D3248E
:10026000D924DF24E524EB24F124F724FD240325FD
:1002700009250F2515251B25212527252D25332566
:1002800065265F2659266B2651256F258F239523DA
:100290009B236D2D4A2D232D8A2DE12DA92DD82D9F
:1002A000C72D922E752E4E2EE22EAF2EAF2ED12EB2
:1002B000BA2E67346734813467348E34A734C2343D
:1002C000DD340038343869388938BE382639363953
:1002D000603AAA39B439E8391D3A2B3A603AF23813
:1002E000D13EE83EFF3E163F2D3F5B3F723F893FC8
:1002F000A03FBF3FD73FEE3F0D402340443F224643
:100300002546144618461E465C4629462D46334669
:1003100037463B464146454649465C464F4653466E
:1003200057462A482F4834483E484848C148524812
:100330005A4862486C48764880488F489948C14876
:10034000A348AD48B74852615B61636177618961D9
:100350009B61A66105A84CCDB2D44EB93836A9022E
:100360000C50B9918688083CA6AAAA2ABE000000B3
:10037000803F3400330032004E6F6E650053746F5F
:1003800070706564004E65757472616C205475728E
:100390006E004D6F76696E67205265766572736583
:1003A000004D6F76696E6720466F727761726400E8
:1003B0004272616B696E670054414E4B2052455347
:1003C000544F5245440025004865616C7468204CC8
:1003D0006576656C3A200056454849434C452052A5
:1003E000455041495220434F4D504C4554450054CF
:1003F000414E4B2044455354524F5945440025002B
:100400004865616C7468204C6576656C3A200029FB
:100410000056454849434C452052455041495220D9
:1004200053544152544544202800524550414952AA
:10043000204F5045524154494F4E2043414E434571
:100440004C4C45440029004D414348494E45204706
:10045000554E2048495421202800524550414952C8
:10046000204F5045524154494F4E2043414E434541
:100470004C4C454400290043414E4E4F4E204849C4
:10048000542120280054757272657420726F746153
:1004900074696F6E206973206E6F74206F662074AC
:1004A00079706520536572766F2E204E6F207365CC
:1004B00074757020617661696C61626C652E004EA6
:1004C0006F207374656572696E6720736572766FED
:1004D0002061737369676E65642C2072652D636893
:1004E00065636B2076656869636C652074797065F7
:1004F0002E0054757272657420656C65766174693E
:100500006F6E206973206E6F74206F66207479702F
:100510006520536572766F2E204E6F20736574755B
:100520007020617661696C61626C652E00546F7039
:10053000204C65667400546F702043656E7465725C
:1005400000546F70205269676874004D6964646C70
:1005500065204C656674004D6964646C6520436574
:100560006E746572004D6964646C652052696768D9
:100570007400426F74746F6D204C65667400426F36
:1005800074746F6D2043656E74657200426F74748D
:100590006F6D205269676874004649524D57415249
:1005A000452056455253494F4E3A200069427573D3
:1005B00000534275730050504D004E6F6E652044DD
:1005C0006574656374656400417A696D757468204B
:1005D00020202000456C65766174696F6E202000D4
:1005E0005475726E20202020202020005468726FE5
:1005F00074746C6520202000537469636B20202084
:10060000202020204D696E2020202043656E7465D7
:10061000722020204D617820202020446561646292
:10062000616E642020526576657273656400524184
:1006300044494F20494E464F202D20004E4F542014
:1006400044455445435445440049474E4F52454460
:1006500000416E616C6F67004469676974616C008A
:10066000417578204368616E2E2020204D696E20F0
:10067000202020204D617820202020205479706592
:10068000004368616E6E656C73207574696C697A7D
:1006900065643A20004368616E6E656C7320646522
:1006A0007465637465643A2000202844697361624C
:1006B0006C656429002028456E61626C65642900C0
:1006C0004D656368616E6963616C207265636F6913
:1006D0006C00416972736F6674004D656368616E8A
:1006E0006963616C2042617272656C3A2000202857
:1006F0004D31290020284D3229002028422900426E
:10070000617272656C20456C65766174696F6E3AD2
:1007100020200020284D30290020284D312900209C
:100720002841290054757272657420526F74617487
:10073000696F6E3A2020200020416D7073290020DF
:100740002843757272656E74204C696D69743A2025
:10075000004472697665204D6F746F72733A202081
:1007600020202020004D4F544F52205459504553C3
:100770000054616E6B202854616D69796120444D8D
:1007800044290054616E6B2028444B4C4D20476532
:100790006172626F7829004361720048616C66740F
:1007A0007261636B0054616E6B00554E4B4E4F5738
:1007B0004E00596573004E6F002900252C204465BA
:1007C00063656C65726174696F6E20666163746FD6
:1007D00072200020284B69636B6261636B20737029
:1007E0006565642000547261636B205265636F69B4
:1007F0006C20456E61626C65643A202020004E2FAB
:100800004120666F722076656869636C6520747933
:100810007065005475726E204D6F64653A2020201B
:100820002020202020202020202020004E2F41208A
:10083000666F722076656869636C6520747970658F
:1008400000596573202854616D697961290025007C
:10085000202D20004E65757472616C205475726E87
:1008600020416C6C6F7765643A202020002073650E
:1008700063005472616E736D697373696F6E2044A7
:10088000656C61793A202020202000207365630088
:10089000456E67696E652050617573652054696D9A
:1008A000653A2020202020200020736563005368D3
:1008B0006966742054696D653A202020202020202C
:1008C000202020202020004175746F6D61746963C1
:1008D000004D616E75616C005472616E736D697369
:1008E00073696F6E20547970653A20202020202093
:1008F000002500596573202D2000526576657273BE
:1009000065205370656564204C696D697465643A4F
:100910002020002500596573202D2000466F727736
:10092000617264205370656564204C696D697465FB
:10093000643A202000206D73290025207468726FAE
:1009400074746C6520666F7220002028004D6F74EF
:100950006F72204E7564676520456E61626C6564D8
:100960003A202020200029004E6F6E65004E6F6EE9
:1009700065002C205072657365743A2000290020B0
:100980002841646A757374656420746F20002028A0
:100990004C6576656C3A2000446563656C20526155
:1009A0006D7020456E61626C65643A2020202020C5
:1009B0000029004E6F6E65004E6F6E65002C205052
:1009C00072657365743A20002900202841646A75B5
:1009D0007374656420746F200020284C6576656C04
:1009E0003A2000416363656C2052616D7020456E52
:1009F00061626C65643A20202020200041637469A4
:100A000076652044726976696E672050726F6669F8
:100A10006C653A200056656869636C65205479708E
:100A2000653A202020202020202020202000445231
:100A30004956452053455454494E47530020736549
:100A400063005265636F696C2064656C61793A205C
:100A50002020202020202020202020202020202096
:100A60002020002500596573202D200042617272FC
:100A7000656C20456C65766174696F6E2053706596
:100A80006564204C696D697465643A2000250059DD
:100A90006573202D200054757272657420526F7436
:100AA0006174696F6E205370656564204C696D696F
:100AB0007465643A202000545552524554205345E1
:100AC0005454494E475300556E6B6E6F776E004815
:100AD00065617679004D656469756D004C6967687C
:100AE0007400437573746F6D00556E6B6E6F776E27
:100AF000004E6F6E65004F70656E2050616E7A65B6
:100B0000720054616D6979612053706563002073D0
:100B10006563207265636F7665727929002073655D
:100B2000632072656C6F61642C2000204D47206843
:100B30006974732C20002063616E6E6F6E2068698B
:100B400074732C2000280057656967687420436C13
:100B50006173733A20202020200044616D61676535
:100B60002050726F66696C653A20202000596573C9
:100B7000202800416363657074204D472044616DF7
:100B80006167653A200059657320280053656E64DB
:100B9000204D4720495220436F64653A2020004E83
:100BA0002F410052657061697265642062793A2054
:100BB0002020202020004E2F4100486974205072D0
:100BC0006F746F636F6C20323A2020200029002060
:100BD000285465616D2000466972652050726F74FB
:100BE0006F636F6C3A2020202000466972652050A8
:100BF000726F746F636F6C3A20202020004973205D
:100C00005265706169722054616E6B3F2020200034
:100C1000495220262054616E6B20426174746C69C5
:100C20006E672044697361626C656400424154548C
:100C30004C4520494E464F00554E4B4E4F574E00A7
:100C400042656E6564696E6920544253204D696344
:100C5000726F0042656965722055534D2D52432DC8
:100C6000320054616967656E20536F756E6420436E
:100C7000617264004F70656E2050616E7A657220FB
:100C8000536F756E6420436172640042656E6564E3
:100C9000696E6920544253204D696E6900536F7527
:100CA0006E6420636172643A2000534F554E4420B5
:100CB0004341524400556E6B6E6F776E0042617215
:100CC00072656C20456C65766174696F6E20436F48
:100CD0006D6D616E640054757272657420526F742C
:100CE0006174696F6E20436F6D6D616E6400537443
:100CF000656572696E6720436F6D6D616E64005645
:100D0000656869636C6520537065656400456E674E
:100D1000696E65205370656564005468726F747401
:100D20006C6520436F6D6D616E6400537065656422
:100D3000206465637265617365732062656C6F77AB
:100D40002000537065656420696E63726561736528
:100D5000732061626F766520005475726E20537443
:100D60006F70706564004C656674205475726E20F7
:100D700053746172746564005269676874205475B5
:100D8000726E20537461727465640056656869639D
:100D90006C652053746F70706564004D6F76696E7A
:100DA000672052657665727365004D6F76696E6770
:100DB00020466F727761726400456E67696E6520C8
:100DC00053746F7000456E67696E6520537461726D
:100DD000740043616E6E6F6E2052656C6F61646566
:100DE000640056656869636C652044657374726F4E
:100DF0007965640043616E6E6F6E204869740042CD
:100E000072616B6573204170706C69656400566136
:100E1000726961626C6500290020286F66200050AD
:100E20006F732000417578204368616E6E656C2099
:100E3000005661726961626C65004F6E004F6666B4
:100E4000004200410045787465726E616C20496E05
:100E50007075742000070809090B0C0C0B0C0C545E
:100E6000757272657420537469636B202D2000467F
:100E7000756E6374696F6E202300202D3E20002064
:100E800073656300547572726574206D6F76656D5D
:100E9000656E742064656C61793A2020004E6F6E37
:100EA00065005965730054757272657420737469B6
:100EB000636B2066756E6374696F6E733A200046CB
:100EC000554E4354494F4E2054524947474552537B
:100ED0000076206375746F666629002028004C56E2
:100EE0004320456E61626C65643A202020202020FA
:100EF000007600566F6C746167653A2020202020D0
:100F0000202020202000596573004E6F004261743C
:100F1000746572792044657465637465643A200071
:100F2000424154544552590053657269616C2033F3
:100F300020547820426175643A2020004175782061
:100F400053657269616C20426175643A202020000B
:100F50004D6F746F722053657269616C20426175C8
:100F6000643A20005553422053657269616C2042F7
:100F70006175643A2020200042415544205241547A
:100F8000455300212000464143544F5259205245B9
:100F9000534554212000401F7017D007A00FA00F09
:100FA000DC05D007C40910278813983A1027580287
:100FB0006C0258026C0258026C0258026C02580211
:100FC0006C0258026C0258026C0258026C02580201
:100FD000B0366C023A026C023A026C023A026C02BF
:100FE000B036384A5C121C255C125C121C255C125F
:100FF000BC7FC7F2C07887A5B7C5A00F8813B80B10
:10100000401FB80BB80B7017401F416972736F66B1
:1010100074202D20456E61626C6564004D656368C7
:10102000616E6963616C205265636F696C202D206D
:10103000456E61626C656400416972736F6674200D
:101040002D2044697361626C6564004D656368615D
:101050006E6963616C205265636F696C202D20445A
:10106000697361626C656400436F6D6D73206368C2
:10107000616E67656420746F2055534200436F6D45
:101080006D73206368616E67656420746F205365BB
:101090007269616C20310044726976696E67205014
:1010A000726F66696C652073657420746F2023000D
:1010B00025005370656564207265647563656420FE
:1010C000746F2000537065656420726573746F726D
:1010D0006564005475726E20456E67696E65204FB9
:1010E0006E004D616E75616C207472616E736D6916
:1010F0007373696F6E202D2070757420696E206E79
:1011000065757472616C2067656172206265666FD7
:101110007265207374617274696E6720656E6769A9
:101120006E6521005475726E20456E67696E65208C
:101130004F666600456E67696E65204175746F2065
:1011400053687574646F776E00456E6761676520DC
:101150005472616E736D697373696F6E0044697365
:10116000656E67616765205472616E736D69737334
:10117000696F6E00536574205475726E204D6F64F4
:10118000653A203100536574205475726E204D6F9E
:1011900064653A203200536574205475726E204D98
:1011A0006F64653A203300456E61626C65204E6560
:1011B000757472616C205475726E7300446973614A
:1011C000626C65204E65757472616C205475726E28
:1011D0007300494F20506F72742041204F75747016
:1011E0007574202D204F6E00494F20506F7274206F
:1011F00041204F7574707574202D204F666600492C
:101200004F20506F72742042204F75747075742097
:101210002D204F6E00494F20506F72742042204F96
:101220007574707574202D204F66660000002100D3
:10123000240027002A002D003000330001010000A7
:10124000040107010A0100002200250028002B00EC
:101250002E003100340002010000050108010B01DD
:1012600020287769746820495229004669726520F0
:1012700043616E6E6F6E00466972652052657061E3
:101280006972205369676E616C00416972736F66A1
:1012900074202D204D616E75616C205472696767F2
:1012A0006572004D656368616E6963616C205265AB
:1012B000636F696C202D204D616E75616C205472D6
:1012C000696767657200536572766F205265636F58
:1012D000696C202D204D616E75616C2054726967B8
:1012E000676572004869676820496E74656E736946
:1012F000747920466C61736820556E6974202D20C6
:101300004D616E75616C2054726967676572004D3E
:1013100047205374617274004D472053746F7000FE
:101320004952204E4F5420656E61626C6564202DD9
:10133000206E6F2049522070726F746F636F6C73F0
:101340002073656C65637465642E00556E61626C14
:101350006520746F20656E61626C6520495200499A
:101360005220656E61626C65640049522064697345
:1013700061626C656400417578204F757470757496
:1013800020466C617368656400417578204F757400
:1013900070757420496E766572736520466C617352
:1013A0006865640053746F7020417578204F7574C0
:1013B00070757420426C696E6B696E670053746F50
:1013C00070205265766F6C76696E67204175782063
:1013D0004C6967687400494F20506F727420412037
:1013E0002D2050756C73656400494F20506F7274E6
:1013F0002041202D20537461727420426C696E6B01
:10140000696E6700494F20506F72742042202D2072
:1014100050756C73656400494F20506F72742042A0
:10142000202D20537461727420426C696E6B696E5A
:101430006700524144494F204641494C534146457B
:1014400000526164696F205265616479202D20002B
:1014500052657665727365643A2020004D6178208C
:1014600050756C73653A20004D696E2050756C7331
:10147000653A2000456E642056616C7565730045C1
:101480006E64205265636F696C20536572766F20BD
:10149000536574757000456E6420526F7461746991
:1014A0006F6E20536572766F2053657475700045BA
:1014B0006E6420456C65766174696F6E2053657249
:1014C000766F20536574757000536572766F207562
:1014D0006E2D726576657273656400536572766F02
:1014E0002072657665727365640052657665727305
:1014F00065643A2020004D61782050756C73653A20
:1015000020004D696E2050756C73653A200053744D
:101510006172742056616C75657300494E56414C7A
:10152000494420534552564F2E204E4F2053455488
:1015300055502E005365747570205265636F696C49
:1015400020536572766F0053657475702054757200
:1015500072657420526F746174696F6E2050616E91
:1015600020536572766F00536574757020537465EF
:101570006572696E6720536572766F20284F7574A7
:10158000707574203229005365747570205374652A
:101590006572696E6720536572766F20284F757487
:1015A00070757420342900536574757020547572F9
:1015B00072657420456C65766174696F6E20536541
:1015C00072766F0054616967656E2056322F56330C
:1015D00000536F6E790052435441204D6163686936
:1015E0006E652047756E00436C61726B204D6163C0
:1015F00068696E652047756E0052435441205265FC
:1016000070616972004942552052657061697200CB
:10161000436C61726B20526570616972004F706536
:101620006E50616E7A657200567354616E6B00463F
:101630004F560054616967656E2056310048656EEB
:1016400067204C6F6E670054616D69796120312F9E
:1016500033350054616D69796120322D53686F74A0
:101660000054616D69796100556E6B6E6F776E0025
:101670003A200042697420004761703A2000557397
:1016800065722046756E6374696F6E203100557304
:1016900065722046756E6374696F6E203200466F06
:1016A00072776172642047656172004E657574726D
:1016B000616C2047656172005265766572736520C2
:1016C000476561720053657420416363656C205205
:1016D000616D70204C6576656C3A2000536574200E
:1016E000446563656C2052616D70204C6576656C55
:1016F0003A2000416E616C6F672055736572204619
:10170000756E6374696F6E2031202D2000416E610B
:101710006C6F6720557365722046756E6374696FD0
:101720006E2032202D20002D00202D20002000547E
:101730005255450046414C53450025005761697498
:10174000696E6720666F7220726164696F2E2E2E3B
:101750002000556E6B6E6F776E0044657461636830
:1017600065642F4E41005265636F696C205365724A
:10177000766F0050616E20536572766F005365720C
:10178000766F2F455343004F6E626F617264204D38
:101790006F746F7220447269766572004F70656E67
:1017A0002050616E7A65722053636F7574205365A3
:1017B0007269616C20455343005361626572746FB6
:1017C0006F74682053657269616C00506F6C6F6C48
:1017D000752053657269616C00536572766F2031B4
:1017E00000536572766F203200536572766F203336
:1017F00000536572766F203400536572766F203522
:1018000000536572766F203600536572766F20370D
:1018100000536572766F2038004C56432045786936
:1018200074202D20566F6C74616765205265737447
:101830006F726564007629004C56432074687265A7
:1018400073686F6C64207265616368656421202829
:10185000004C696768742031204F6E004C696768DE
:10186000742031204F6666004C696768742032200E
:101870004F6E004C696768742032204F66660032F4
:101880006E64204D472053746F7000326E64204D9B
:10189000472053746172740052756E6E696E6720D2
:1018A0004C6967687473204F6E0052756E6E696E76
:1018B00067204C6967687473204F666600417578CD
:1018C000204F7574707574204F6E00417578204FED
:1018D0007574707574204F66660053746F70205273
:1018E00065766F6C76696E6720417578204C696704
:1018F00068740053746F7020417578204F75747050
:10190000757420426C696E6B696E67004175782052
:101910004F757470757420507265736574204469D6
:101920006D00537461727420417578204F75747026
:10193000757420426C696E6B696E67000000200050
:101940002300260029002C002F0032000001000097
:101950000301060109010505050507050808080832
:10196000020202020A0A0808040404040101010137
:101970000101010103030303030303030407070732
:101980000C0C0C0C0C0C0C0C0202020206060606D7
:10199000060606060B0B0B0B0B0B0B0B01021020A4
:1019A0002008081020401020408002010201080495
:1019B0000201010204081020408080402010080429
:1019C0000201800402018040201008040201080482
:1019D00002010102040810204080010204081020C6
:1019E000408000000A0B02090C0D0E0807030401D9
:1019F00000000000000000000000000000000000E7
:101A000000000000000000000000000000001211B3
:101A100010000000000000000000000000000000B6
:101A20000000000000000000536D6F6B65722065C0
:101A30006E61626C656400536D6F6B6572206469E2
:101A40007361626C65640053657420766F6C756DAC
:101A5000653A2000202D2053746172742052657005
:101A6000656174696E6700202D2053746F70005596
:101A700073657220536F756E64200041202D200025
:101A800042202D2000536F756E642042616E6B20E2
:101A900000506C61792F53746F7000506C61792025
:101AA00052616E646F6D00506C6179205072657682
:101AB000696F757300506C6179204E6578740053BE
:101AC00074617274205265766F6C76696E6720411E
:101AD0007578204C69676874000001AA11241FBE44
:101AE000CFEFD1E2DEBFCDBF00E00CBF16E0A0E03B
:101AF000B2E0E1E9F9E901E00BBF02C007900D9205
:101B0000A031B107D9F723E1A0E1B6E001C01D92F1
:101B1000A13AB207E1F71DE0CEE6DDE000E006C045
:101B200021970109802FFE010E948BB5CD36D10788
:101B300080E00807A9F70E94E9970C94CEBB0C94AB
:101B400000002F923F924F925F926F927F928F92FE
:101B50009F92AF92BF92CF92DF92EF92FF920F933C
:101B60001F93CF93DF93CDB7DEB7E6970FB6F89408
:101B7000DEBF0FBECDBF8091B2069091B3060E942A
:101B80009D8C0E947B6E69E975E08091B206909110
:101B9000B3060E943F8B62EF75E0CE0101960E9472
:101BA000008B0091B2061091B306D801ED91FC9123
:101BB0004D815E8169817A810280F381E02DC801C7
:101BC0001995C8010E949D8CCE0101960E94D08A71
:101BD0000E9402918091B2069091B306DC01ED91D2
:101BE000FC910284F385E02D19958091B2069091C5
:101BF000B3060E949D8C0E947B6E6EE276E080911F
:101C0000B2069091B3060E943F8BE091F40AE43053
:101C10000CF0E0E08AEB95E09A83898386EB95E00F
:101C20009C838B8381EB95E09E838D838CEA95E08A
:101C300098878F83EE0FFF0B81E090E08C0F9D1F44
:101C4000E80FF91F608171818091B2069091B3060F
:101C50000E94B08C0E947B6E68EF75E08091B206A6
:101C60009091B3060E94B08C0E947B6E6CEE75E082
:101C70008091B2069091B3060E943F8BE0919D1037
:101C8000F0919E1081819281883E934014F40E94CD
:101C90006B6EE0919D10F0919E1061817281809138
:101CA000B2069091B3060E94B33B84E00E940A946E
:101CB000E0919D10F0919E10658176818091B20631
:101CC0009091B3060E94B33B85E00E940A94E09194
:101CD0009D10F0919E10638174818091B206909165
:101CE000B3060E94B33B84E00E940A94E0919D10E9
:101CF000F0919E1067818091B2069091B3060E9488
:101D0000863A88E00E940A94E0919D10F0919E101E
:101D100080850E94576E60EE75E08091B2069091CA
:101D2000B3060E943F8BE091A710F091A81081812B
:101D30009281883E934014F40E946B6EE091A7104C
:101D4000F091A810618172818091B2069091B306E2
:101D50000E94B33B84E00E940A94E091A710F091A6
:101D6000A810658176818091B2069091B3060E9499
:101D7000B33B85E00E940A94E091A710F091A8106F
:101D8000638174818091B2069091B3060E94B33B47
:101D900084E00E940A94E091A710F091A810678156
:101DA0008091B2069091B3060E94863A88E00E9424
:101DB0000A94E091A710F091A81080850E94576EB8
:101DC00064ED75E08091B2069091B3060E943F8B5E
:101DD000E091B110F091B21081819281883E9340E0
:101DE00014F40E946B6EE091B110F091B210618119
:101DF00072818091B2069091B3060E94B33B84E059
:101E00000E940A94E091B110F091B2106581768140
:101E10008091B2069091B3060E94B33B85E00E9488
:101E20000A94E091B110F091B210638174818091B5
:101E3000B2069091B3060E94B33B84E00E940A94DC
:101E4000E091B110F091B21067818091B20690914B
:101E5000B3060E94863A88E00E940A94E091B1108D
:101E6000F091B21080850E94576E68EC75E0809109
:101E7000B2069091B3060E943F8BE091BB10F091A7
:101E8000BC1081819281883E934014F40E946B6E55
:101E9000E091BB10F091BC10618172818091B2061B
:101EA0009091B3060E94B33B84E00E940A94E091B3
:101EB000BB10F091BC10658176818091B206909143
:101EC000B3060E94B33B85E00E940A94E091BB10E8
:101ED000F091BC10638174818091B2069091B30639
:101EE0000E94B33B84E00E940A94E091BB10F09101
:101EF000BC1067818091B2069091B3060E94863A29
:101F000088E00E940A94E091BB10F091BC1080859B
:101F10000E94576E8091B2069091B3060E949D8CEC
:101F20000E949D80C82E60E676E08091B206909176
:101F3000B3060E94B08C0E947B6E0CE310E1E12C92
:101F4000F12CD12C57012FEFA21AB20AB5018091C2
:101F5000B2069091B3060E94B33B49E0E416F10447
:101F600010F48BE001C08AE00E940A94D8012C9101
:101F70008091B2069091B3062223C9F11596ED9196
:101F8000FC911697618172810E94B33BD80115962E
:101F9000ED91FC91169781819281883E934014F4D3
:101FA0000E946B6E84E00E940A94D8011596ED9110
:101FB000FC911697638174818091B2069091B3066B
:101FC0000E94B33B84E00E940A94D8011596ED91DB
:101FD000FC91169727818091B2069091B306222337
:101FE00019F068E576E00BC061E576E008C0EC1416
:101FF000FD041CF469E476E002C06CE376E00E9424
:10200000B08C095F1F4F7501BCE0AB16B10409F03D
:1020100099CF0E947B6E65E976E08091B20690913F
:10202000B3060E943F8B0E949D80682F8091B2066C
:102030009091B3060E946F3A61E876E08091B20613
:102040009091B3060E943F8B6091F10A7091F20A61
:102050008091B2069091B3060E94E93B0E940291E2
:102060008091B2069091B306DC01ED91FC9102845F
:10207000F385E02D19958091B2069091B3060E94E8
:102080009D8C0E947B6E65E677E08091B206909110
:10209000B3060E94B08C0E947B6E61E577E0809170
:1020A000B2069091B3060E943F8B8091E20E0E948F
:1020B0007572BC018091B2069091B3060E943F8B6D
:1020C0008091E20E8A30C1F46FE377E08091B2062E
:1020D0009091B3060E943F8B6091960F8091B2065B
:1020E0009091B3060E94863A68E377E08091B20649
:1020F0009091B3060E943F8B8091B2069091B306F7
:102100000E949D8C64E277E08091B2069091B306C4
:102110000E943F8B8091E30E0E947572BC018091FA
:10212000B2069091B3060E943F8B2091E30E8091FE
:10213000B2069091B3062B303CF4293054F4283089
:1021400069F463E177E007C02B3041F46FE177E099
:1021500002C069E177E00E94B08C02C00E949D8CB1
:102160006FEF76E08091B2069091B3060E943F8BAC
:102170008091E40E0E947572BC018091B20690912C
:10218000B3060E943F8B2091E40E8091B20690919D
:10219000B3062B303CF4293054F4283069F46EEE49
:1021A00076E007C02B3041F46AEF76E002C064EFBE
:1021B00076E00E94B08C02C00E949D8C6AED76E0B1
:1021C0008091B2069091B3060E943F8B2091F60E4B
:1021D0008091B2069091B306222319F062ED76E069
:1021E00002C060EC76E00E943F8B2091A6118091A6
:1021F000B2069091B306222319F065EB76E002C097
:1022000069EA76E00E943F8B8091B2069091B30616
:102210000E949D8C0E9402918091B2069091B3061B
:10222000DC01ED91FC910284F385E02D19958091FC
:102230000002823011F00C949D19F090130F009160
:10224000160F10E08091B2069091B3060E949D8C0B
:102250000E947B6E6EE27AE08091B2069091B306A6
:102260000E94B08C0E947B6E65E17AE08091B2069C
:102270009091B3060E943F8BE091230FE6300CF063
:10228000E0E08AEA97E09A83898385EA97E09C8375
:102290008B838BE997E09E838D8387E997E098870E
:1022A0008F8383E897E09A87898781E797E09C8707
:1022B0008B87EE0FFF0B81E090E08C0F9D1FE80FE6
:1022C000F91F608171818091B2069091B3060E94DE
:1022D000B08C6CEF79E08091B2069091B3060E94C9
:1022E0003F8B609100028091B2069091B3060E94EC
:1022F0006F3A63EE79E08091B2069091B3060E9446
:102300003F8B8F2D0E94426EFF2009F44AC069ED79
:1023100079E08091B2069091B3060E943F8B809144
:10232000B2069091B306112339F060910E0F0E940E
:10233000863A90910E0F06C06091140F0E94863A63
:102340009091140F809188139813FEC76DEB79E07C
:102350008091B2069091B3060E943F8B8091B206A5
:102360009091B306112339F060910F0F61110CC0E9
:1023700068EB79E006C06091150F611105C063EB51
:1023800079E00E943F8B05C0062E000C770B0E945F
:10239000B33B61EB79E08091B2069091B3060E9465
:1023A0003F8B8091B2069091B3060E949D8C68E9A4
:1023B00079E08091B2069091B3060E943F8B802F06
:1023C0000E94426E002309F44AC06EE879E08091D1
:1023D000B2069091B3060E943F8B8091B206909115
:1023E000B306112339F06091110F0E94863A909143
:1023F000110F06C06091170F0E94863A9091170F37
:1024000080918A139813BAC762E779E08091B20687
:102410009091B3060E943F8B8091B2069091B306D3
:10242000112339F06091120F61110CC06DE679E053
:1024300006C06091180F611105C068E679E00E943E
:102440003F8B05C0062E000C770B0E94B33B66E65F
:1024500079E08091B2069091B3060E943F8B809103
:10246000B2069091B3060E949D8C6DE479E0809154
:10247000B2069091B3060E943F8B80912C0F811180
:1024800003C00E94506E35C062EB77E08091B206C7
:102490009091B3060E943F8B6AE479E08091B20686
:1024A0009091B3060E943F8B60912C0F8091B206F1
:1024B0009091B3060E94863A6AE379E08091B20671
:1024C0009091B3060E943F8B40912D0F50912E0F9B
:1024D00060E070E02AE08091B2069091B3060E941D
:1024E000788B65E379E08091B2069091B3060E9403
:1024F000B08C6CE179E08091B2069091B3060E94B5
:102500003F8B8091240F8436C8F465E179E0809197
:10251000B2069091B3060E943F8B6091240F809188
:10252000B2069091B3060E94863A63E179E0809109
:10253000B2069091B3060E94B08C03C080E00E9466
:10254000506E6AEF78E08091B2069091B3060E94D7
:102550003F8B8091250F8436C8F463EF78E080913B
:10256000B2069091B3060E943F8B6091250F809137
:10257000B2069091B3060E94863A61EF78E08091AE
:10258000B2069091B3060E94B08C03C080E00E9416
:10259000506E68ED78E08091B2069091B3060E948B
:1025A0003F8B2091AB068091B2069091B306222317
:1025B00019F061ED78E002C067EC78E00E94B08C21
:1025C0006EEA78E08091B2069091B3060E943F8B4C
:1025D00060911A0F70911B0F072E000C880B990B3E
:1025E0000E942EBA20E030E04AE754E40E9404B68C
:1025F000AB01BC0121E08091B2069091B3060E942C
:10260000C08B69EA78E08091B2069091B3060E948F
:10261000B08C60E978E08091B2069091B3060E9498
:102620003F8B60911C0F70911D0F072E000C880BC3
:10263000990B0E942EBA20E030E04AE754E40E9451
:1026400004B6AB01BC0121E08091B2069091B306C3
:102650000E94C08B6BE878E08091B2069091B3063F
:102660000E94B08C62E778E08091B2069091B30648
:102670000E943F8B60911E0F70911F0F072E000C60
:10268000880B990B0E942EBA20E030E04AE754E410
:102690000E9404B6AB01BC0121E08091B20690918A
:1026A000B3060E94C08B6DE678E08091B2069091EF
:1026B000B3060E94B08C64E578E08091B2069091F8
:1026C000B3060E943F8B9091230F913011F094300C
:1026D000F9F48091200F0E94426E8091200F882390
:1026E00029F160E578E08091B2069091B3060E94EE
:1026F0003F8B6091210F8091B2069091B3060E94AA
:10270000863A6EE478E08091B2069091B3060CC0F0
:102710002091B2063091B306953019F461E478E067
:1027200002C06CE278E0C9010E943F8B8091B20642
:102730009091B3060E949D8C63E178E08091B2068F
:102740009091B3060E943F8B9091230F2FEF290F9A
:102750008091B2069091B306223028F46091100661
:102760000E946F3A04C06EEF77E00E94B08C65EE75
:1027700077E08091B2069091B3060E943F8B8091E2
:10278000300F0E94426E8091300F882341F163ED3B
:1027900077E08091B2069091B3060E943F8B6091E2
:1027A000310F8091B2069091B3060E94863A6BEB8E
:1027B00077E08091B2069091B3060E943F8B6091C2
:1027C000320F8091B2069091B3060E94863A69EB6F
:1027D00077E08091B2069091B3060E943F8B809182
:1027E000B2069091B3060E949D8C0E940291809146
:1027F000B2069091B306DC01ED91FC910284F38561
:10280000E02D19958091B2069091B3060E949D8C9F
:102810000E947B6E67EB7AE08091B2069091B306DE
:102820000E94B08C0E947B6E66E97AE08091B206CD
:102830009091B3060E943F8B8091EB0E8436C8F4D2
:102840006FE87AE08091B2069091B3060E943F8BC8
:102850006091EB0E8091B2069091B3060E94863A89
:102860006DE87AE08091B2069091B3060E94B08C38
:1028700003C080E00E94506E6CE67AE08091B20660
:102880009091B3060E943F8B8091EA0E8436C8F483
:1028900065E67AE08091B2069091B3060E943F8B84
:1028A0006091EA0E8091B2069091B3060E94863A3A
:1028B00063E67AE08091B2069091B3060E94B08CF4
:1028C00003C080E00E94506E62E47AE08091B2061C
:1028D0009091B3060E943F8B6091F80E7091F90EB3
:1028E0001616170614F50091B2061091B306072EBE
:1028F000000C880B990B0E942EBA20E030E04AE7CA
:1029000054E40E9404B6AB01BC0122E0C8010E945D
:10291000C08BC8010E949D8C6DE37AE08091B20665
:102920009091B3060E94B08C03C080E00E94506E6C
:102930000E9402918091B2069091B306DC01ED9164
:10294000FC910284F385E02D19958091B206909157
:10295000B3060E949D8C0E947B6E6CE27CE08091AD
:10296000B2069091B3060E94B08C0E947B6E2091BB
:1029700032068091B2069091B306222309F4C3C1B6
:102980006DEF7BE00E943F8B0E9452680E94506E68
:102990000E9452682091B2063091B306882389F0D4
:1029A0006AEE7BE0C9010E943F8B809135060E9450
:1029B0001A63BC018091B2069091B3060E94B08C5C
:1029C0004FC067ED7BE0C9010E943F8B80913206CA
:1029D0000E941A63BC018091B2069091B3060E94D6
:1029E0003F8B809133068823A9F16FEC7BE08091C7
:1029F000B2069091B3060E943F8BE0913306E4301B
:102A00000CF0E0E088E793E09A83898386E793E01F
:102A10009C838B8384E793E09E838D8382E793E09E
:102A200098878F83EE0FFF0B81E090E08C0F9D1F46
:102A3000E80FF91F608171818091B2069091B30611
:102A40000E943F8B6DEC7BE08091B2069091B306C3
:102A50000E943F8B8091B2069091B3060E949D8C9C
:102A60006AEB7BE08091B2069091B3060E943F8BA7
:102A7000809134060091B2061091B306882321F0AC
:102A80000E941A63BC0102C066EB7BE0C8010E9491
:102A9000B08C63EA7BE08091B2069091B3060E940D
:102AA0003F8B809135060091B2061091B3068823C2
:102AB00021F00E941A63BC0102C06FE97BE0C801EB
:102AC0000E94B08C6CE87BE08091B2069091B306D6
:102AD0000E943F8B809137068823E1F066E87BE017
:102AE0008091B2069091B3060E943F8B809136068A
:102AF0000E941A63BC018091B2069091B3060E94B5
:102B00003F8B6AEF75E08091B2069091B3060E9408
:102B1000A08C03C080E00E94506E63E77BE0809150
:102B2000B2069091B3060E943F8B809138068823AD
:102B3000E1F06DE67BE08091B2069091B3060E94D1
:102B40003F8B809136060E941A63BC018091B206C9
:102B50009091B3060E943F8B6AEF75E08091B206B8
:102B60009091B3060E94A08C03C080E00E94506E3A
:102B70006AE57BE08091B2069091B3060E943F8B9C
:102B8000E0913906E3300CF0E3E082E09BE09A83C9
:102B9000898386EF9AE09C838B8381EF9AE09E8302
:102BA0008D8389EE9AE098878F83EE0FFF0BA1E06B
:102BB000B0E0AC0FBD1FEA0FFB1F608171818091F7
:102BC000B2069091B3060E94B08C67E47BE08091DE
:102BD000B2069091B3060E943F8BE0912B06E43041
:102BE0000CF0E4E082EE9AE09A8389838CED9AE01F
:102BF0009C838B8385ED9AE09E838D838FEC9AE096
:102C000098878F8387EC9AE09A878987EE0FFF0B6E
:102C100081E090E08C0F9D1FE80FF91F60817181AA
:102C20008091B2069091B3060E94B08C65E47BE07F
:102C30008091B2069091B3060E943F8B609130065E
:102C40008091B2069091B3060E94863A66E37BE0DB
:102C50008091B2069091B3060E943F8B80912B0623
:102C6000811110C0609131068091B2069091B30637
:102C70000E94863A6BE27BE08091B2069091B306A7
:102C80000E943F8B60912C0670912D06072E000C40
:102C9000880B990B0E942EBA20E030E04AE754E4FA
:102CA0000E9404B6AB01BC0121E08091B206909174
:102CB000B3060E94C08B6DE17BE08091B2069091DB
:102CC000B3060E943F8B60912E0670912F06072E4F
:102CD000000C880B990B0E942EBA20E030E04AE7E6
:102CE00054E40E9404B6AB01BC0121E08091B2061D
:102CF0009091B3060E94C08B6EE07BE08091B2069B
:102D00009091B30602C060E17CE00E94B08C0E940A
:102D100002918091B2069091B306DC01ED91FC9195
:102D20000284F385E02D19958091B2069091B30647
:102D30000E949D8C0E947B6E6AEA7CE08091B206C4
:102D40009091B3060E94B08C0E947B6E6DE97CE08E
:102D50008091B2069091B3060E943F8BE091390FAB
:102D6000E5300CF0E5E08BE89CE09A83898384E70A
:102D70009CE09C838B8382E69CE09E838D8383E52D
:102D80009CE098878F8380E49CE09A87898788E31A
:102D90009CE09C878B87EE0FFF0B81E090E08C0F0F
:102DA0009D1FE80FF91F608171818091B20690919B
:102DB000B3060E94B08C0E9402918091B20690915D
:102DC000B306DC01ED91FC910284F385E02D1995A9
:102DD0008DE398E7A1E0BB278BAB9CABADABBEAB63
:102DE0008091B2069091B3060E949D8C0E947B6EEA
:102DF0006FEB7EE08091B2069091B3060E94B08C9A
:102E00000E947B6E66EA7EE08091B2069091B306E6
:102E10000E943F8B2091EF0A8091B2069091B306F9
:102E2000222319F062EA7EE002C06DE97EE00E9492
:102E3000B08C8091EF0A882349F164E87EE08091AC
:102E4000B2069091B3060E943F8B6091370F70914C
:102E5000380F072E000C880B990B0E942EBA20E029
:102E600030E04AE754E40E9404B6AB01BC0122E022
:102E70008091B2069091B3060E94C08B6FE77EE00E
:102E80008091B2069091B3060E94B08C9CE6E92E28
:102E90009EE0F92E29E2622E38E1232E3CEF332EFC
:102EA0004AE0A42EB12C54E6C52ED12CD7012C918A
:102EB000222309F400C2F701329700811181011524
:102EC000110509F4F8C18CE997E7A1E0BB27820F4F
:102ED000911DA11DB11DABBFFC0187917724739497
:102EE000811101C0712C2091B2063091B306C80146
:102EF0000197849790F56FE57EE0C9010E943F8BB2
:102F000009500C3148F4E02FF0E0EE0FFF1FE25EB5
:102F1000FD4F6081718102C065EB7CE08091B2065B
:102F20009091B3060E943F8B0C3130F4E02FF0E01B
:102F3000EA5AFD4F808101C080E090E08B5A914FAA
:102F4000092E000CAA0BBB0BABBFFC0187919EE0C6
:102F5000981B892F09F051C152C1C80184569109AB
:102F60008438934008F03FC065E47EE0C9010E94C8
:102F70003F8BC801B6010E9464B56130710531F024
:102F80006230710559F461E47EE002C063E47EE0E2
:102F90008091B2069091B3060E943F8B0E94736E9F
:102FA0008090B2069090B3067720B1F0C8010E94DD
:102FB000438F811107C06DE37EE0C4010E943F8B07
:102FC00087E01BC1813009F01AC16AE37EE0C401C9
:102FD0000E943F8B88E011C161E37EE0C4010E9442
:102FE0003F8B82E00AC1C801885E934080359644D9
:102FF00008F05AC0C80168EE73E00E9464B54B0146
:1030000064E27EE0C9010E943F8BFAE08F169104D2
:1030100010F40E946B6EB4018091B2069091B306D9
:103020000E94B33B0E94736E4090B2065090B3066C
:103030007720A1F1C8010E94438F782E6FE17EE0D6
:10304000C2010E943F8B672D8091B2069091B3061A
:103050000E94863A69E17EE08091B2069091B306C3
:103060000E943F8B829CC001839C900D929C900D8E
:103070001124800F911FB5010E9478B577278091A8
:10308000B2069091B3060E94B33B67E17EE0809167
:10309000B2069091B3060E943F8BB1C06EE07EE015
:1030A000C2010E943F8B61C0F801E853FA44E83E38
:1030B00043E0F40708F046C0EC30F10508F09FC08B
:1030C0008827EE58FF4F8F4F0C948BB56FEF7DE044
:1030D00019C064EF7DE0C9010E943F8B83E18DC080
:1030E00062EE7DE027C062ED7DE016C065EC7DE01C
:1030F00055C069EB7DE0C9010E943F8B82E17DC034
:103100006AEA7DE0C9010E943F8B8FE076C06BE9DF
:103110007DE0F8CF6BE87DE0C9010E943F8B8EE037
:103120006CC068E77DE0C9010E943F8B8BE065C001
:1031300066E67DE0C9010E943F8B8CE05EC069E5D8
:103140007DE02CC0C80180529E44883E934078F4B4
:10315000005262E47DE0C9010E943F8B0A3010F406
:103160000E946B6E802F0E94336E84E046C0C801BF
:1031700088509245883E934020F408506BE27DE0F1
:10318000EACF013FE5E51E0719F46AE17DE01CC0C6
:10319000023FF5E51F0739F46DE07DE0C9010E94AB
:1031A0003F8B81E12AC0033F45E5140739F46FEFF7
:1031B0007CE0C9010E943F8B80E11FC0043F85E590
:1031C000180739F46EEE7CE0C9010E943F8B8DE058
:1031D00014C0053F95E5190739F466ED7CE0C90197
:1031E0000E943F8B86E009C0063F154541F46DEB18
:1031F0007CE0C9010E943F8B85E00E940A946AE747
:103200007EE08091B2069091B3060E943F8B6FE6FC
:103210007EE08091B2069091B3060E943F8BF70149
:10322000608170E08091B2069091B3060E94B33B3A
:10323000D7018C918A3020F482E00E940A9404C065
:10324000843610F40E946B6E0E94736EF701408109
:10325000649EA0011124052E000C660B770B8BA930
:103260009CA9ADA9BEA9480F591F6A1F7B1FDE018B
:1032700011968A019B010F5F1F4F2F4F3F4F6BBF6E
:10328000FA0187918D93B901A8018111F2CFBE0196
:103290006F5F7F4F8091B2069091B3060E94A08C21
:1032A0008091B2069091B306DC01ED91FC9102840D
:1032B000F385E02D1995B3E0EB0EF11CE4EEEE166C
:1032C000EEE0FE0609F0F2CD0E9402918091B20676
:1032D0009091B306DC01ED91FC910284F385E02D21
:1032E00019958091B2069091B3060E949D8C0E9420
:1032F0007B6E60E27FE08091B2069091B3060E94FF
:10330000B08C0E947B6E6DE07FE08091B206909160
:10331000B3060E943F8B0E94498520E030E040E0E8
:1033200050E40E9428BA2091B2063091B30687FF7C
:103330003EC06AE07FE0C90158C0F0900D0F0091D7
:10334000100F11E00C9422116AEC79E08091B20622
:103350009091B3060E943F8B609188138091B206D2
:103360009091B3060E94863A68EC79E08091B206AB
:103370009091B3060E943F8B0C94A6116FE779E001
:103380008091B2069091B3060E943F8B60918A13A0
:103390008091B2069091B3060E94863A6DE779E07B
:1033A0008091B2069091B3060E943F8B2DC866E0D3
:1033B0007FE0C9010E94B08C63EF7EE08091B2068D
:1033C0009091B3060E943F8B0E944985AB01BC01DE
:1033D00022E08091B2069091B3060E94C08B61EF0B
:1033E0007EE08091B2069091B3060E94B08C6EEDA3
:1033F0007EE08091B2069091B3060E943F8B80914F
:10340000830F0E94426E2091830F8091B2069091AB
:10341000B306222379F06BED7EE00E943F8B0E9481
:10342000489461ED7EE08091B2069091B3060E94CF
:10343000B08C02C00E949D8C0E9402918091B206C5
:103440009091B306DC01ED91FC910284F385E02DAF
:1034500019958091B2069091B3060E949D8C0E94AE
:103460007B6E68E77FE08091B2069091B3060E9480
:10347000B08C0E947B6E64E67FE08091B2069091F2
:10348000B3060E943F8B4091730F5091740F60916F
:10349000750F7091760F8091B2069091B3060E94DD
:1034A000A03B60E57FE08091B2069091B3060E9458
:1034B0003F8B40917B0F50917C0F60917D0F7091FD
:1034C0007E0F8091B2069091B3060E94A03B6CE300
:1034D0007FE08091B2069091B3060E943F8B4091AD
:1034E000770F5091780F6091790F70917A0F8091DA
:1034F000B2069091B3060E94A03B68E27FE0809103
:10350000B2069091B3060E943F8B40917F0F50917D
:10351000800F6091810F7091820F8091B20690911F
:10352000B3060E94A03B0E9402918091B206909146
:10353000B306DC01ED91FC910284F385E02D199531
:103540008091B2069091B3060E949D8C0E947B6E82
:10355000E6960FB6F894DEBF0FBECDBFDF91CF91D8
:103560001F910F91FF90EF90DF90CF90BF90AF90A1
:103570009F908F907F906F905F904F903F902F9093
:1035800008952F923F924F925F926F927F928F9207
:103590009F92AF92BF92CF92DF92EF92FF920F93E2
:1035A0001F93CF93DF93CDB7DEB7AB970FB6F894E9
:1035B000DEBF0FBECDBF83ED91E00E9459BB6338E3
:1035C000714F8105910519F00E94576408C047EDBD
:1035D00051E060E070E085EC9DE00E9441BB40E07E
:1035E00052EC61E070E087ED98E00E941871409124
:1035F000770F5091780F6091790F70917A0F8AE36D
:1036000098E00E94187140917B0F50917C0F60915F
:103610007D0F70917E0F8DE997E00E9418714091A7
:103620007F0F5091800F6091810F7091820F80E029
:1036300097E00E94187189EA9DE09093FE068093BE
:10364000FD068AE69BE09093FC068093FB0687EDDF
:1036500098E090939B1380939A131092C711109245
:10366000AE0D1092AB0D1092AD0D1092AC0D11E09D
:103670001093B6120E94E7448091970F8093B5068D
:103680001092B4061092800082E0809381008FE255
:1036900086BB10926F0010928500109284009BE20E
:1036A0009093A00099E09093A10089BB10927200C2
:1036B0001092A5001092A4001092A9001092A800E8
:1036C0001092AB001092AA001092AD001092AC00C4
:1036D00099EA90932001109321018ABB1092730004
:1036E00010922501109224011092290110922801B4
:1036F00010922B0110922A0110922D0110922C0190
:103700008091620E9091630E8093460690934706D7
:10371000813001F58FE38093120B1092130B61E05F
:103720000E94C74788E09BE00E9434921092140BDD
:103730001092170B1092160B80914706882329F0E0
:1037400088E09BE00E94F79311C088E09BE00E9414
:10375000E0930CC080914706882311F062E001C01D
:1037600060E08FE30E94C7470E94C5418091640ECC
:103770009091650E80934C0690934D06813001F533
:103780008EE38093430B1092440B61E00E94C74785
:1037900089E39BE00E9434921092450B1092480BF3
:1037A0001092470B80914D06882329F089E39BE016
:1037B0000E94F79311C089E39BE00E94E0930CC044
:1037C00080914D06882311F062E001C060E08EE335
:1037D0000E94C7470E94924160E085E40E94C7476B
:1037E00062E08CE30E94C74762E08BE30E94C74718
:1037F00062E080E40E94C74762E081E40E94C7471C
:1038000062E082E40E94C74762E081E20E94C7470B
:1038100062E084E40E94C74761E089E30E94C747F1
:1038200061E08AE30E94C7470E9402840E943984B3
:1038300061E085E30E94C74761E085E00E94C747D9
:1038400061E070E085E00E94034861E084E00E944E
:10385000C74761E087E00E94C74761E089E20E94B4
:103860005D4661E089E20E94C7476A9A60E085E3AD
:103870000E945D4660E085E00E945D4660E084E075
:103880000E945D4660E087E00E945D46729861E0BC
:1038900088E00E94C74780E090E09C012B53324FA4
:1038A000F901E955FF4F40814F3629F432972081C5
:1038B0003181232B31F403968837910571F760E04D
:1038C00001C061E088E00E945D4661E08BE20E94F9
:1038D000C74760E08BE20E945D460E9439840E94E7
:1038E000313B8091F80A813009F06CC08091FB0A6D
:1038F0009091FC0AA091FD0AB091FE0A4091FF0A46
:103900005091000B6091010B7091020B841B950B81
:10391000A60BB70B84379E40A105B10500F30E94AA
:1039200057648091B2069091B3060E949D8C80915D
:10393000B2069091B3060E949D8C0E947B6E66E851
:103940007FE08091B2069091B3060E943F8B01E028
:1039500010E00E9406840E9439846EEE72E080E0DE
:1039600090E00E94534A63E87FE08091B206909114
:10397000B3060E943F8B0E9402840E94358405306A
:10398000110531F064EF71E080E090E00E94534A4D
:103990000F5F1F4F06301105E1F68091B20690913E
:1039A000B3060E949D8C0E947B6E8091B20690911E
:1039B000B3060E949D8C8091B2069091B3060E943E
:1039C0009D8C02C081118BCF80916F0082608093AB
:1039D0006F0080918400909185008056904F909365
:1039E0008900809388000E9408298BE69BE09093D1
:1039F000EF118093EE111091320F2091310F8091D1
:103A0000200F9091220F3091230F3093FF06909357
:103A100010068093110630E0AFEFB0E00E94BFBB0C
:103A200024E630E040E050E00E9471BB2093911307
:103A3000612F70E080E090E00E942CBA23EC34E625
:103A40004AEA5AE30E948DBA2AE939E949E55FE377
:103A50000E94A0B560938B1370938C1380938D1389
:103A600090938E13109295001092940010929000F3
:103A70008CE08093910084EF90E090939900809384
:103A8000980011E018BB82E08093710080910002E1
:103A90000E9482448091B2069091B3062091B506AF
:103AA00040911C0F50911D0F50937E1340937D1336
:103AB000209381119093801180937F1110921206B0
:103AC00010937F138091390F853040F01092390F99
:103AD00060E070E084E791E00E94C23A1091390FF3
:103AE000123009F444C008F5112309F466C01130FE
:103AF00009F05BC08CE090E00E9428B722E433E03C
:103B0000DC0111963C932E932DE937E01B963C93F4
:103B10002E931A979093AF068093AE061093A1123E
:103B20001093A4121093A71267C0133009F45EC05B
:103B30001430D9F586E090E00E9428B78C0128EA7D
:103B400033E0DC012D933D93CD0141E06BE67BE05A
:103B50000E94B86086E792E0F80191838083109319
:103B6000AF060093AE0681E08093A11241C086E0CB
:103B700090E00E9428B72CED32E0FC0131832083D5
:103B80009093AF068093AE068FB7F8942CED35E096
:103B90003093BF102093BE101092C4108FBF81E0ED
:103BA0008093A1128093A41225C01092390F60E077
:103BB00070E084E791E00E94C23A86E090E00E94C3
:103BC00028B78C0128EA33E0DC012D933D93CD0129
:103BD00040E06BE67BE00E94B86086E792E0F80187
:103BE000918380831093AF060093AE061092A112CA
:103BF0001092A4121092A7128091AE069091AF0677
:103C0000DC01ED91FC910190F081E02D19958091FE
:103C1000951281111FC08091981281111BC0809153
:103C20009B12811117C080919E12811113C0809147
:103C3000A11281110FC08091A41281110BC080913B
:103C4000A712811107C081E00E94E344882309F490
:103C500018C310C3A12CB12C612C912C1DA2712C66
:103C6000812C412C512C0AEE15E0EE24EA94A3E0BD
:103C7000FA2ECC24CA94DD24D3948EED282E85E030
:103C8000382EC5018B53924FFC01E955FF4FE0815F
:103C9000EE2309F4E6C2DC01AB55BF4F8D919C9138
:103CA000892B09F4DEC28E2F90E0FC01F797EB32EE
:103CB000F10508F0D6C28827E258FF4F8F4F0C94C9
:103CC0008BB580919512882309F4CBC25110C9C2DB
:103CD00089E190E00E9428B79C01FC0111830083D8
:103CE00087E090E09383828315821482F782E682D4
:103CF000D186C086108EC9012AA73BA70E94887E64
:103D00002AA53BA5E2E3F4E0D901ED93FC933093BF
:103D1000861220938512C9010E9435767DC180915B
:103D20009812882309F49DC241109BC289E190E05A
:103D30000E9428B79C01DC0111961C930E93E6E0CB
:103D4000F0E01396FC93EE93129715961C921E9238
:103D500014971796FC92EE9216971996DC92CE92D3
:103D6000189758961C922AA73BA70E94887E2AA5DE
:103D70003BA5E2E3F4E0D901ED93FC933093881284
:103D800020938712C9010E94357674C180919B12DD
:103D9000882309F466C2811064C289E190E00E9420
:103DA00028B79C01DC0111961C930E93E5E0F0E02E
:103DB0001396FC93EE93129715961C921E921497ED
:103DC0001796FC92EE9216971996DC92CE9218975F
:103DD00058961C922AA73BA70E94887E2AA53BA53D
:103DE000E2E3F4E0D901ED93FC9330938A1220933F
:103DF0008912C9010E9435766BC180919E12882379
:103E000009F42FC271102DC289E190E00E9428B7F9
:103E10009C01DC0111961C930E93E4E0F0E01396F4
:103E2000FC93EE93129715961C921E921497179678
:103E3000FC92EE9216971996DC92CE9218975896AD
:103E40001C922AA73BA70E94887E2AA53BA5E2E3F5
:103E5000F4E0D901ED93FC9330938C1220938B12F4
:103E6000C9010E94357662C18091A112882309F4AC
:103E7000F8C12DA12111F5C189E190E00E9428B778
:103E80009C01DC0111961C930E93E2E0F0E0139686
:103E9000FC93EE93129715961C921E921497179608
:103EA000FC92EE9216971996DC92CE92189758963D
:103EB0001C922AA73BA70E94887E2AA53BA5E2E385
:103EC000F4E0D901ED93FC9330938E1220938D1280
:103ED000C9010E94357662C18091A412882309F439
:103EE000C0C19110BEC189E190E00E9428B79C0139
:103EF000DC0111961C930E93E1E0F0E01396FC9325
:103F0000EE93129715961C921E9214971796FC9298
:103F1000EE9216971996DC92CE92189758961C92AC
:103F20002AA73BA70E94887E2AA53BA5E2E3F4E0EE
:103F3000D901ED93FC933093901220938F12C90115
:103F40000E94357662C18091A712882309F489C145
:103F5000611087C189E190E00E9428B79C01DC01D3
:103F600011961C930E9313961C921E9212971596FF
:103F70001C921E9214971796FC92EE921697199621
:103F8000DC92CE92189758961C922AA73BA70E94C3
:103F9000887E2AA53BA582E394E0F9019183808382
:103FA0003093921220939112C9010E94357657C125
:103FB00080919512882309F454C1511052C18CE1AB
:103FC00090E00E9428B79C01DC0111961C930E938F
:103FD000E7E0F0E01396FC93EE93129715961C928F
:103FE0001E9214971796FC92EE9216971996DC92F1
:103FF000CE92189758961C922AA73BA70E94887EBB
:104000002AA53BA5D9012D923C923093941220937E
:104010009312C9010E94F1765524539422C18091D4
:104020009812882309F41DC141101BC18CE190E056
:104030000E9428B79C01FC011183008386E090E078
:104040009383828315821482F782E682D186C086AA
:10405000108EC9012AA73BA70E94887E2AA53BA5EE
:10406000D9012D923C923093971220939612C90158
:104070000E94F17644244394F4C080919B128823DB
:1040800009F4EFC08110EDC08CE190E00E9428B7E8
:104090009C01FC011183008385E090E0938382837F
:1040A00015821482F782E682D186C086108EC901FD
:1040B0002AA73BA70E94887E2AA53BA5D9012D925D
:1040C0003C9230939A1220939912C9010E94F17682
:1040D00088248394C6C080919E12882309F4C1C0AD
:1040E0007110BFC08CE190E00E9428B79C01FC01D8
:1040F0001183008384E090E093838283158214828D
:10410000F782E682D186C086108EC9012AA73BA716
:104110000E94887E2AA53BA5D9012D923C9230931E
:104120009D1220939C12C9010E94F176772473940A
:1041300098C08091A112882309F493C02DA1211168
:1041400090C08CE190E00E9428B79C01DC011196A0
:104150001C930E93E2E0F0E01396FC93EE9312971B
:1041600015961C921E9214971796FC92EE92169733
:104170001996DC92CE92189758961C922AA73BA7C4
:104180000E94887E2AA53BA5D9012D923C923093AE
:10419000A01220939F12C9010E94F17621E02DA365
:1041A00060C08091A412882309F45BC0911059C0AB
:1041B0008CE190E00E9428B79C01DC0111961C93D1
:1041C0000E93E1E0F0E01396FC93EE9312971596B0
:1041D0001C921E9214971796FC92EE9216971996BF
:1041E000DC92CE92189758961C922AA73BA70E9461
:1041F000887E2AA53BA5D9012D923C923093A3122B
:104200002093A212C9010E94F1769924939429C0A7
:104210008091A712882329F1611023C08CE190E0DE
:104220000E9428B79C01FC01118300831382128233
:1042300015821482F782E682D186C086108E2AA764
:104240003BA70E94887E2AA53BA5D9012D923C92CE
:104250003093A6122093A512C9010E94F17666241C
:104260006394B3E0AB0EB11CE8E7AE16B10409F0FD
:1042700008CDE9CC82E00E94E344882311F01FA21C
:1042800016C081E00E94E344882329F082E00E9466
:10429000C744811178C78CE30E948F8E892B09F067
:1042A00063C78CE30E948F8E892B09F063C786E079
:1042B000E9E6FFE0DE01549601900D928A95E1F760
:1042C000B090620F0091720F1091630F7091640FA4
:1042D0006091650F5091660F4091670F3091680FA4
:1042E00020916F0F8091700F9091710FA091AE0689
:1042F000B091AF06BEA3ADA3E0911B12F0911C12CA
:10430000F9A7E8A79090950F6090900FE090890F23
:10431000F0908A0F8090930F7090920FC090F80EDB
:10432000D090F90E5090FB0E4090F60E3090F70EA4
:10433000FFA1FB8BBA8E0B8F1C8F7D8F6E8F5F8FD3
:1043400048A339A32AA39CA38BA3F2E1AF2EFE01BD
:104350007396DE01119601900D92AA94E1F7EBE6B7
:10436000FBE0F0931B06E0931A06AFA1A983B88681
:1043700009871A877B876C875D874E873F87288BE5
:104380009A8B898B82E1FE013196ABE2B6E0019017
:104390000D928A95E1F73092A6114092A7115092A2
:1043A0008312D0927C12C0927B1260921D12709286
:1043B000801280927F12F0927E12E0927D12909293
:1043C000841288A599A590938212809381128DA161
:1043D0009EA190931D0680931C0687E08093F809A8
:1043E0001092F90961E00E94C7478EEE99E00E94A1
:1043F00034921092FA091092FD091092FC098091F2
:104400003606811102C01092370690913206911142
:1044100005C0811103C01092DF0A98C08091DA0AAA
:104420009091DB0A0E949B8881E08093DF0A809153
:104430002B06882359F1813071F08330C1F488E272
:1044400093E290932D0680932C0689E080933006AA
:1044500080E197E217C088EB9BE090932D06809354
:104460002C0683E08093300688E99AE30BC088E845
:1044700093E190932D0680932C0686E0809330067E
:1044800080EE9EE290932F0680932E068091320656
:104490008823E9F1809136066091300670E0882328
:1044A000C9F0809138068823A9F080E090E00E944E
:1044B0002CBA9B01AC0160E070E088EC92E40E94B1
:1044C00004B660931E0670931F0680932006909397
:1044D000210625C080E090E00E942CBA9B01AC012F
:1044E00060E070E088EC92E40E9404B660931E06DF
:1044F00070931F0680932006909321061092150654
:104500001092160610921706109218061FC01092ED
:104510001E0610921F06109220061092210660912E
:10452000310670E080E090E00E942CBA9B01AC0163
:1045300060E070E088EC92E40E9404B66093150697
:10454000709316068093170690931806109228060B
:104550001092220610921906109223061092240639
:1045600010922506109226060E94C6456E98769AED
:10457000EE9880916A008F7C80936A008091A711E9
:10458000882321F080916A00806203C080916A00D4
:10459000806380936A00EE980E94A54780E090E0D7
:1045A00040E09C012B53324FF901E955FF4F5081F8
:1045B000552331F0329720813181232B09F04F5F51
:1045C00003968837910569F740933F06AEE4B6E05D
:1045D00020E030E08EE2282E8EE6382E91EA492E39
:1045E00090E4592E46E7642E40E4742E59E8852E57
:1045F00050E4952E61E3A62E6EE6B62E4FE95CE6FA
:1046000005E81CE672E9E72E7CE6F72EEBEACE2EF3
:10461000EBE6DE2EC9018B53924FFC01E955FF4FAB
:104620006081662309F492C38B559F4FFC01808102
:104630009181892B09F48AC370E0FB013197E03A3C
:10464000F10508F083C38827E755FF4F8F4F0C947F
:104650008BB58DEE9EE811969C938E9377C38BEE6F
:104660009EE811969C938E9371C389EE9EE81196F5
:104670009C938E936BC382EE9EE811969C938E93CF
:1046800065C380EE9EE811969C938E935FC38AEC7F
:1046900097E511969C938E9359C38CEC97E51196F0
:1046A0009C938E9353C38DEA97E511969C938E93BA
:1046B0004DC389E997E511969C938E9347C38AE889
:1046C00097E511969C938E9341C38EE297E51196E0
:1046D0009C938E933BC382ED95E511969C938E93AC
:1046E00035C381E297E511969C938E932FC38CEA94
:1046F00096E511969C938E9329C386E197E51196D2
:104700009C938E9323C38FE197E511969C938E9390
:104710001DC388E197E511969C938E9317C38FED87
:1047200096E511969C938E9311C387E097E51196B9
:104730009C938E930BC380E097E511969C938E9388
:1047400005C38FEC96E511969C938E93FFC28DEC7A
:1047500096E511969C938E93F9C28BEC96E5119693
:104760009C938E93F3C28BEB96E511969C938E935C
:10477000EDC289EB96E511969C938E93E7C28AEA87
:1047800096E511969C938E93E1C28AE996E511967F
:104790009C938E93DBC288E996E511969C938E9349
:1047A000D5C286E996E511969C938E93CFC282EF8F
:1047B00093E511969C938E93C9C280EF93E5119671
:1047C0009C938E93C3C28EEE93E511969C938E9329
:1047D000BDC286EC92E811969C938E93B7C284E991
:1047E00096E511969C938E93B1C284E896E5119656
:1047F0009C938E93ABC285EC94E511969C938E931B
:10480000A5C286EA94E511969C938E939FC282E896
:1048100096E511969C938E9399C283E596E5119641
:104820009C938E9393C28CE496E511969C938E9301
:104830008DC28BE196E511969C938E9387C28CEF87
:104840009EE811969C938E9381C280ED95E511961A
:104850009C938E937BC28EEC95E511969C938E93E0
:1048600075C28BEC95E511969C938E936FC287EA87
:1048700095E511969C938E9369C283E895E5119610
:104880009C938E9363C288EC95E511969C938E93CE
:104890005DC284EA95E511969C938E9357C280E899
:1048A00095E511969C938E9351C285EC95E51196F2
:1048B0009C938E934BC281EA95E511969C938E93BF
:1048C00045C28DE795E511969C938E933FC282EC8D
:1048D00095E511969C938E9339C28EE995E51196D4
:1048E0009C938E9333C28AE795E511969C938E93A1
:1048F0002DC28FEB95E511969C938E9327C28BE981
:1049000095E511969C938E9321C287E795E51196C4
:104910009C938E931BC28CEB95E511969C938E9382
:1049200015C288E995E511969C938E930FC284E792
:1049300095E511969C938E9309C289EB95E51196A6
:104940009C938E9303C285E995E511969C938E9373
:10495000FDC181E795E511969C938E93F7C186EB97
:1049600095E511969C938E93F1C182E995E5119698
:104970009C938E93EBC18EE695E511969C938E9356
:10498000E5C183EB95E511969C938E93DFC18FE88B
:1049900095E511969C938E93D9C18BE695E511967A
:1049A0009C938E93D3C180EB95E511969C938E9347
:1049B000CDC18CE895E511969C938E93C7C188E68E
:1049C00095E511969C938E93C1C18DEA95E511965C
:1049D0009C938E93BBC189E895E511969C938E9329
:1049E000B5C185E695E511969C938E93AFC18AEA91
:1049F00095E511969C938E93A9C186E895E511964D
:104A00009C938E93A3C182E695E511969C938E9319
:104A10009DC18EE595E511969C938E9397C18AE58D
:104A200095E511969C938E9391C186E595E5119637
:104A30009C938E938BC182E595E511969C938E9302
:104A400085C18EE495E511969C938E937FC18AE48F
:104A500095E511969C938E9379C186E495E5119620
:104A60009C938E9373C182E495E511969C938E93EB
:104A70006DC189E395E511969C938E9367C18CEE89
:104A800093E511969C938E9361C18AEE93E51196FE
:104A90009C938E935BC18AE095E511969C938E93CF
:104AA00055C182E094E511969C938E934FC180E3AB
:104AB00095E511969C938E9349C188EE93E51196E6
:104AC0009C938E9343C186EE93E511969C938E93AF
:104AD0003DC184EE94E511969C938E9337C184E595
:104AE00094E511969C938E9331C18AE89DE61196C8
:104AF0009C938E932BC18FE39DE611969C938E938E
:104B000025C183ED90E411969C938E931FC18FEB8A
:104B100090E411969C938E9319C18BEA90E41196C0
:104B20009C938E9313C188EB9EE811969C938E9371
:104B30000DC182E69CE611969C938E9307C180E599
:104B40009CE611969C938E9301C189E99BE6119690
:104B50009C938E93FBC08FE49BE611969C938E935F
:104B6000F5C081E79BE611969C938E93EFC081E69A
:104B70009BE611969C938E93E9C083E89BE6119681
:104B80009C938E93E3C087E29BE611969C938E9351
:104B9000DDC087E19BE611969C938E93D7C089E395
:104BA0009BE611969C938E93D1C083E39DE611966C
:104BB0009C938E93CBC087E29DE611969C938E9337
:104BC000C5C08BE19DE611969C938E93BFC08FE08C
:104BD0009DE611969C938E93B9C083E09DE6119655
:104BE0009C938E93B3C087EF9CE611969C938E9313
:104BF000ADC08BEE9CE611969C938E93A7C087E187
:104C00009CE611969C938E93A1C085E09CE611963C
:104C10009C938E939BC083EF9BE611969C938E93FF
:104C200095C081EE9BE611969C938E938FC08FEC7E
:104C30009BE611969C938E9389C08DEB9BE6119613
:104C40009C938E9383C01196DC92CE927FC0119676
:104C5000FC92EE927BC011961C930E9377C085EC6C
:104C60009CE611969C938E9371C011965C934E9323
:104C70006DC01196BC92AE9269C011969C928E92B4
:104C800065C011967C926E9261C011965C924E92B4
:104C90005DC011963C922E9259C0EBE2FEE6119651
:104CA000FC93EE9353C082E29EE611969C938E9302
:104CB0004DC0EFE1FEE61196FC93EE9347C08CE108
:104CC0009EE611969C938E9341C0E9E1FEE6119613
:104CD000FC93EE933BC086E19EE611969C938E93E7
:104CE00035C0EBE0FEE61196FC93EE932FC084E115
:104CF0009EE611969C938E9329C0EDE0FEE61196F8
:104D0000FC93EE9323C083E49CE611969C938E93D0
:104D10001DC0E6E3FCE61196FC93EE9317C089E212
:104D20009CE611969C938E9311C0E9EFFDE61196D7
:104D3000FC93EE930BC087EE9DE611969C938E93A9
:104D400005C0E5EDFDE61196FC93EE932D5F3F4F18
:104D500012962837310509F05DCC109242068091F9
:104D60004606811114C080E090E0FC01E659F14F45
:104D700020813181245631092436310528F00396EB
:104D80008837910591F703C081E080934206109225
:104D9000480680914C06811114C080E090E0FC012F
:104DA000E659F14F20813181285C310924363105E3
:104DB00028F003968837910591F703C081E080932E
:104DC00048068091AE069091AF06DC01ED91FC9112
:104DD000E25BFF4F20913C0F30913D0F40913A0F25
:104DE00050913B0F0190F081E02D61E01995809189
:104DF000AE069091AF06DC01ED91FC91E25BFF4FB6
:104E00002091400F3091410F40913E0F50913F0F44
:104E10000190F081E02D62E019958091AE069091AD
:104E2000AF06DC01ED91FC91E25BFF4F2091440F56
:104E30003091450F4091420F5091430F0190F08106
:104E4000E02D63E019958091AE069091AF06DC01EC
:104E5000ED91FC91E25BFF4F20914F0F3091500F8D
:104E600040914D0F50914E0F0190F081E02D64E084
:104E700019958091AE069091AF06DC01ED91FC9101
:104E8000E25BFF4F2091530F3091540F4091510F2F
:104E90005091520F0190F081E02D65E019958091BD
:104EA000AE069091AF06DC01ED91FC91E25BFF4F05
:104EB0002091570F3091580F4091550F5091560F38
:104EC0000190F081E02D66E019958091AE069091F9
:104ED000AF06DC01ED91FC91E05BFF4F0190F081AA
:104EE000E02D4091460F61E019958091AE069091BA
:104EF000AF06DC01ED91FC91E05BFF4F0190F0818A
:104F0000E02D4091470F62E019958091AE06909197
:104F1000AF06DC01ED91FC91E05BFF4F0190F08169
:104F2000E02D4091480F63E019958091AE06909175
:104F3000AF06DC01ED91FC91E05BFF4F0190F08149
:104F4000E02D4091590F64E019958091AE06909143
:104F5000AF06DC01ED91FC91E05BFF4F0190F08129
:104F6000E02D40915A0F65E019958091AE06909121
:104F7000AF06DC01ED91FC91E05BFF4F0190F08109
:104F8000E02D40915B0F66E019958091AE069091FF
:104F9000AF06DC01ED91FC9100ACF1ADE02D60912C
:104FA0004A0F19958091AE069091AF06DC01ED9104
:104FB000FC9104ACF5ADE02D60915F0F19958091E7
:104FC000AE069091AF06DC01ED91FC9106A4F7A529
:104FD000E02D60914B0F19958091AE069091AF0630
:104FE000DC01ED91FC9104A8F5A9E02D60914C0F36
:104FF00019958091AE069091AF06DC01ED91FC9180
:10500000EA5BFF4F0190F081E02D4091600F60E07E
:1050100019958091AE069091AF06DC01ED91FC915F
:10502000EA5BFF4F0190F081E02D4091610F61E05C
:10503000199580E090E09C012B53324FF901E9551E
:10504000FF4F4081423731F4329720813181232B49
:1050500009F09FC003968837910569F70E94379041
:105060008091AE069091AF06DC01ED91FC91E05A83
:10507000FF4F0190F081E02D40E060915C0F1995A9
:105080008091AE069091AF06DC01ED91FC91E05A63
:10509000FF4F0190F081E02D41E060915E0F199586
:1050A0008091AE069091AF06DC01ED91FC91E05A43
:1050B000FF4F0190F081E02D42E060915D0F199566
:1050C0002091870F30E0AFEFB0E00E94BFBB24E635
:1050D00030E040E050E00E9471BB20936213809169
:1050E000860F81110E9492840E945F5E0E948B4A0B
:1050F0006B017C0110E011110FC08091B50688236F
:1051000059F024E73CE640ED57E060E070E08BE6C4
:105110009BE00E94CD7B11E00E949379882351F09F
:105120000E94AD830E9439430E9439840E942179F4
:105130000E94C9830E94C880029711F00E94154DF9
:105140000E9402910E94C8800297A9F60E948B4A91
:10515000DC01CB018C199D09AE09BF098C3B924043
:10516000A105B10540F218C082E00E94E34481111C
:105170000DC097C882E00E94C744882309F497C8ED
:1051800083E08FA394C8F1E0FFA391C822E02FA38E
:105190008EC80E942B9064CF0E940C5E0E943984BE
:1051A0008091F30A811102C00E94383C0E949D80C8
:1051B00086E30E940F4ABC01990F880B990B611579
:1051C00071058105910511F00E94B3B922E13BE61A
:1051D00048EE53E060E070E08BE69BE0AB960FB6E4
:1051E000F894DEBF0FBECDBFDF91CF911F910F911D
:1051F000FF90EF90DF90CF90BF90AF909F908F90F7
:105200007F906F905F904F903F902F900C94CD7B4C
:105210007F928F929F92AF92BF92CF92DF92EF9246
:10522000FF920F931F93CF93DF9381E080939512AA
:105230008093981280939B1280939E128093AA125F
:105240008093AD129091230F9150953040F0809350
:10525000230F61E070E08EE591E00E94C23A9091E8
:10526000230F2DEF290F8091E20E233008F006C2A4
:105270008A3079F03CF4883009F461C0893009F44F
:10528000B7C1ADC18B3009F4A0C08C3009F4E1C0C6
:10529000A6C184E290E00E9428B7FC018091960F9D
:1052A00028E030E0338322838824839499249A94DD
:1052B00095828482AA24AA94B12CB782A6821186F0
:1052C0001086108E33E8D32ED18E4DE9E42E47E0C0
:1052D000F42EF38EE28E02E614E011830083CBE716
:1052E000DFE0D1A3C0A312A283A3F093A406E093AE
:1052F000A306CF010E94B67184E290E00E9428B715
:10530000FC018091960F29E030E03383228395825F
:105310008482B782A68211861086108ED18EF38E7B
:10532000E28E11830083D1A3C0A312A283A3F093C2
:10533000A206E093A106CF010E94B671FEC280E2F0
:1053400090E00E9428B7FC0188E090E0938382837C
:10535000AA24A394BB24BA94B582A482CC24CA9470
:10536000D12CD782C68211861086108E0AE0F02ECC
:10537000F18E0DE917E0138F028FCAE4D4E0D183D8
:10538000C083F093A406E093A306CF010E941F718F
:1053900080E290E00E9428B7FC0189E090E09383CE
:1053A0008283B582A482D782C68211861086108E2F
:1053B000F18E138F028FD183C083F093A206E09306
:1053C000A106CF010E941F71B8C289E190E00E943E
:1053D00028B7FC0188E090E093838283EE24E39475
:1053E000FF24FA94F582E4820FEF10E0178306831E
:1053F00011861086108ECEE3D4E0D183C083F09363
:10540000A406E093A306CF010E9493771092AA12FC
:105410008091230F843009F090C289E190E00E94CE
:1054200028B7FC0189E090E093838283F582E482CF
:105430001783068311861086108ED183C083F09364
:10544000A206E093A106CF010E9493771092AD12BD
:1054500074C2943009F049C089E190E00E9428B7F5
:10546000EC01FAEEAF2EF5E0BF2EB982A88287E0FC
:1054700090E09B838A83CC24C394DD24DA94DD827C
:10548000CC82EE24EA94F12CFF82EE8219861886F3
:10549000188ECE010E94887E02E314E019830883EF
:1054A000D093A406C093A306CE010E943576109235
:1054B000951289E190E00E9428B7EC01B982A88298
:1054C00086E090E09B838A83DD82CC82FF82EE823D
:1054D00019861886188ECE010E94887E198308834B
:1054E000D093A206C093A1064BC0953009F04EC0E0
:1054F00089E190E00E9428B7EC016AEEA62E65E0F3
:10550000B62EB982A88287E090E09B838A83CC2460
:10551000C394DD24DA94DD82CC82EE24EA94F12C6B
:10552000FF82EE8219861886188ECE010E94887E30
:1055300002E314E019830883D093A206C093A10666
:10554000CE010E9435761092951289E190E00E947A
:1055500028B7EC01B982A88286E090E09B838A8319
:10556000DD82CC82FF82EE8219861886188ECE01EB
:105570000E94887E19830883D093A406C093A30653
:10558000CE010E94357610929812D7C189E190E041
:105590000E9428B7EC018AEE95E09983888387E022
:1055A00090E09B838A8381E09FEF9D838C838FEFC4
:1055B00090E09F838E8319861886188ECE010E94F4
:1055C000887E82E394E099838883D093A406C09375
:1055D000A306CE010E94357610929512AEC189E0E5
:1055E0008093E20E69E070E08DE191E00E94C23AA2
:1055F00080E290E00E9428B7FC0188E090E093836D
:105600008283AA24A394BB24BA94B582A482CC2416
:10561000CA94D12CD782C68211861086108E50E88B
:10562000F52EF18E0DE917E0138F028FC6E5D4E059
:10563000D183C083F093A406E093A306CF010E9418
:10564000617180E290E00E9428B7FC0189E090E05F
:1056500093838283B582A482D782C6821186108604
:10566000108EF18E138F028FD183C083F093A20628
:10567000E093A106CF010E9461715FC18A3009F4F5
:1056800056C03CF4883009F4A0C0893009F400C148
:10569000F6C08B3009F4BAC08C3009F0F0C089E153
:1056A00090E00E9428B7EC017AEEA72E75E0B72EA5
:1056B000B982A88287E090E09B838A83CC24C3943C
:1056C000DD24DA94DD82CC82EE24EA94F12CFF8290
:1056D000EE8219861886188ECE010E94887E02E31B
:1056E00014E019830883D093A606C093A50689E128
:1056F00090E00E9428B7EC01B982A88286E090E091
:105700009B838A83DD82CC82FF82EE821986188693
:10571000188ECE010E94887E19830883D093A80634
:10572000C093A7061092951210929812F0C084E2CE
:1057300090E00E9428B7FC01C091960FD0912F0FE6
:1057400088E090E0938382838824839499249A94B8
:1057500095828482AA24AA94B12CB782A68211864B
:105760001086108E83E8782E718E9DE9C92E97E001
:10577000D92ED38EC28E22E6E22E24E0F22EF182C2
:10578000E0820BE71FE011A300A3D2A3C3A3F09311
:10579000A606E093A50684E290E00E9428B7FC01EB
:1057A00089E090E09383828395828482B782A68287
:1057B00011861086108E718ED38EC28EF182E08299
:1057C00011A300A3D2A3C3A39EC080E290E00E94D5
:1057D00028B7FC0188E090E093838283AA24A394F5
:1057E000BB24BA94B582A482CC24CA94D12CD7828B
:1057F000C68211861086108EDAE0FD2EF18E0DE93C
:1058000017E0138F028FCAE4D4E062C089E190E010
:105810000E9428B7FC0188E090E093838283EE2405
:10582000E394FF24FA94F582E4820FEF10E01783EB
:10583000068311861086108ECEE3D4E0D183C08318
:10584000F093A606E093A50689E190E00E9428B7B0
:10585000FC0189E090E093838283F582E4821783E0
:10586000068311861086108ED183C083F093A8061C
:10587000E093A7061092AA121092AD1248C089E0D8
:105880008093E20E69E070E08DE191E00E94C23AFF
:1058900080E290E00E9428B7FC0188E090E09383CA
:1058A0008283AA24A394BB24BA94B582A482CC2474
:1058B000CA94D12CD782C68211861086108E60E8D9
:1058C000F62EF18E0DE917E0138F028FC6E5D4E0B6
:1058D000D183C083F093A606E093A50680E290E012
:1058E0000E9428B7FC0189E090E093838283B5820F
:1058F000A482D782C68211861086108EF18E138FF5
:10590000028FD183C083F093A806E093A70680910D
:10591000A7069091A806DC01ED91FC910280F3812D
:10592000E02D19958091A5069091A606DC01ED91D8
:10593000FC910280F381E02D19958091230F833033
:1059400039F0823009F06CC08091E20E8C3051F158
:1059500089E190E00E9428B7EC018AEE95E09983F6
:10596000888386E090E09B838A8381E09FEF9D831C
:105970008C838FEF90E09F838E8319861886188E14
:10598000CE010E94887E82E394E099838883D0933D
:105990009F06C0939E06CE010E9435761092981203
:1059A000C6E029C089E190E00E9428B7EC018AEEA8
:1059B00095E09983888384E090E09B838A8381E0EB
:1059C0009FEF9D838C838FEF90E09F838E8319865A
:1059D0001886188ECE010E94887E82E394E0998317
:1059E0008883D0939F06C0939E06CE010E94357691
:1059F00010929E12C4E06091F10E7091F20E8C2F05
:105A00000E94A17D6091F30E7091F40E8C2F0E9484
:105A10009D7D8091F50EE0919E06F0919F06808F0E
:105A2000E091E30E8E2FEE0F990BAA0BBB0BFC013E
:105A30003897E830F10508F0BBC08827E75BFE4FD8
:105A40008F4F0C948BB584E290E00E9428B7FC0144
:105A50008091960F28E030E03383228321E03FEFEE
:105A6000358324832FEF30E0378326831186108619
:105A7000108E94E8918F2DE937E0338F228F22E644
:105A800034E0318320832BE73FE031A320A312A22F
:105A900083A31EC080E290E00E9428B7FC0188E04A
:105AA00090E09383828381E09FEF958384838FEFDF
:105AB00090E09783868311861086108E87E8818F09
:105AC0008DE997E0938F828F86E594E091838083C0
:105AD000F093AD06E093AC0699C080E290E00E949E
:105AE00028B7FC0188E090E09383828381E09FEFF8
:105AF000958384838FEF90E0978386831186108649
:105B0000108E8DE0818F8DE997E0938F828F8AE4EC
:105B100094E0DCCF89E190E00E9428B7FC0188E0A6
:105B200090E09383828381E09FEF958384838FEF5E
:105B300090E09783868311861086108E8EE394E022
:105B400091838083F093AD06E093AC061092AA1285
:105B50005DC08CE190E00E9428B7EC018AEE95E0F0
:105B60009983888385E090E09B838A8381E09FEF1F
:105B70009D838C838FEF90E09F838E831986188698
:105B8000188ECE010E94887E8EED95E037C089E1A7
:105B900090E00E9428B7FC011382128215821482C1
:105BA0001782168211861086108E8EE094E08ECFBA
:105BB0008CE08093E30E6CE070E08EE191E00E9457
:105BC000C23A89E190E00E9428B7EC018AEE95E0A4
:105BD0009983888385E090E09B838A8381E09FEFAF
:105BE0009D838C838FEF90E09F838E831986188628
:105BF000188ECE010E94887E82E394E09983888388
:105C0000D093AD06C093AC0610929B128091AC0667
:105C10009091AD06DC01ED91FC910280F381E02DC5
:105C200019958091EB0E843658F4853608F084E699
:105C300064E6681B8091AC069091AD060E944972A3
:105C40008091E30E8C508230A8F46091EC0E70913C
:105C5000ED0E85E00E94D37C6091EE0E7091EF0E08
:105C600085E00E94B87C8091F00EE091AC06F09146
:105C7000AD06808F2091E40E822F022E000C990B2E
:105C8000AA0BBB0BFC013897E830F10508F089C07E
:105C90008827EF5AFE4F8F4F0C948BB584E290E02B
:105CA0000E9428B7FC018091960F29E030E03383F1
:105CB000228321E03FEF358324832FEF30E03783C9
:105CC000268311861086108E94E8918F2DE937E097
:105CD000338F228F22E634E0318320832BE73FE0AD
:105CE00031A320A312A283A357C080E290E00E94B8
:105CF00028B7FC0189E090E09383828381E09FEFE5
:105D0000958384838FEF90E0978386831186108636
:105D1000108E87E8818F8DE997E0938F828F86E5DB
:105D200094E038C080E290E00E9428B7FC0189E04E
:105D300090E09383828381E09FEF958384838FEF4C
:105D400090E09783868311861086108E8DE0818F78
:105D50008DE997E0938F828F8AE494E01BC0809155
:105D6000230F823009F0BBC18091E20E8C3009F024
:105D7000B6C11FC089E190E00E9428B7FC011382E0
:105D80001282158214821782168211861086108E56
:105D90008EE094E091838083F093B106E093B006A7
:105DA0005EC08091230F823061F58091E20E8C30CD
:105DB00041F58BE08093E40E6BE070E08FE191E0C1
:105DC0000E94C23A89E190E00E9428B7FC0189E074
:105DD00090E09383828381E09FEF958384838FEFAC
:105DE00090E09783868311861086108E8EE394E070
:105DF00091838083F093B106E093B0061092AD12C8
:105E00002EC08CE08093E40E6CE070E08FE191E0B6
:105E10000E94C23A89E190E00E9428B7EC018AEE24
:105E200095E09983888384E090E09B838A8381E076
:105E30009FEF9D838C838FEF90E09F838E831986E5
:105E40001886188ECE010E94887E82E394E09983A2
:105E50008883D093B106C093B00610929E128091B1
:105E6000B0069091B106DC01ED91FC910280F381C6
:105E7000E02D19958091EA0E843658F4853608F0A5
:105E800084E664E6681B8091B0069091B1060E949A
:105E900049728091E40E8C50823000F56091E50EDD
:105EA0007091E60E84E00E94D37C6091E70E7091C1
:105EB000E80E84E00E94B87C8091E90EE091B00683
:105EC000F091B106808F8091E40E8D3039F480918D
:105ED000E90EE0912812F0912912808F8EE190E076
:105EE0000E9428B7EC01F090FA0EC090FE0ED09000
:105EF000FF0EA090FC0EB090FD0E8AEE95E0998307
:105F0000888383E090E09B838A8381E09FEF9D8379
:105F10008C830FEF10E01F830E8319861886188E6E
:105F2000CE010E94887E86E294E099838883BA8EAF
:105F3000A98EDC8ECB8EFD8ED0931C12C0931B12CB
:105F40006091000F7091010F83E00E94D37C6091FB
:105F5000020F7091030F83E00E94B87C8091FA0ECB
:105F6000E0911B12F0911C12808F8091FA0E0E941A
:105F70008D3A80911B1290911C12DC01ED91FC91E5
:105F80000280F381E02D19958091040F882339F167
:105F900085E290E00E9428B7FC018091090F909162
:105FA0000A0F2091070F3091080F4091050F509173
:105FB000060F68E070E07383628315821482178392
:105FC000068311861086108E6AE174E07183608307
:105FD000528F418F348F238F968F858F22C085E219
:105FE00090E00E9428B7FC018091070F9091080F64
:105FF0002091050F3091060F48E050E05383428313
:10600000158214821783068311861086108E4AE14A
:1060100054E051834083328F218F948F838F168F6A
:10602000058FF0932A06E093290680912906909126
:106030002A060E9471778091AA128823F9F089E1DB
:1060400090E00E9428B7FC0188E090E0938382836F
:10605000158214828FEF93E0978386838FEF91E010
:1060600091878087108E8EE394E091838083F093F4
:10607000A912E093A812CF010E9493778091AD12EC
:10608000882309F474C089E190E00E9428B7FC01DC
:1060900089E090E093838283158214828FEF93E0EE
:1060A000978386838FEF91E091878087108E8EE3B0
:1060B00094E091838083F093AC12E093AB12CF0114
:1060C000DF91CF911F910F91FF90EF90DF90CF90D4
:1060D000BF90AF909F908F907F900C9493772C30CF
:1060E00009F498CE8CE190E00E9428B7EC018AEE8A
:1060F000882E85E0982E9982888294E0A92EB12C72
:10610000BB82AA82CC24C394DD24DA94DD82CC82C3
:10611000EE24EA94F12CFF82EE8219861886188EFE
:10612000CE010E94887E0EED15E019830883D0937E
:10613000B106C093B0068CE190E00E9428B7EC0154
:1061400099828882BB82AA82DD82CC82FF82EE8223
:1061500019861886188E0E94887E19830883D0932A
:106160002912C0932812CE010E94F17676CEDF91DB
:10617000CF911F910F91FF90EF90DF90CF90BF9044
:10618000AF909F908F907F9008952F923F924F9263
:106190005F926F927F928F929F92AF92BF92CF92B7
:1061A000DF92EF92FF920F931F93CF93DF93CDB7C0
:1061B000DEB7C65AD1090FB6F894DEBF0FBECDBF09
:1061C000CDB6DEB6CC55DF4F1882C45AD040CD557F
:1061D000DF4F1882C35AD0408091AF0D8A3709F43F
:1061E00047C0C0F4873709F4D9C238F48F3109F4B5
:1061F0002CC5863709F4E2C1EBC5883709F4DDC246
:10620000893709F0E5C50E9486800E948B4A2B01E0
:106210003C0129C08E3709F42DC338F48B3709F4BB
:10622000CAC18C3709F4D8C2D3C5813809F4FEC479
:10623000823809F4E9C4803809F0CAC563C40E94F1
:106240008B4ADC01CB0184199509A609B709803274
:106250009340A105B10508F003C50E94154D0E94A9
:1062600086800E94A9530E94C880029741F7F8C413
:106270000E94C880029729F060E084E80E94359768
:106280008BC18091F40A823031F0833039F482E09E
:106290008093CC1103C081E080933F1381E0809311
:1062A000B90D8E010C551F4F2BE0AE0144575F4FC7
:1062B00068E871E90E94AF960E949D80893058F08D
:1062C000015011092BE0AE014F575F4F68E872E9AA
:1062D00081E00E94AF961092B80D772473940E94CB
:1062E000B380882309F43DC1198222961FAE2297FC
:1062F0008091B80D81110EC0BE0164577F4FCE0151
:106300008F5B9F4F0E9446B9CC55DF4F0881C45A1E
:10631000D0400FC07092B80DBE016F577F4FCE01B5
:106320008F5B9F4F0E9446B9CD55DF4F0881C35AFE
:10633000D0401091B80DADB6BEB68091F00AEDB761
:10634000FEB722E0829FE019F10911240FB6F894FC
:10635000FEBF0FBEEDBF8DB79EB701967C016EE00C
:1063600076E0CE0183569F4F0E94008B8091F40A05
:10637000823089F0833061F1813009F0A1C0409111
:10638000F00A50E0B70180911813909119130E9400
:10639000DF4F10E039C02091F00A30E05FB7F89489
:1063A00040E0842F90E08217930774F4880F991FC0
:1063B000F701E80FF91FDC01A25EBC4E8D919C91A4
:1063C000918380834F5FEDCF5FBF10923E131CC05F
:1063D0002091F00A30E05FB7F89440E0842F90E01D
:1063E0008217930774F4880F991FF701E80FF91FBC
:1063F000DC01AE52BE4E8D919C91918380834F5FA4
:10640000EDCF5FBF109215136DE270E0CE018356A1
:106410009F4F0E942F8A2091F00A293048F01123C3
:1064200021F0113021F418E004C028E001C020E080
:1064300010E0121758F5F701E10FF11DE10FF11D02
:10644000608171814AE0CE0189569F4FCB55DF4F65
:106450002883C55AD0400E94D58ABE0169567F4F15
:10646000CE0183569F4F0E94568ACE0189569F4F78
:106470000E94D08ACE0183569F4F0E94E73D1F5F46
:10648000CB55DF4F2881C55AD040D3CF40E450E0F0
:10649000BE016F5F7F4FCE0183569F4F0E94DF3D4D
:1064A000CF55DF4F1881C15AD040CE0183569F4F40
:1064B0000E94D08A0FB6F894BEBE0FBEADBE0BC010
:1064C000CE0183569F4F0E94D08A0FB6F894BEBE6D
:1064D0000FBEADBE10E0BE016F5F7F4FCE018F5B80
:1064E0009F4F0E9446B9010F10E0E1E4F0E0EC0F8D
:1064F000FD1FE00FF11F1082BE016F5B7F4F809187
:106500009A1390919B130E94638BB801CE018F5B0D
:106510009F4F0E94C653BC0180919A1390919B1388
:106520000E94B33B6AE080919A1390919B130E9462
:10653000388B80919A1390919B13DC01ED91FC9123
:106540000284F385E02D19950E949D80893048F0E2
:106550008091B80D811103C07092B80D02C01092E5
:10656000B80D0E9486800E94A9530E941E78811156
:106570000CDE8091AE0D81110FC08091B90D882382
:1065800059F08091C711811107C08091AC0D909195
:10659000AD0D0A970CF4A3CE8091F40A823039F045
:1065A000833009F015C481E08093CC1111C481E0DF
:1065B00080933F130DC41092B90D44C31091B20DD6
:1065C0008FEF810F853028F060E089E80E943597D1
:1065D000FFC3133079F018F41230F9F004C014300E
:1065E00079F0153099F040E6442E49E0542E612CA4
:1065F000712C19C0412C3BE4532E612C712C13C01B
:10660000412C26E9522E612C712C0DC0412C92ECAC
:10661000592E66246394712C06C080E8482E85E2CA
:10662000582E612C712C00E0E12EF12C5701BFE8AF
:10663000AB0EB11C1501E89427F83324E6E9EE0E01
:10664000F11CE894E7F8FF24023091F018F40130CF
:1066500051F004C0033089F00430A1F040E659E065
:1066600060E070E013C040E855E260E070E00EC00A
:1066700040E05BE460E070E009C040E056E960E0C3
:1066800070E004C040E052EC61E070E08DE997E01A
:106690000E9418718DE997E00E94AA890E948B4A96
:1066A0004B015C01F2E38F0E911CA11CB11C0E94F6
:1066B00069530E948B4A681579058A059B05B8F3D2
:1066C00060E870E08DE997E00E94127A6FE070E078
:1066D0008DE997E00E94127A612F8DE997E00E9480
:1066E0006489B1018DE997E00E94127A0E948B4A79
:1066F0004B015C012AE0820E911CA11CB11C0E947E
:1067000069530E948B4A681579058A059B05B8F381
:1067100067E870E08DE997E00E94127A6FE070E020
:106720008DE997E00E94127A612F8DE997E00E942F
:106730006489B7018DE997E00E94127A8DE997E0AC
:106740000E94AA890E948B4A4B015C013EE5830EA0
:1067500031E0931EA11CB11C0E9469530E948B4A18
:10676000681579058A059B05B8F30F5F053009F0B8
:106770006BCFB301A2018DE997E00E94187140929E
:106780007B0F50927C0F60927D0F70927E0FB30151
:10679000A20186EB91E00E941A3E54C283E090E091
:1067A0000E9428B72AE0DC012C932DE937E01296ED
:1067B0003C932E9311976AE00CC083E090E00E9416
:1067C00028B72DE0FC0120832DE937E032832183B7
:1067D0006DE00E943D4F36C24091B20D5091B30D15
:1067E0000091B40D1091B50D6091B00D7091B10D87
:1067F000CE010196CB55DF4F4883C55AD040CA55CC
:10680000DF4F5883C65AD0400E94E766CB55DF4F12
:106810004881C55AD040CA55DF4F5881C65AD0402A
:10682000892BE1F08D81873050F4853080F4813000
:10683000A8F0642F8B819C810E941E3C0CC0893083
:1068400068F4B8018B819C810E941A3E04C0BA0191
:106850008B819C8197D60E94B19704C061E085E846
:106860000E9435978091AB0D8111B2C281E0809377
:10687000AB0DAEC2B090B00DE090B10DC956DF4F78
:106880001882C759D0406EE076E0CE018F579F4FF7
:106890000E94008B6B2D7E2DCE0184579F4F0E944E
:1068A000E766892B09F4C9C0C057DF4FE881C0599A
:1068B000D0404E2F50E0FA013197E830F10508F052
:1068C000BCC08827E75AFE4F8F4F0C948BB5C25738
:1068D000DF4F88819981CE58D0400E9451BB2396CA
:1068E0001FAE1EAE239725961FAE1EAE2597279688
:1068F0001FAE1EAE27974AE0BE016F5F7F4F90E04C
:106900003EC0C257DF4F88819981CE58D0400E9447
:1069100051BB682F880F770B4AE00AC0C257DF4F80
:1069200088819981CE58D0400E945EBB4AE0BC016C
:10693000CE0101960E94D58ABE016F5F7F4FCE01C6
:106940008F579F4F0E94F689CE01019663C0C257B0
:10695000DF4F88819981CE58D0400E945EBB23963C
:106960001FAE1EAE239725961FAE1EAE2597279607
:106970001FAE1EAE27974AE0BE016F5F7F4F0E9499
:10698000FFB935C0C257DF4F88819981CE58D040BA
:106990000E9459BB23961FAE1EAE239725961FAEAD
:1069A0001EAE259727961FAE1EAE27972AE0AE0192
:1069B0004F5F5F4F0E94D0B91AC0C257DF4F888126
:1069C0009981CE58D0400E9459BB23961FAE1EAE6F
:1069D000239725961FAE1EAE259727961FAE1EAE97
:1069E00027972AE0AE014F5F5F4F0E94DEB9BE01DC
:1069F0006F5F7F4FCE018F5B9F4F0E94B08ABE01B9
:106A00006F5B7F4FCE018F579F4F0E94F689CE015B
:106A10008F5B9F4F0E94D08A4BE050E0BE016F5BBE
:106A20007F4FCE018F579F4F0E94DF3DCB57DF4FE7
:106A3000F880C558D04011E002C0F12C10E0CE0122
:106A40008F579F4F0E94D08A112309F4BDCD8E012C
:106A500009561F4F20E4AE014F5F5F4F68E87B2D62
:106A60008E2D0E94AF96BE016F5B7F4FCE010196C7
:106A70000E9446B9C956DF4F8881C759D040F80EE9
:106A800081E08F0DC956DF4F8883C759D040E1E0C0
:106A9000F0E0EC0FFD1FEF0DF11D9CE79083E1E0AE
:106AA000F0E0EC0FFD1FE80FF11D1082BE016F5FDB
:106AB0007F4F80919A1390919B130E94638BC956CC
:106AC000DF4F6881C759D04070E0CE0101960E9427
:106AD000C653BC0180919A1390919B1344D66AE0EF
:106AE00080919A1390919B130E94388B80919A13F6
:106AF00090919B13DC01ED91FC910284F385E02DD4
:106B0000199566C18091B00D9091B10D80389105B5
:106B100009F05EC18E0104571F4F20E4AE014F5FA4
:106B20005F4F68E870E880E00E94AF9662EF75E022
:106B3000CE018F579F4F0E94008BCE018F579F4FE2
:106B40000E94E73DC457DF4F2881CC58D040CB5737
:106B5000DF4F88819981C558D040820F911DC4575D
:106B6000DF4F8883CC58D04022961FAE22974BE04F
:106B700050E0BE016F5B7F4FCE018F579F4FFCD718
:106B8000BE016F5B7F4FCE0101960E9446B9C4578C
:106B9000DF4F8881CC58D040E1E0F0E0EC0FFD1FE2
:106BA000E80FF11D1082BE016F5F7F4F80919A1335
:106BB00090919B130E94638BC457DF4F6881CC5820
:106BC000D04070E0CE0101960E94C653BC01809176
:106BD0009A1390919B13C7D56AE080919A13909174
:106BE0009B130E94388B80919A1390919B13DC0128
:106BF000ED91FC910284F385E02D1995CE018F571C
:106C00009F4F0E94D08AE4C08091B00D9091B10D49
:106C10008238910509F0DCC08E0104571F4F20E433
:106C2000AE014F5F5F4F68E872E87DCF8091B00D95
:106C30009091B10D8138910509F0CAC08091B90DCC
:106C40008111C6C00E94B197C3C08091B00D9091D0
:106C5000B10D4F9709F0BCC081E08093AE0DB8C074
:106C60000E94C880029719F060E084E8AFCC809160
:106C7000F30A811101C0FCD50E949D80F82E6EE0C0
:106C800076E0CE0184579F4F0E94008BC956DF4F9C
:106C90001882C759D0408E0109561F4F20E4AE011B
:106CA0004F5F5F4F68E879E780E00E94AF96CF576B
:106CB000DF4F19821882C158D040CD57DF4F19825B
:106CC0001882C358D040CB57DF4F19821882C5585D
:106CD000D0406F2D70E080E090E02AE0AE014F5B85
:106CE0005F4F0E94D0B9BE016F5B7F4FCE018F57BF
:106CF0009F4F0E94B08ABE016F577F4FCE018457CD
:106D00009F4F0E94F689CE018F579F4F0E94D08AD5
:106D10004BE050E0BE016F5B7F4FCE0184579F4F29
:106D20002BD7C057DF4F1881C059D040BE016F5BD1
:106D30007F4FCE0101960E9446B9C956DF4F888128
:106D4000C759D040810F91E0980FC956DF4F988303
:106D5000C759D040E1E0F0E0EC0FFD1FE80FF11D56
:106D60008CE78083E1E0F0E0EC0FFD1FE90FF11DFF
:106D70001082BE016F5F7F4F80919A1390919B1399
:106D80000E94638BC956DF4F6881C759D04070E0BD
:106D9000CE0101960E94C653BC0180919A13909136
:106DA0009B13E1D46AE080919A1390919B130E9407
:106DB000388B80919A1390919B13DC01ED91FC919B
:106DC0000284F385E02D1995CE0184579F4F19CF8A
:106DD0000FB6F894DEBE0FBECDBECA55DF4F0FB65C
:106DE000F894DEBF0FBECDBFDF91CF911F910F9101
:106DF000FF90EF90DF90CF90BF90AF909F908F90DB
:106E00007F906F905F904F903F902F900895CF9319
:106E1000DF93EC010E948B4A688379838A839B838A
:106E2000CE01DF91CF910895EF92FF921F93CF9300
:106E3000DF93CDB7DEB765970FB6F894DEBF0FBE10
:106E4000CDBF182F7B018EEE99E00E94229281E047
:106E500080931C0A84E690E09093FF098093FE09DA
:106E600084E6E816F10418F484E6E82EF12CC70154
:106E700064E670E00E9464B570931E0A60931D0A78
:106E80007093010A6093000A1093FB098FEF810F42
:106E9000823010F41230D1F08EEE99E00E943492DC
:106EA0008091F909882329F083EC95EFA8ECBFE3E2
:106EB00004C084EB98ECA6E9B0E48093180A9093A0
:106EC000190AA0931A0AB0931B0A55C08091F909B8
:106ED000882329F084EB98ECA6E9B0E404C083ECA5
:106EE00095EFA8ECBFE38093180A9093190AA0933A
:106EF0001A0AB0931B0A8EEE99E00E943E9280918E
:106F00001C0A8823C1F11092FB098EE690E09A8357
:106F1000898388E290E09C838B838CE390E09E835E
:106F20008D831D8A83E08F938DB79EB745970FB6EB
:106F3000F8949EBF0FBE8DBFADB7BEB7119685E169
:106F4000FE01319601900D928A95E1F78EEE99E05F
:106F50000E9448920FB6F894DEBF0FBECDBF659673
:106F60000FB6F894DEBF0FBECDBFDF91CF911F915A
:106F7000FF90EF9008958EEE99E065960FB6F89425
:106F8000DEBF0FBECDBFDF91CF911F91FF90EF907D
:106F90003ECF0F931F93CF93DF93EC01AB0160E0E3
:106FA00070E02AE00E94788B8C01CE010E949D8CBB
:106FB000800F911FDF91CF911F910F9108958F92B4
:106FC0009F92AF92BF92CF92DF92EF92FF920F9378
:106FD0001F93CF93DF931F921F92CDB7DEB7082E7A
:106FE000000C990BAA0BBB0BFC013197EF30F1059C
:106FF00008F066C28827EF59FE4F8F4F0C948BB56F
:1070000084E08093DD098AE08093DE0986E2809344
:10701000E00981E08093E3098093E4098093E20929
:1070200042E050E120E030E08091DD0990E0281757
:1070300039070CF08CC1FA0185919491A0E0B0E081
:10704000880F991FAA1FBB1FF901EE0FFF1FEE0F3C
:10705000FF1FEC58F64F80839183A283B3832F5F89
:107060003F4F4E5F5F4FE0CF84E08093DD098AE0C1
:107070008093DE0986E28093E00981E08093E30952
:107080008093E40982E08093E2094AEF5FE020E028
:1070900030E08091DD0990E0281739070CF057C1E6
:1070A000FA0185919491A0E0B0E0880F991FAA1F82
:1070B000BB1FF901EE0FFF1FEE0FFF1FEC58F64F3D
:1070C00080839183A283B3832F5F3F4F4E5F5F4FD7
:1070D000E0CF84E08093DE0985E28093E00981E0DF
:1070E0008093E30988E08093E40983E08093E209D8
:1070F00080E090E0FC01EE50F04FE491DC01AB51F8
:10710000B64FEC93019688309105A1F70E94318625
:107110001EC188E08093DD0986E08093DE0986E267
:107120008093E00981E08093E3098093E40984E09F
:107130008093E20942EE5FE020E030E08091DD09DB
:1071400090E0281739070CF002C1FA01859194915B
:10715000A0E0B0E0880F991FAA1FBB1FF901EE0F36
:10716000FF1FEE0FFF1FEC58F64F80839183A28321
:10717000B3832F5F3F4F4E5F5F4FE0CF88E0809338
:10718000DD0981E08093DE0997E29093E009809326
:10719000E3098093E40985E08093E20942ED5FE032
:1071A00020E030E08091DD0990E0281739070CF0ED
:1071B000CEC0FA0185919491A0E0B0E0880F991FAC
:1071C000AA1FBB1FF901EE0FFF1FEE0FFF1FEC58A8
:1071D000F64F80839183A283B3832F5F3F4F4E5F2F
:1071E0005F4FE0CF82E18093DD0981E08093DE098B
:1071F00097E29093E0098093E3098093E4098FE09C
:107200008093E2094EEA5FE020E030E08091DD0902
:1072100090E0281739070CF09AC0FA0185919491F3
:10722000A0E0B0E0880F991FAA1FBB1FF901EE0F65
:10723000FF1FEE0FFF1FEC58F64F80839183A28350
:10724000B3832F5F3F4F4E5F5F4FE0CFE091480A1F
:10725000F091490A74978081918140E550E060E0A7
:1072600070E0885B954F0E94FC862AC182E1809382
:10727000DD0985E08093DE0982E28093E00981E008
:107280008093E3098093E40987E08093E20980E931
:1072900093E3A0E0B0E08093740990937509A09304
:1072A0007609B0937709F2E08F2E912C01E010E07F
:1072B00080E090E0A0E0BBE54CE454E060E070E0EA
:1072C00024EEC22E2CE0D22EE12CF12C9801220FBC
:1072D000331F220F331F5401AA0CBB1CAA0CBB1C6A
:1072E0002C58364FF901B7FF0DC0C082D182E2821F
:1072F000F38295012C58364FF90140835183628304
:1073000073830CC0408351836283738395012C582F
:10731000364FF901C082D182E282F382880F991F31
:10732000AA1FBB1F0E5F1F4FF2E08F0E911C22E1C0
:107330008216910459F688E79FEFA0E0B0E08093B1
:10734000B8099093B909A093BA09B093BB090E94F8
:10735000A086B6C0CE0101960E942A7523E040E1C6
:1073600050E060E070E072C084E08093DD0982E369
:107370008093DE0986E28093E00981E08093E3094F
:107380008093E4098AE08093E20946EA5FE020E026
:1073900030E08091DD0990E028173907C4F6FA0142
:1073A00085919491A0E0B0E0880F991FAA1FBB1FA0
:1073B000F901EE0FFF1FEE0FFF1FEC58F64F808311
:1073C0009183A283B3832F5F3F4F4E5F5F4FE1CF27
:1073D00084E08093DD0980E28093DE0986E2809379
:1073E000E00981E08093E3098093E4098BE08093D6
:1073F000E2094EE95FE020E030E08091DD0990E0B5
:10740000281739070CF0A3CFFA0185919491A0E0D9
:10741000B0E0880F991FAA1FBB1FF901EE0FFF1FD5
:10742000EE0FFF1FEC58F64F80839183A283B38346
:107430002F5F3F4F4E5F5F4FE0CFCE0101960E941E
:107440002A7521E040E154E060E070E0CE01019651
:107450000E949D7435C084E08093DD0983E08093B1
:10746000DE0986E28093E00981E08093E30980935E
:10747000E4098DE08093E20946E95FE020E030E036
:107480008091DD0990E0281739070CF060CFFA01F0
:1074900085919491A0E0B0E0880F991FAA1FBB1FAF
:1074A000F901EE0FFF1FEE0FFF1FEC58F64F808320
:1074B0009183A283B3832F5F3F4F4E5F5F4FE0CF37
:1074C0000F900F90DF91CF911F910F91FF90EF9050
:1074D000DF90CF90BF90AF909F908F9008950F93C3
:1074E0001F93CF93DF93EC01462F50E060E070E0F4
:1074F0002AE00E94788B8C01CE010E949D8C800F27
:10750000911FDF91CF911F910F910895462F50E069
:1075100060E070E02AE00C94788B2FB7F894882311
:1075200081F08091FF109091001190930E11809343
:107530000D1180910F119091101118161906ACF0D1
:107540000FC0809101119091021190930E118093C0
:107550000D1180910F1190911011181619062CF42D
:1075600080910F119091101107C080910F1190918F
:1075700010119195819591099093101180930F119D
:107580002FBF0895AF92BF92CF92DF92EF92FF92FA
:107590000F931F93CF93DF931F921F92CDB7DEB748
:1075A0008C017A836983CE0101966C01580192E0C7
:1075B000A90EB11CE12CF12CC8010E9451BBF601AF
:1075C00061916F01861731F0C8010E9463BBFFEF24
:1075D000EF1AFF0A0F5F1F4F0A151B0569F781E0BD
:1075E000EF2809F480E00F900F90DF91CF911F9169
:1075F0000F91FF90EF90DF90CF90BF90AF900895E4
:10760000EF92FF920F931F93CF93DF931F921F92DE
:10761000CDB7DEB78C017B018AEA8A8341E050E076
:10762000BE016E5F7F4FC8010E94D14ED701ED9120
:10763000FC910284F385E02DC701199582E88983C6
:1076400041E050E0BE016F5F7F4FC8010E94D14E04
:107650000F900F90DF91CF911F910F91FF90EF90BE
:107660000895CF92DF92EF92FF920F931F930E94A3
:107670008B4A6B017C0160937B1170937C1180932A
:107680007D1190937E118091F50A0E948F8E8093D8
:107690007A119091F70A992329F091E0811190E0F5
:1076A00090937A118091FF0A9091000BA091010BA9
:1076B000B091020B97018601081B190B2A0B3B0B9B
:1076C0004091030B5091040B6091050B7091060BD8
:1076D0009091F80A041715072607370760F4C0923F
:1076E000FB0AD092FC0AE092FD0AF092FE0A109288
:1076F000FA0A892F1EC09093F90A80917A1180931B
:10770000F80AC092FB0AD092FC0AE092FD0AF092BD
:10771000FE0A891761F0C092FF0AD092000BE09236
:10772000010BF092020B91E09093FA0A02C01092C2
:10773000FA0A1F910F91FF90EF90DF90CF9008957C
:107740000F931F93CF93DF93EC012AE00E94788B75
:107750008C01CE010E949D8C800F911FDF91CF91F3
:107760001F910F910895CF92DF92EF92FF920F93A6
:107770001F93CF93DF936B01770FEE08FF08F7FE9F
:107780001BC0EC016DE20E94388B8C014427552709
:10779000BA014C195D096E097F092AE0CE010E94E9
:1077A000788B800F911FDF91CF911F910F91FF90E8
:1077B000EF90DF90CF9008952AE0B701A601DF9106
:1077C000CF911F910F91FF90EF90DF90CF900C948D
:1077D000788BCF92DF92EF92FF920F931F93CF930C
:1077E000DF938C016B01770FEE08FF08F7FE12C0E4
:1077F0006DE20E94388BEC0144275527BA014C19E1
:107800005D096E097F092AE0C8010E94788BC80FC4
:10781000D91F06C02AE0B701A6010E94788BEC01AF
:10782000C8010E949D8C8C0F9D1FDF91CF911F91ED
:107830000F91FF90EF90DF90CF9008950F931F93DB
:10784000CF93DF931F92CDB7DEB78C0169830E947F
:1078500051BB6981861729F0C8010E9463BB81E092
:1078600001C080E00F90DF91CF911F910F9108959B
:10787000CF930E949D8084E090E09093F20A8093E1
:10788000F10A86EC9DE090939E1080939D101092DB
:1078900098108091F00A9091C60D891718F091E028
:1078A000909395102FEC3DE03093A8102093A710F3
:1078B0001092A2109091CF0D891718F091E090933B
:1078C0009F1028ED3DE03093B2102093B11010923C
:1078D000AC109091D80D891718F091E09093A910F1
:1078E00021EE3DE03093BC102093BB101092B610F7
:1078F0009091E10D891718F091E09093B3101092D8
:10790000EF0A20E030E0F901E659F14F4081518162
:10791000415051094432510520F491E09093EF0A0F
:1079200005C02D5F3F4F2837310569F79091EF0A69
:10793000992341F12091D90D3091DA0D2D5D3F4F02
:107940003093DA0D2093D90D2091DB0D3091DC0DB1
:10795000235231093093DC0D2093DB0D2091E20D91
:107960003091E30D2D5D3F4F3093E30D2093E20DF9
:107970002091E40D3091E50D235231093093E50D4E
:107980002093E40D9091E30E9F3049F49091E40E22
:107990009F3029F4109294101092931008C02091F7
:1079A000370F3091380F309394102093931022E1C9
:1079B00030E030939110209390102091F10A309193
:1079C000F20AAAEEBDE0ECE3F0E141E0B683A58364
:1079D0009C91992329F0891718F040832F5F3F4F1E
:1079E0001A96379690E1E039F90781F73093F20A59
:1079F0002093F10A2131310534F080E190E0909339
:107A0000F20A8093F10A0E94888089E990E19093BC
:107A10009F0F80939E0F80919D1090919E10909348
:107A20009D0F80939C0F86E990E19093A10F809326
:107A3000A00F87E990E19093A30F8093A20F85E9AF
:107A400090E19093A50F8093A40F83EA90E1909327
:107A5000A90F8093A80F8091A7109091A8109093E0
:107A6000A70F8093A60F80EA90E19093AB0F8093CD
:107A7000AA0F81EA90E19093AD0F8093AC0F8FE94C
:107A800090E19093AF0F8093AE0F8DEA90E19093C9
:107A9000B30F8093B20F8091B1109091B210909378
:107AA000B10F8093B00F8AEA90E19093B50F809365
:107AB000B40F8BEA90E19093B70F8093B60F89EAE9
:107AC00090E19093B90F8093B80F87EB90E190937A
:107AD000BD0F8093BC0F8091BB109091BC10909310
:107AE000BB0F8093BA0F84EB90E19093BF0F80930C
:107AF000BE0F85EB90E19093C10F8093C00F83EB95
:107B000090E19093C30F8093C20F2091F10A3091BE
:107B1000F20A2450310960E07AE0C7E0462F50E0D5
:107B20004217530724F5CA010496789FF001799F04
:107B3000F00D1124E456F04FC49FC001C59F900D75
:107B40001124AC01425C5F4E53834283DC01A45C90
:107B5000BF4E15964D915C91169751834083835C7F
:107B60009F4E95838483B187A0876F5FD7CF81E0D5
:107B70008093F30ACF9108950F931F93CF93DF93D0
:107B8000FC01248135812115310519F4FB01108296
:107B900011C0EA0121972C173D0708F4E9018B0178
:107BA000FC0160817181AE01C8010E9458B9C00F0B
:107BB000D11F1882DF91CF911F910F910895411528
:107BC000510521F06115710509F0D6CF0895EF92A6
:107BD000FF920F931F93CF93DF931F921F92CDB706
:107BE000DEB78C018CE789831A82F801E480F58086
:107BF000FFEFEF1AFF0AB701C8010E942F8A8823FE
:107C000081F0F8012081318184819581BE016F5F0F
:107C10007F4F820F931F0E9451B9F801F582E482D1
:107C200081E00F900F90DF91CF911F910F91FF9006
:107C3000EF900895AF92BF92CF92DF92EF92FF92B2
:107C40000F931F93CF93DF9300D01F92CDB7DEB772
:107C50008C0149835A836B837C83CE0101966C012E
:107C6000580194E0A90EB11CE12CF12CC8010E942E
:107C700051BBF60161916F01861731F0C8010E9476
:107C800063BBFFEFEF1AFF0A0F5F1F4F0A151B05BB
:107C900069F781E0EF2809F480E00F900F900F90D2
:107CA0000F90DF91CF911F910F91FF90EF90DF9098
:107CB000CF90BF90AF900895CF92DF92EF92FF9256
:107CC0000F931F93CF93DF93EC010091BA0DE0E087
:107CD000F0E020E030E0A90110E0CE17DF071CF152
:107CE000309711F40D32E1F0DF01A654B24FFC9051
:107CF00080ED8F0D8A30A8F4AAE0B0E00E948DBB21
:107D00002F2DFF0C330B205331096901330FEE087F
:107D1000FF089B01AC012C0D3D1D4E1D5F1D01C0D8
:107D200011E03196DACFCA01B901112339F09095EB
:107D30008095709561957F4F8F4F9F4FDF91CF91C9
:107D40001F910F91FF90EF90DF90CF900895809159
:107D5000F80A811105C081E09091FA0A911101C0E1
:107D600080E00895CF93DF9320911F0A3091200A7D
:107D7000E9012697A881B981A15EB54F12961C92A0
:107D8000082E000C990BAA0BBB0BFC013197EF30AE
:107D9000F10508F06EC18827E059FE4F8F4F0C9413
:107DA0008BB5F9013A9780819181815E954F0E9450
:107DB000EDAE882309F462C1E0911F0AF091200A18
:107DC00036970190F081E02DE15EF54F81E0EDC046
:107DD000F9013C9780819181815E954F0E9421AE8F
:107DE000882309F44BC1E0911F0AF091200A3697CD
:107DF0000190F081E02DE15EF54F82E0D6C0F901FF
:107E00003E9780819181815E954F0E9464AD882369
:107E100009F434C1E0911F0AF091200A36970190CD
:107E2000F081E02DE15EF54F83E0BFC0F90170976E
:107E300080819181815E954F0E94E3AC882309F493
:107E40001DC1E0911F0AF091200A36970190F08140
:107E5000E02DE15EF54F84E0A8C0F90172978081C2
:107E60009181815E954F0E9410B5882309F406C167
:107E7000E0911F0AF091200A36970190F081E02DE1
:107E8000E15EF54F85E091C0F901749780819181A1
:107E9000815E954F0E94CBB4882309F4EFC0E09136
:107EA0001F0AF091200A36970190F081E02DE15EE3
:107EB000F54F8FE07AC0F901769780819181815EDC
:107EC000954F0E9452B4882309F4D8C0E0911F0A4C
:107ED000F091200A36970190F081E02DE15EF54F98
:107EE00086E063C0F901789780819181815E954F2A
:107EF0000E94CCB3882309F4C1C0E0911F0AF0911D
:107F0000200A36970190F081E02DE15EF54F87E081
:107F10004CC0F9017A9780819181815E954F0E94D2
:107F2000BEB3882309F4AAC0E0911F0AF091200A89
:107F300036970190F081E02DE15EF54F88E035C085
:107F4000F901B29780819181815E954F0E94F2B0D4
:107F5000882309F493C0E0911F0AF091200A369714
:107F60000190F081E02DE15EF54F83819481A58140
:107F7000B6814097A105B10509F080C08FC0F90115
:107F80007C9780819181815E954F0E94FBB288230E
:107F900009F474C0E0911F0AF091200A369701900D
:107FA000F081E02DE15EF54F8AE0828367C0F90140
:107FB0007E9780819181815E954F0E9436B28823A1
:107FC00009F45CC0E0911F0AF091200A36970190F5
:107FD000F081E02DE15EF54F8BE0E7CFF901B2973C
:107FE00080819181815E954F0E94F2B0882309F4CF
:107FF00045C0E0911F0AF091200A36970190F08168
:10800000E02DE15EF54F83819481A581B6818031B9
:108010009440A105B10591F543C0F901B097808165
:108020009181815E954F0E946BB1882339F1E09177
:108030001F0AF091200A36970190F081E02DE15E51
:10804000F54F8DE0B2CFF901B29780819181815EC9
:10805000954F0E94F2B0882389F0E0911F0AF091B9
:10806000200A36970190F081E02DE15EF54F8EE019
:108070009CCFE881F981E15EF54F1282E0911F0A01
:10808000F091200A36970190F081E02DE15EF54FE6
:1080900081E09281911106C080E004C089E085CF23
:1080A0008CE083CFDF91CF9108958091AE069091BF
:1080B000AF06DC01ED91FC910084F185E02D19956E
:1080C0008091AE069091AF06DC01ED91FC910480A9
:1080D000F581E02D199480910702813019F485E033
:1080E0008093070208951092A906089580911106C1
:1080F000882371F0109211068091B406882341F014
:108100006CEB71E18091B2069091B3060C94B08C47
:1081100008958091230F833099F080911106811189
:108120000FC081E0809311068091B406882341F04E
:1081300067EA71E18091B2069091B3060C94B08C1D
:10814000089580911106882319F080E090E0CECF49
:1081500080E090E0DECF80911006833079F083E0FC
:10816000809310068091B406882341F066E971E19E
:108170008091B2069091B3060C94B08C08958091D2
:108180001006823079F082E0809310068091B40668
:10819000882341F065E871E18091B2069091B306C1
:1081A0000C94B08C089580911006813079F081E0B4
:1081B000809310068091B406882341F064E771E152
:1081C0008091B2069091B3060C94B08C0895809182
:1081D000070180FF1BC08091B406882351F089E31A
:1081E0009BE00E94F393811108C08091450B81119F
:1081F00004C089E39BE00C94E09365E172E1809117
:10820000B2069091B3060E94B08CF3CF089580918E
:10821000070181FF1BC08091B406882351F088E0DC
:108220009BE00E94F393811108C08091140B81118F
:1082300004C088E09BE00C94E09368EE71E18091CB
:10824000B2069091B3060E94B08CF3CF089580914E
:10825000070180FF17C08091B406882331F089E3BD
:108260009BE00E94F393882321F089E39BE00C9428
:10827000F7936FEF71E18091B2069091B3060E947F
:10828000B08CF3CF08958091070181FF17C08091D2
:10829000B406882331F088E09BE00E94F3938823A2
:1082A00021F088E09BE00C94F79362ED71E18091FE
:1082B000B2069091B3060E94B08CF3CF08950E944D
:1082C000889180911206882361F18091DE0A8111E4
:1082D00028C08091AA06811124C081E08093AA065B
:1082E0000E94759080913D06882319F010923D06FA
:1082F0000CC08091AE069091AF06DC01ED91FC912F
:108300000088F189E02D61E019958091B4068823F9
:1083100041F069E471E18091B2069091B3060C944A
:10832000B08C0895CF93DF938091070180FD2AC020
:10833000C0914906D0914A0680914D06882371F07C
:108340008EE30E940F4A813092402CF010924A0630
:10835000109249060AC081E090E003C08EE30E94BB
:108360000F4A90934A06809349068091490690915E
:108370004A068C179D0719F410924B0603C081E042
:1083800080934B06DF91CF910895CF93DF93809137
:10839000070181FD2AC0C0914306D0914406809117
:1083A0004706882371F08FE30E940F4A8130924084
:1083B0002CF010924406109243060AC081E090E02F
:1083C00003C08FE30E940F4A9093440680934306B4
:1083D00080914306909144068C179D0719F41092E2
:1083E000450603C081E080934506DF91CF91089553
:1083F0008091230F833041F12CF48130A9F0823039
:1084000099F02DC086305CF58091A3069091A4066A
:10841000DC01ED91FC910480F581E02D19958091AE
:10842000A1069091A20614C08091A7069091A8067B
:10843000DC01ED91FC910480F581E02D199580918E
:10844000A5069091A60604C08091A3069091A4066B
:10845000DC01ED91FC910480F581E02D199580916E
:10846000AE069091AF06DC01ED91FC91E65BFF4F0B
:108470000190F081E02D19958091AE069091AF06A4
:10848000DC01ED91FC910284F385E02D60E070E069
:1084900019940E948891809112068823D1F08091CE
:1084A000AA068823B1F01092AA060E9443908091F8
:1084B0003D06882389F010923D068091B4068823FA
:1084C00041F06DE571E18091B2069091B3060E9492
:1084D000B08C1092AA0608958091AE069091AF06D6
:1084E000DC01ED91FC910088F189E02D60E01995A7
:1084F000E4CFCF93DF93C091A211D091A311BE011D
:108500008BE69BE00E94667B882329F0BE018BE608
:108510009BE00E947E7B1092A3111092A211DF912A
:10852000CF9108950F931F93CF93DF938091280FDE
:108530009091290FA0912A0FB0912B0F18161906B0
:108540001A061B060CF043C00E9488918091120607
:108550008823C1F10091A2111091A311B8018BE6FB
:108560009BE00E94667B8823D1F0E9E6FDE0C0E055
:10857000D0E0819191918017910761F4CCD7CC0F15
:10858000DD1FCC0FDD1FC559D44F688379838A83E3
:108590009B831DC02196CE31D10559F718C040915B
:1085A000280F5091290F60912A0F70912B0F28E608
:1085B00033E48BE69BE00E94CD7B9093A3118093E4
:1085C000A21105C0DF91CF911F910F9192CFDF9142
:1085D000CF911F910F9108958091DE0A811148C0BB
:1085E0000E94889180917F138823B1F080911206B8
:1085F000882391F01092120610927F130E94AF917F
:1086000080918111882341F064E271E180917F11B2
:10861000909180110E94B08C80914006909141060B
:10862000806290934106809340068091AA06882339
:1086300011F081E001C080E00E94A79081E080936A
:108640003D0627DF8091390F81110FC080912806E8
:10865000882359F025E530E444E650E060E070E01E
:108660008BE69BE00E94CD7B01C01FDDC1DE5ACFAF
:108670000895BEDE0E94534C0E948891809112069C
:108680008111AADF8091B0069091B106DC01ED91D5
:10869000FC910480F581E02D19958091AC069091B4
:1086A000AD06DC01ED91FC910480F581E02D19957A
:1086B0008091040F882359F08091290690912A0611
:1086C000DC01ED91FC910480F581E02D1994089571
:1086D0000E94889180911206882369F07DDF809145
:1086E000B406882341F064E371E18091B206909171
:1086F000B3060C94B08C08958091DE0A81115EC09F
:108700008091AB06823068F08091B406882309F42A
:1087100055C062EE70E18091B2069091B3060C9460
:10872000B08C0E94889180917F13882309F446C001
:1087300080911206811142C081E08093120610924E
:108740007F130E94AF9180918111882341F063EDE6
:1087500070E180917F11909180110E94B08C809186
:1087600040069091410680619093410680934006B7
:108770008091AE069091AF06DC01ED91FC910280F4
:10878000F381E02D19958091AB06811116C04091BF
:108790001E0F50911F0F81E080933D06411551053A
:1087A00059F060E070E02FE531E48BE69BE00E9439
:1087B000CD7B0E94439001C082DDB4CE0895AF927C
:1087C000BF92CF92DF92EF92FF920F931F93CF93BE
:1087D000DF9390919A1191110BC02091BA063091BC
:1087E000BB06309399112093981191E090939A11C0
:1087F0009091901191110BC02091B8063091B9065B
:1088000030938F1120938E1191E090939011A0904E
:108810009811B090991100918E1110918F11D091F3
:10882000B406843608F047C0C82F682F70E080E097
:1088300090E00E942CBA20E030E048EC52E40E9424
:1088400004B66B017C01B501BB0C880B990B0E942F
:108850002EBA9B01AC01C701B6010E948DBA0E94DD
:108860006CB67093BB066093BA06B801110F880B03
:10887000990B0E942EBA9B01AC01C701B6010E9460
:108880008DBA0E946CB67093B9066093B806DD236A
:1088900071F162EB70E18091B2069091B3060E9493
:1088A0003F8B6C2F8091B2069091B3060E94863A5E
:1088B00060EB70E10CC0B092BB06A092BA061093B8
:1088C000B9060093B806DD2391F064EC70E1809165
:1088D000B2069091B306DF91CF911F910F91FF9057
:1088E000EF90DF90CF90BF90AF900C94B08CDF9161
:1088F000CF911F910F91FF90EF90DF90CF90BF909D
:10890000AF900895CF93823069F49091170F209122
:10891000140F3091180F4091150F5091160F609160
:10892000130F0CC09091110F20910E0F3091120F68
:1089300040910F0F5091100F60910D0F60938913AC
:108940005093861340938713309385132093881395
:1089500090938A13909100028917B9F080930002D6
:108960009091B406992389F0C82F67E970E180914E
:10897000B2069091B3060E943F8B6C2F8091B20695
:108980009091B306CF910C946F3ACF9108958330B4
:1089900079F030F4813051F0823091F48BE30BC0E8
:1089A000843041F0853061F482E405C08CE303C07B
:1089B00080E401C081E40E948F8E21E0892B09F4BC
:1089C00020E0822F0895E3DF91E0892708950F9337
:1089D0001F938091861181110CC09DD560938211E7
:1089E00070938311809384119093851181E080931B
:1089F000861180910A028A3AF1F485E0C8DF882363
:108A000071F08AE398E090939B1380939A1390936C
:108A1000B3068093B2068FEF80930A020CC087EDF5
:108A200098E090939B1380939A139093B30680934E
:108A3000B20610920A026FD5009182111091831133
:108A40002091841130918511DC01CB01801B910BA9
:108A5000A20BB30BC397A105B10508F448C05BD5C1
:108A60006093821170938311809384119093851188
:108A700085E08DDF882321F080910A02882349F068
:108A800085E085DF811133C080910A028F3F79F53F
:108A900018C08AE398E090939B1380939A13909365
:108AA000B3068093B2068091B406882331F06DE757
:108AB00070E18AE398E00E94B08C8FEF80930A0205
:108AC00016C087ED98E090939B1380939A13909330
:108AD000B3068093B2068091B406882331F068E62D
:108AE00070E187ED98E00E94B08C10920A021F910D
:108AF0000F9108951092A6118091B406882379F001
:108B00002091F60E8091B2069091B306222319F0BF
:108B100068E370E102C06BE470E10C94B08C0895DE
:108B200081E08093A6118091B406882379F020918A
:108B3000F60E8091B2069091B306222319F06AE0F6
:108B400070E102C06CE170E10C94B08C0895109259
:108B500028061092220610921906109223061092EF
:108B60002406109225061092260681E08093DC0AE6
:108B700040912E0650912F0660E070E026EC35E41F
:108B800080911A0690911B060C94CD7B8091DF0A90
:108B9000882361F18091E10981111CC01092230AA0
:108BA0001092240A1092250A1092260A1092270A7F
:108BB0001092280A10922B0A8091DA0A9091DB0A0F
:108BC000DC01ED91FC910190F081E02D199510925E
:108BD000DC0A089526EC35E445E050E060E070E002
:108BE00080911A0690911B060C94CD7B089560919C
:108BF000B0117091B11180911A0690911B060E94DC
:108C0000667B882319F081E08093AF11089590E08E
:108C1000FC013197E231F10508F04EC08827E15898
:108C2000FE4F8F4F0C948BB5809180008F7703C0DF
:108C3000809180008F7D80938000089580918000D6
:108C4000877FF9CF84B58F7702C084B58F7D84BDCF
:108C500008958091B0008F7703C08091B0008F7D20
:108C60008093B0000895809190008F7707C0809125
:108C700090008F7D03C080919000877F809390004B
:108C800008958091A0008F7707C08091A0008F7D0C
:108C900003C08091A000877F8093A00008958091F9
:108CA00020018F7707C0809120018F7D03C08091C4
:108CB0002001877F8093200108951F93CF93DF9336
:108CC000282F30E0F901EE51F64E8491F901E45677
:108CD000F64ED491F901EA5AF64EC491CC23C1F074
:108CE000162F811194DFEC2FF0E0EE0FFF1FEA5BEF
:108CF000FD4EA591B4918FB7F894111105C09C91C8
:108D0000ED2FE095E92302C0EC91ED2BEC938FBFA2
:108D1000DF91CF911F91089560E087E0CEDF109240
:108D2000DD0A089561E087E0C8DF81E08093DD0A15
:108D30000895CF93DF938091BD11811110C084EF0E
:108D400091E09093BC118093BB118BE290E09093E3
:108D5000BA118093B91181E08093BD1120C0809138
:108D6000B9119091BA118532910514F0049709C098
:108D70008331910514F0029704C0823091052CF0E4
:108D800001979093BA118093B9118091B911909184
:108D9000BA1197FF04C01092BA111092B911C09184
:108DA000B811CC2311F0B8DF01C0BCDF81E08C2703
:108DB0008093B811C091BB11D091BC111C161D0637
:108DC00054F01092BD11A8DF29E037E44AEF50E0DB
:108DD00060E070E007C029E936E4AE010D2E000C1A
:108DE000660B770B80911A0690911B060E94CD7B33
:108DF0009093B7118093B6118091B9119091BA11E7
:108E0000C81BD90BD093BC11C093BB11DF91CF917C
:108E100008950F931F93CF93DF938091DE0A8823E9
:108E200029F0DF91CF911F910F9183CF0091B6115F
:108E30001091B711C0911A06D0911B06B801CE014E
:108E40000E94667B882321F0B801CE010E947E7BC0
:108E5000DF91CF911F910F915FCFCF92DF92EF9271
:108E6000FF921092DE0A20911E0630911F0640915B
:108E7000200650912106609123067091240680916E
:108E80002506909126060E949FB56B017C0120E08B
:108E900030E0A9010E9428BA87FD09C0C0922306CC
:108EA000D0922406E0922506F092260608C0109281
:108EB0002306109224061092250610922606FF9093
:108EC000EF90DF90CF90A5CFEF92FF921F93CF93BB
:108ED000DF9300D0CDB7DEB784E689838CE38A8345
:108EE00088E28B831091B2111330E8F4E12EF12C5B
:108EF00010FF02C011DF01C015DFE1E0F0E0EC0F70
:108F0000FD1FEE0DFF1D408150E060E070E024E6A3
:108F100037E480911A0690911B060E94CD7B1F5F5B
:108F20001093B21103C0F8DE1092B2110F900F909F
:108F30000F90DF91CF911F91FF90EF90089560E027
:108F400088E0BBCE61E089E2B8CE0F931F93CF9348
:108F5000DF9360E08BE2B1DE0091A4111091A511C6
:108F6000C0911A06D0911B06B801CE010E94667B03
:108F7000882341F0B801CE01DF91CF911F910F916D
:108F80000C947E7BDF91CF911F910F910895CF9329
:108F9000DF9390E0FC01E456F64E2491FC01EA5A7E
:108FA000F64E8491882361F190E0880F991FFC01AF
:108FB000E45DFD4EC591D491FC01EA5BFD4EA591A7
:108FC000B491611109C09FB7F894888120958223DC
:108FD0008883EC912E230BC0623061F49FB7F89424
:108FE0003881822F809583238883EC912E2B2C93BC
:108FF0009FBF06C08FB7F894E8812E2B28838FBFC0
:10900000DF91CF9108951F93CF93DF93182FEB013A
:1090100061E0BDDF209711F460E004C0CF3FD105CF
:1090200031F461E0812FDF91CF911F9146CEE12F86
:10903000F0E0EE51F64EE4914E2F50E0FA013197F8
:10904000E231F10508F09DC08827EF56FE4F8F4FA3
:109050000C948BB584B5806884BDC7BD97C084B5BA
:10906000806284BDC8BD92C080918000806880937A
:109070008000D0938900C093880088C080918000D0
:10908000806280938000D0938B00C0938A007EC062
:1090900080918000886080938000D0938D00C09381
:1090A0008C0074C08091B00080688093B000C09341
:1090B000B3006CC08091B00080628093B000C09318
:1090C000B40064C080919000806880939000D09339
:1090D0009900C09398005AC080919000806280935C
:1090E0009000D0939B00C0939A0050C08091900054
:1090F000886080939000D0939D00C0939C0046C0F0
:109100008091A00080688093A0008091A0008F7B58
:109110008093A000D093A900C093A80037C080918D
:10912000A00080628093A000D093AB00C093AA00FF
:109130002DC08091A00088608093A000D093AD00E6
:10914000C093AC0023C080912001806880932001EF
:10915000D0932901C093280119C080912001806219
:1091600080932001D0932B01C0932A010FC08091DE
:109170002001886080932001D0932D01C0932C01A1
:1091800005C0C038D1050CF04CCF46CFDF91CF9150
:109190001F9108950F931F93CF93DF938091B51183
:1091A0009091280681112AC0992309F456C0009194
:1091B000B3111091B411C0911A06D0911B06B801D9
:1091C000CE010E94667B882321F0B801CE010E9467
:1091D0007E7BA8DD2AEC38E442EC51E060E070E0F0
:1091E00080911A0690911B060E94D57B9093B41132
:1091F0008093B31181E08093B51159C08091DD0A4D
:10920000992361F0882329F0DF91CF911F910F916D
:1092100083CDDF91CF911F910F9184CD8823C9F326
:109220006091B3117091B41180911A0690911B0650
:109230000E947E7B2AEC38E444E150E060E070E07C
:1092400080911A0690911B060E94D57B9093B411D1
:109250008093B3111092B5112AC0C0910B02D09126
:109260000C022297D0930C02C0930B021C161D0611
:109270006CF4BE01772787E0C6DECC2321F081E0C5
:109280008093DD0A14C01092DD0A11C06091B31101
:109290007091B41180911A0690911B060E947E7BFA
:1092A0003BDD8FEF90E090930C0280930B02DF91F7
:1092B000CF911F910F9108950F931F93CF93DF9339
:1092C0000091AB111091AC11C091AD11D091AE11C4
:1092D000C00FD11FD093AE11C093AD11BE0177273F
:1092E00087E091DECC2321F081E08093DD0A02C08B
:1092F0001092DD0A10161106ECF58091A9119091DB
:10930000AA11C817D9070CF485C08091AF11882322
:1093100071F01092AA111092A9118CEF9FEF909307
:10932000AC118093AB1181E08093A81173C068E702
:1093300070E080E090E00E94148BDC01CB010A9683
:10934000A11DB11D9093AA118093A91168E270E04C
:1093500080E090E00E94148BDC01CB010A96A11DF5
:10936000B11D66277727681B790B7093AC1160934A
:10937000AB1150C0012B09F44DC08091A9119091FF
:10938000AA118C179D070CF445C08091A811882361
:1093900011F10091B0111091B111C0911A06D09144
:1093A0001B06B801CE010E94667B882399F1B801A3
:1093B000CE010E947E7BB0DC1092AE111092AD11F6
:1093C0001092A81180912806882321F1DF91CF9176
:1093D0001F910F91DFCE69E670E080E090E00E947F
:1093E000148BDC01CB018A569F4FAF4FBF4F909338
:1093F000AA118093A91168E270E080E090E00E94D9
:10940000148BDC01CB010A96A11DB11D9093AC1108
:109410008093AB11DF91CF911F910F910895863307
:1094200008F0865390917B00282F2870977F922B0D
:1094300090937B008770806480937C0080917A0099
:10944000806480937A0080917A0086FDFCCF8091C1
:1094500078002091790090E0922B08953FB7F8941E
:109460008091C3119091C411A091C511B091C61102
:1094700026B5A89B05C02F3F19F00196A11DB11D6F
:109480003FBFBA2FA92F982F8827820F911DA11DAA
:10949000B11DBC01CD0142E0660F771F881F991FE7
:1094A0004A95D1F708958F929F92AF92BF92CF9233
:1094B000DF92EF92FF926B017C01D0DF4B015C01E8
:1094C000C114D104E104F104E9F0C8DFDC01CB01EF
:1094D00088199909AA09BB09883E9340A105B105DD
:1094E00078F321E0C21AD108E108F10888EE880E6D
:1094F00083E0981EA11CB11CC114D104E104F10445
:1095000021F7DECFFF90EF90DF90CF90BF90AF902C
:109510009F908F9008952FB7F8946091BF1170912C
:10952000C0118091C1119091C2112FBF08951F9257
:109530000F920FB60F9211242F933F938F939F9307
:10954000AF93BF938091BF119091C011A091C111B1
:10955000B091C2113091BE1123E0230F2D3720F4BA
:109560000196A11DB11D05C026E8230F0296A11D7D
:10957000B11D2093BE118093BF119093C011A09391
:10958000C111B093C2118091C3119091C411A091E7
:10959000C511B091C6110196A11DB11D8093C311D3
:1095A0009093C411A093C511B093C611BF91AF9110
:1095B0009F918F913F912F910F900FBE0F901F9011
:1095C00018950F931F93CF93DF930091B6111091CD
:1095D000B711C0911A06D0911B06B801CE010E94A6
:1095E000667B8823A1F0B801CE010E947E7B27EF25
:1095F00035E448EB5BE060E070E080911A06909102
:109600001B060E94CD7B9093B7118093B611609199
:10961000B0117091B11180911A0690911B060E94B1
:10962000667B81114BC01092AF118FEF90E0909349
:10963000AE118093AD1176DB68E770E080E090E0DA
:109640000E94148BDC01CB010A96A11DB11D9093E1
:10965000AA118093A91168E270E080E090E00E9476
:10966000148BDC01CB010A96A11DB11D662777275B
:10967000681B790B7093AC116093AB112CE539E446
:1096800044E150E060E070E080911A0690911B0682
:109690000E94D57B9093B1118093B01127EF35E4F0
:1096A00048EB5BE060E070E080911A0690911B0649
:1096B0000E94CD7B9093B7118093B611DF91CF912B
:1096C0001F910F9108958F929F92AF92BF92CF9268
:1096D000EF92FF920F931F93CF93DF932091390660
:1096E000223008F07AC07B018C0180902306909094
:1096F0002406A0902506B090260620E030E0A901BF
:10970000C501B4010E9428BA181654F520E030E0D3
:10971000A901C501B4010E949DB6181654F420E0B9
:1097200030E048E452E4C501B4010E9428BA18169A
:10973000D4F420E030E048E452E4C501B4010E94D2
:109740009DB618169CF420E030E048EC52E4C501C8
:10975000B4010E9428BA87FF09C0CBE4D0E008C05A
:10976000C0E0D0E005C0C2E3D0E002C0C4E6D0E073
:109770008FEF8C0D823070F4209739F06C2FC80178
:109780000E9449726C2FC7010DC0C8010E940A7166
:10979000C70116C08DEF8C0D8330F8F4209779F057
:1097A0006C2FC801DF91CF911F910F91FF90EF9027
:1097B000CF90BF90AF909F908F900C944972C8014A
:1097C000DF91CF911F910F91FF90EF90CF90BF90BD
:1097D000AF909F908F900C940A71DF91CF911F9161
:1097E0000F91FF90EF90CF90BF90AF909F908F9090
:1097F00008958F929F92AF92BF92CF92DF92EF9295
:10980000FF92C0902306D0902406E0902506F090A9
:10981000260620E030E0A901C701B6010E949DB6EE
:1098200020E030E040E05FE387FD0BC0C701B601F8
:109830000E94A0B54B015C010E946CB697FD27C049
:1098400010C0C701B6010E949FB50E946CB697FD7B
:109850001EC06536710581059105DCF424E6822F72
:1098600014C0C501B4010E946CB66536710581054E
:1098700091057CF420E030E040E05FE3C701B601F1
:109880000E94A0B50E946CB684E6861B03C084E6E5
:1098900001C080E0FF90EF90DF90CF90BF90AF903D
:1098A0009F908F9008950F931F93CF93DF93009114
:1098B000130610911406C0911A06D0911B06B80128
:1098C000CE010E94667B882321F0B801CE010E9460
:1098D0007E7B8091DE0A882339F01092DE0ADF91C8
:1098E000CF911F910F9195CADF91CF911F910F9149
:1098F0000895EC981092DF0A68EC70E082E00C9416
:10990000143780913206811105C08091360681118D
:1099100001C0EFCF8091DA0A9091DB0A0E949B8808
:1099200081E08093DF0A64E670E00C94143760E015
:1099300089E2C3D922EA37E442E350E060E070E014
:1099400080911A0690911B060C94CD7B1F920F926A
:109950000FB60F9211240BB60F922F933F934F9394
:109960005F936F937F938F939F93AF93BF93EF9387
:10997000FF938091A7118823B1F0669918C0EE98E3
:1099800025EA37E44CE251E060E070E080911A068D
:1099900090911B060E94CD7B8091A611882339F0FF
:1099A0000E94AD6804C0669B02C0EE98CEDAFF91BB
:1099B000EF91BF91AF919F918F917F916F915F9147
:1099C0004F913F912F910F900BBE0F900FBE0F90B4
:1099D0001F90189581E08093EB0A089581E08093B1
:1099E000EC0A089581E08093ED0A0895CF93DF9308
:1099F000C091EE11D091EF11609117127091181271
:109A0000CE010E94667B81110DC026E73AE74CE249
:109A100051E060E070E0CE010E94CD7B909318127F
:109A200080931712DF91CF910895CF9380911212F6
:109A3000C0910D02811100C1C23009F44FC0C33082
:109A400009F49CC0C13009F027C18091ED0A811151
:109A500023C181E090E00E9428B79093191380936E
:109A6000181362E083E093DA10921112109212132D
:109A7000109211131092161380E090E0FC01EE0F8B
:109A8000FF1FE150FE4E1182108201968830910531
:109A9000A9F71092101210920F1280916A008C6038
:109AA00080936A00ED9A8FB7F894209184003091EA
:109AB00085003093FE112093FD118FBF22EF3CE40F
:109AC0004AEF50E060E070E08091EE119091EF116C
:109AD0000E94CD7B81E080931212DEC08091EC0A5F
:109AE0008111DAC081E090E00E9428B790931B13A7
:109AF00080931A13809104018E7F809304018091DA
:109B0000050181608093050180E097E09093451303
:109B1000809344132EE240EA56E861E070E00E9430
:109B20002A8E809165008B7F8093650010923501AD
:109B300089E0809334018EE2809332018CEF809330
:109B4000300180E980933101109243131092421347
:109B5000109241131092401310923E13EEE1F3E184
:109B60008CED95E08193919323E1EE33F207D1F7E9
:109B7000C1E0C0933F132EEE3CE451C08091EB0A4C
:109B800081118AC081E090E00E9428B790931D1354
:109B900080931C13809104018E7F80930401809137
:109BA000050181608093050180E097E09093D111D9
:109BB0008093D01126E040E052EC61E070E00E941A
:109BC0002A8E809165008B7F80936500109235010D
:109BD00080E18093340186E0809332018EEF8093A0
:109BE000300180E980933101109214131092131305
:109BF0001092CF111092CE1110921513E2EDF1E1F7
:109C00008CED95E08193919321E1EE3EF207D1F73F
:109C10001092CD11C1E0C093CC112AEE3CE44AEF82
:109C200050E060E070E08091EE119091EF110E94A1
:109C3000CD7BC093121230C0C23069F0C330D1F076
:109C4000C13051F58091ED0A811126C08091111328
:109C5000909112131DC08091EC0A81111DC080915A
:109C60001A1390911B130E947E7F80914213909152
:109C700043130EC08091EB0A81110EC080911C131A
:109C800090911D130E947763809113139091141388
:109C9000029711F4C093F40A80910D028230A1F171
:109CA000833009F454C0813009F074C08091ED0A0A
:109CB000882309F46FC0ED98E59A10921112109262
:109CC000171310921213109211131092161380E0B2
:109CD00090E0FC01EE0FFF1FE150FE4E118210825A
:109CE000019688309105A9F71092101210920F1268
:109CF00080911813909119130E94BDB710921212FF
:109D00001092EC0A82E044C08091EC0A882309F4A6
:109D100041C080914413909145130E94088E809118
:109D200031018F7780933101809131018F7E809353
:109D300031011092300180911A1390911B130E94EF
:109D4000BDB7109212121092EB0A83E021C08091ED
:109D5000EB0A8823F9F08091D0119091D1110E94E3
:109D6000088E809131018F7780933101809131018C
:109D70008F7E809331011092300180911C1390915D
:109D80001D130E94BDB7109212121092ED0A81E0CD
:109D900080930D028091EE119091EF11CF910C9470
:109DA000DD7BAF92BF92CF92DF92EF92FF920F9343
:109DB0001F93CF93DF937C016B015A01D0E0C0E089
:109DC0008D2F90E0F701A181B2818A159B05D0F417
:109DD000F601E80FF91F608106E012E921E0332760
:109DE000C6270C0F111D211D311D2BBFF801C79176
:109DF000ED91FC9111970190F081E02DCD01199525
:109E0000DF5FDECFED91FC9111970190F081E02DA5
:109E10006C2FCD01DF91CF911F910F91FF90EF90AB
:109E2000DF90CF90BF90AF901994CF93DF9300D085
:109E30001F921F92CDB7DEB7FE01319625E0DF01FC
:109E40001D922A95E9F724E8298325E52C832AE247
:109E50002D836A834B8345E050E0BF01A2DF65E0BC
:109E600070E080E090E01FDB80E00F900F900F909B
:109E70000F900F90DF91CF910895EF92FF921F9373
:109E8000CF93DF931F92CDB7DEB77C01162FFC0175
:109E9000618172810E94003B65E070E080E090E0AB
:109EA00002DB42E462E4C701C0DF412F60E0C7018A
:109EB000BCDF811162C040E061E0C701B6DF811103
:109EC0005CC040E062E0C701B0DF811156C046E0EF
:109ED00062E0C701AADF811150C040E063E0C70122
:109EE000A4DF81114AC040E064E0C7019EDF11E0B9
:109EF000811110E040E065E0C70197DF811101C0EA
:109F00001F5F40E066E0C70190DF811101C01F5F65
:109F100040E067E0C70189DF811101C01F5F40E0B9
:109F200068E0C70182DF811101C01F5F40E069E086
:109F3000C7017BDF811101C01F5F44E06AE0C701F8
:109F400074DF811101C01F5F44E06AE0C7016DDF6B
:109F5000811101C01F5F62E370E080E090E0A3DA4E
:109F600082E8898341E050E0BE016F5F7F4FC70107
:109F700018DF81E0183011F0111180E00F90DF91AF
:109F8000CF911F91FF90EF900895CF93DF9300D072
:109F90001F92CDB7DEB72AEA2983FC0120812A83EC
:109FA0006B834C8344E050E0BE016F5F7F4FF9DE6E
:109FB0000F900F900F900F90DF91CF9108953FB7C2
:109FC000F89420E0822F90E0841795079CF4FC0120
:109FD000EE0FFF1FEF5FFD4EA081B181880F991F2B
:109FE000FB01E80FF91FCD0196958795918380833A
:109FF0002F5FE8CF3FBF1092161308952F923F9224
:10A000005F926F927F928F929F92AF92CF92DF92E8
:10A01000EF92FF920F931F93CF93DF931F921F92A4
:10A02000CDB7DEB76DB67EB60E947C800E9471808F
:10A030000E94C880029709F022C20E94B380882340
:10A0400009F418C2C0901712D0901812E090EE11C7
:10A05000F090EF11B601C7010E94667B8823E9F0FA
:10A06000F701E250FE4F00E010E0819191918C15D4
:10A070009D0569F450DA000F111F000F111FF70141
:10A08000E00FF11F608371838283938307C00F5FAA
:10A090001F4F0E31110549F701C0A8DC1092EE0ADE
:10A0A000EDB6FEB64091F10A5091F20ACA01880F4E
:10A0B000991F2DB73EB7281B390B0FB6F8943EBF3A
:10A0C0000FBE2DBF0DB71EB70F5F1F4F8091F40A53
:10A0D000823061F0833021F1813009F070C0B80125
:10A0E00080911813909119136ADF33C03FB7F89429
:10A0F00020E0822F90E08417950774F4880F991F51
:10A10000F801E80FF91FDC01A25EBC4E8D919C9115
:10A11000918380832F5FEDCF3FBF10923E1319C014
:10A120003FB7F89420E0822F90E08417950774F4ED
:10A13000880F991FF801E80FF91FDC01AE52BE4EDF
:10A140008D919C91918380832F5FEDCF3FBF1092C3
:10A15000151320E06AE071E0822F90E04091F10A4F
:10A160005091F20A8417950754F5689FF001699F92
:10A17000F00D1124E456F04FA085B1858C91882311
:10A18000E1F0A081B1813C91C801830F911D830F43
:10A19000911DDC0112978D919C91A281B3814D910B
:10A1A0005C9111970480F581E02D4817590711F44F
:10A1B000108203C070838D939C932F5FCDCF0FB619
:10A1C000F894FEBE0FBEEDBE80919610882321F05C
:10A1D00085E990E10E94E4808091A010882321F01D
:10A1E0008FE990E10E94E4808091AA10882321F0F9
:10A1F00089EA90E10E94E4808091B410882321F0E4
:10A2000083EB90E10E94E4808091EF0A882309F4B7
:10A2100065C08091AA10811105C08091B410882377
:10A2200009F450C08091AD109091AE10E091B11042
:10A23000F091B210238134812817390724F48085E6
:10A24000811109C00EC0218132818217930734F435
:10A250008085811106C088E090E005C080E190E033
:10A2600002C080E290E02091B7103091B810E091E8
:10A27000BB10F091BC10438154814217530724F462
:10A280002085222349F00AC04181528124173507D5
:10A290003CF42085222311F0816003C0846001C05A
:10A2A000826020919010309191102817390719F48D
:10A2B0001092921007C0909391108093901081E0BB
:10A2C000809392108091901090919110429709F490
:10A2D000DAC081E08093B6108093AC10EDE3F0E13A
:10A2E00080E490E19A83898398EE892E93E0992EF9
:10A2F00055245394CF010197DC018C91882309F4F4
:10A30000ACC0E480F580D70117968C91179788230D
:10A3100009F4A3C08081882309F49FC04181528140
:10A3200018966C918401041B150B101611061CF075
:10A330008A01085E134020E030E022242394312C6F
:10A340008FE097E2A12CC62ED12C2C143D04ACF545
:10A350006430A9F040F4623071F0633019F5C9013E
:10A3600080539A4F13C0653071F06630D9F4C9013B
:10A370008E549A4F0BC0C9018A529A4F07C0C90127
:10A3800088539A4F03C0C90182549A4FDC01129638
:10A390008D919C911397841B950B97FF03C091950A
:10A3A000819591098017910714F4A22C8C01BFEFBD
:10A3B0002B1A3B0A2E5F3F4FC8CF81E08A0DD70191
:10A3C00019969C919923F1F1643099F028F4623048
:10A3D00041F0633049F036C06530A1F06630D9F005
:10A3E00031C0813021F52DC0813049F1833051F5E4
:10A3F0001EC0813011F1823011F1833011F18430AF
:10A4000009F515C08130B9F08230B9F08430C9F057
:10A410008530C1F40CC0813061F0823061F083304E
:10A4200061F0843061F0853061F0863059F481E06C
:10A4300009C086E007C085E005C084E003C083E072
:10A4400001C082E0A981BA819C91981302C0108258
:10A4500004C05082A981BA818C93379629813A81B0
:10A46000295F3F4F3A83298330E1E139F30709F04F
:10A4700041CF03C00E948880B9DA81E066C00E94A3
:10A48000888080E062C0E0909310F09094101E14D9
:10A490001F040CF055C08091AB100091EE1110918B
:10A4A000EF1160911512709116128823B1F081E0BE
:10A4B0008093AC10C8010E94667B811115C0A70172
:10A4C000FF0C660B770B25ED3AE7C8010E94CD7BA8
:10A4D000909316128093151207C0C8010E94667BE4
:10A4E000811102C01092AC108091B5100091EE1154
:10A4F0001091EF1160911312709114128823D1F012
:10A5000081E08093B610C8010E94667B8111E6CE7F
:10A510004091931050919410052E000C660B770B10
:10A5200022ED3AE7C8010E94CD7B909314128093EC
:10A530001312D4CEC8010E94667B8111CFCE02C017
:10A540001092AC101092B610C9CE0FB6F8947EBE21
:10A550000FBE6DBE0F900F90DF91CF911F910F91A5
:10A56000FF90EF90DF90CF90AF909F908F907F9073
:10A570006F905F903F902F9008951F920F920FB6AB
:10A580000F9211240BB60F922F933F934F938F93FB
:10A590009F93EF93FF938091840090918500209189
:10A5A000FD113091FE11821B930B2091840030919C
:10A5B00085003093FE112093FD11803727E192072B
:10A5C00070F1909300128093FF118091111390917C
:10A5D0001213029751F4909111128091171398134E
:10A5E0003CC081E0809316133EC08091111390917E
:10A5F0001213892B49F481E090E090931213809319
:10A6000011131092FC112FC080911113909112130D
:10A61000019761F5809111128430D8F527C02091FF
:10A620001112283008F047C09C012C5D3540293BB1
:10A630003B4068F4E0911112EF5FE0931112F0E0FB
:10A64000EE0FFF1FE150FE4E9183808334C0809156
:10A65000111390911213029771F583E090E090939B
:10A660001213809311131092111225C080911113AF
:10A67000909112130397B9F79091111280911713CB
:10A680009813F1CF80911713843068F382E090E043
:10A69000E6CF8091FC118F5F8093FC11863018F318
:10A6A00082E090E090931213809311138091111225
:10A6B00080931713D8CFFF91EF919F918F914F9176
:10A6C0003F912F910F900BBE0F900FBE0F901F90D8
:10A6D00018950F931F938091F41181110DC00E9462
:10A6E0008B4A6093F0117093F1118093F211909363
:10A6F000F31181E08093F4110E948B4A0091F011D4
:10A700001091F1112091F2113091F311DC01CB0184
:10A71000801B910BA20BB30B893E9340A105B105A1
:10A72000A8F08AE30E948F8E892B11F060E001C0AF
:10A7300061E08AE30E945D460E948B4A6093F011BB
:10A740007093F1118093F2119093F3111F910F9177
:10A7500008950F931F930E948B4A0091C811109186
:10A76000C9112091CA113091CB11DC01CB01801BA2
:10A77000910BA20BB30B85339142A105B10518F0E3
:10A7800081E08093C7111F910F91A3CFFC0180E05E
:10A7900090E06150710977FD18C02191022E000CE4
:10A7A000330B322F22278227932728E0AC01440F56
:10A7B000551F97FF06C0CA0131E2832730E1932776
:10A7C00001C0CA01215091F7E4CF08950C94E740ED
:10A7D0000C9427410C9407410C9443410C94F5824E
:10A7E0000C942E8380912512882319F00E94F58203
:10A7F00002C00E942E839091251281E089278093C8
:10A8000025120895CF93DF93CDB7DEB765970FB6C6
:10A81000F894DEBF0FBECDBF8091680E9091690E97
:10A820002091660E3091670E3A8329839C838B8337
:10A8300081E08D8B82E08F938DB79EB745970FB6E1
:10A84000F8949EBF0FBE8DBFADB7BEB7119685E120
:10A85000FE01319601900D928A95E1F788E09BE028
:10A860000E9448920FB6F894DEBF0FBECDBF809114
:10A87000B406882381F069EE73E18091B20690916D
:10A88000B30665960FB6F894DEBF0FBECDBFDF915D
:10A89000CF910C94B08C65960FB6F894DEBF0FBEC6
:10A8A000CDBFDF91CF910895CF93DF93CDB7DEB7C2
:10A8B00065970FB6F894DEBF0FBECDBF8091680ECE
:10A8C0009091690E2091660E3091670E3A8329832C
:10A8D0009C838B8381E08D8B82E08F938DB79EB7B5
:10A8E00045970FB6F8949EBF0FBE8DBFADB7BEB7EC
:10A8F000119685E1FE01319601900D928A95E1F75E
:10A9000089E39BE00E9448920FB6F894DEBF0FBE29
:10A91000CDBF8091B406882381F067E174E1809116
:10A92000B2069091B30665960FB6F894DEBF0FBEDF
:10A93000CDBFDF91CF910C94B08C65960FB6F89493
:10A94000DEBF0FBECDBFDF91CF9108950E94F5828B
:10A950004091890F50918A0F60E070E02EE233E859
:10A960008BE69BE00E94CD7B90937B1380937A13C0
:10A970008091B406882341F069E873E18091B206C2
:10A980009091B3060C94B08C08950E942E83409150
:10A99000890F50918A0F60E070E025EF32E88BE676
:10A9A0009BE00E94CD7B90937B1380937A138091E0
:10A9B000B406882341F066E773E18091B206909176
:10A9C000B3060C94B08C089580914D06882339F01D
:10A9D00089E39BE00E94E09327E231E406C089E32B
:10A9E0009BE00E94F79327EE30E44CE251E060E0F8
:10A9F00070E08BE69BE00E94CD7B8091B4068823BB
:10AA000041F064E074E18091B2069091B3060C9439
:10AA1000B08C089580914706882339F088E09BE048
:10AA20000E94E09323E431E406C088E09BE00E94AA
:10AA3000F79327E031E44CE251E060E070E08BE610
:10AA40009BE00E94CD7B8091B406882341F066EDA7
:10AA500073E18091B2069091B3060C94B08C089586
:10AA600089E39BE00E94F39381110C94E7400C94DE
:10AA7000274188E09BE00E94F39381110C940741E9
:10AA80000C94434169E081E00C94788F68E081E0A8
:10AA90000C94788F67E081E00C94788F61E081E01E
:10AAA0000C94788F69E080E00C94788F68E080E007
:10AAB0000C94788F67E080E00C94788F61E080E000
:10AAC0000C94788F8CE00C94C28F8BE00C94C28F26
:10AAD0008AE00C94C28F89E00C94C28F88E00C94B9
:10AAE000C28F87E00C94C28F86E00C94C28F85E001
:10AAF0000C94C28F84E00C94C28F83E00C94C28FBC
:10AB000082E00C94C28F81E00C94C28F8CE00C9494
:10AB1000E88F8BE00C94E88F8AE00C94E88F89E052
:10AB20000C94E88F88E00C94E88F87E00C94E88F11
:10AB300086E00C94E88F85E00C94E88F84E00C9418
:10AB4000E88F83E00C94E88F82E00C94E88F81E03A
:10AB50000C94E88F8CE00C940E908BE00C940E908B
:10AB60008AE00C940E9089E00C940E9088E00C948E
:10AB70000E9087E00C940E9086E00C940E9085E089
:10AB80000C940E9084E00C940E9083E00C940E9044
:10AB900082E00C940E9081E00C940E900C942B901B
:10ABA0000C9437900F931F93CF93DF930091201253
:10ABB00010912112C0911A06D0911B06B801CE0146
:10ABC0000E94667B882379F0B801CE010E947E7BCB
:10ABD00080911C0690911D06DC01ED91FC9100A076
:10ABE000F1A1E02D199500911E1210911F12C09134
:10ABF0001A06D0911B06B801CE010E94667B8823FD
:10AC000021F0B801CE010E947E7B72988091B4063B
:10AC1000882361F068E173E18091B2069091B306F8
:10AC2000DF91CF911F910F910C94B08CDF91CF9158
:10AC30001F910F910895CF93DF938091791388230B
:10AC400021F11092791360E088E00E945D46C09186
:10AC50007A13D0917B13BE018BE69BE00E94667B4A
:10AC6000882329F0BE018BE69BE00E947E7B8091C9
:10AC7000B406882371F06DEB73E18091B206909178
:10AC8000B306DF91CF910C94B08CDF91CF910C94EF
:10AC90001E94DF91CF91089580917913811102C0A4
:10ACA0000C941E940895CF93DF9380917C13882396
:10ACB00011F10E94F58210927C13C0917A13D09109
:10ACC0007B13BE018BE69BE00E94667B882329F004
:10ACD000BE018BE69BE00E947E7B8091B4068823B8
:10ACE00071F064EA73E18091B2069091B306DF914E
:10ACF000CF910C94B08CDF91CF910C944383DF9172
:10AD0000CF9108950C94438380912612882319F0E3
:10AD10000E94F58202C00E9468849091261281E010
:10AD200089278093261208950C9468840C947B8460
:10AD30000C94928480912412882319F00E947B84C1
:10AD400002C00E9492849091241281E0892780930E
:10AD5000241208950C94BC840E94BC848091AE0699
:10AD60009091AF06DC01ED91FC9104A0F5A1E02DDE
:10AD700019940C94F88480912312882319F00E946E
:10AD8000BC8402C00E94F8849091231281E089273C
:10AD90008093231208950C9413850C942E85809132
:10ADA0002212882319F00E94138502C00E942E856A
:10ADB0009091221281E089278093221208950E94A7
:10ADC000814C8091B4068823D1F02091620F80914C
:10ADD000B2069091B306211107C02091650F211191
:10ADE00003C060E273E109C02091DF0A222319F059
:10ADF0006FE573E102C06BE473E10C94B08C0895CD
:10AE00008091DF0A81110C94794C0C94814C0E9442
:10AE1000794C8091B406882341F06AE673E1809111
:10AE2000B2069091B3060C94B08C08950C949045A2
:10AE30008091A61181110C947A450C9490450C9444
:10AE40007A450E947E838091AE069091AF06DC0128
:10AE5000ED91FC9102A0F3A1E02D1994CF93DF9323
:10AE6000C0911A06D0911B06609120127091211298
:10AE7000CE010E94667B811129C040911D1250E0D5
:10AE800060E070E027E937E6CE010E94D57B909321
:10AE900021128093201280911C0690911D06DC01E6
:10AEA000ED91FC91068CF78DE02D19958091370678
:10AEB000882361F060911E1270911F1280911A0612
:10AEC00090911B060E94667B882371F08091B406E6
:10AED0008823E9F06FE073E18091B2069091B306A8
:10AEE000DF91CF910C94B08C0E94B56725EB37E6CB
:10AEF00044E650E060E070E080911A0690911B06F5
:10AF00000E94D57B90931F1280931E12DFCFDF919A
:10AF1000CF9108950E94974C8091B406882341F008
:10AF200064EE72E18091B2069091B3060C94B08CFD
:10AF30000895E0911B12F0911C1282810E943C7DC9
:10AF40008091B406882341F066EC72E18091B206EC
:10AF50009091B3060C94B08C08958091A71188232A
:10AF600019F00E943C6802C00E9426688091B406D5
:10AF7000882379F02091F60E8091B2069091B30665
:10AF8000222319F06AE872E102C063EA72E10C94CC
:10AF9000B08C08950C944942CF938091E00A8823A5
:10AFA00009F482C00E9452689091DE0A882341F021
:10AFB00091117AC080913E06882309F447C074C07D
:10AFC000911172C08091B4068823D1F06BE672E1D2
:10AFD0008091B2069091B3060E943F8B8091DF0A68
:10AFE000882341F060E672E18091B2069091B30649
:10AFF0000E943F8B8091B2069091B3060E949D8C77
:10B000000E94FB6881E080932706809107028130CF
:10B0100009F04AC08091300F882309F445C080911F
:10B02000F60E882361F18091A611882341F124EB6B
:10B0300037E942E350E060E070E08BE69BE00E947D
:10B04000D57B90931A12809319122EC082E08093C0
:10B050003E068091B406882341F067E772E1809153
:10B06000B2069091B3060E94B08CC1E0C0933D0639
:10B070000E9449420E94FB68C093270615C0409178
:10B08000F80E5091F90E141615065CF4052E000CFE
:10B09000660B770B2BE630E48BE69BE0CF910C94AC
:10B0A000CD7BCF910C946B40CF9108952F923F921E
:10B0B0004F925F926F927F928F929F92AF92BF92C8
:10B0C000CF92DF92EF92FF920F931F93CF93DF9374
:10B0D00000D01F92CDB7DEB75C010E9439430E94B9
:10B0E00002840E9439848091B2069091B3060E9436
:10B0F0009D8C0E947B6E24E0A216B10409F49CC0D2
:10B100000CF04FC0A3E0AA16B10409F03CC18CE1D9
:10B1100090E00E9428B79C838B838AEE95E0AB81F8
:10B12000BC8111969C938E931396BC92AE9212970B
:10B1300081E09FEF15969C938E9314978FEF90E08C
:10B1400017969C938E93169719961C921E92189799
:10B1500058961C925897CD010E94887E8EED95E0FE
:10B16000EB81FC8191838083E0911B12F0911C1292
:10B17000D08C009101111091021116950795E09065
:10B18000FF10F0900011F694E79464E375E180916C
:10B19000B2069091B3060E94B08C812C99249394AE
:10B1A00012C1B5E0AB16B10409F4A6C0E6E0AE16D4
:10B1B000B10409F0E8C08CE190E00E9428B79C83BC
:10B1C0008B838AEE95E0AB81BC8111969C938E9324
:10B1D0001396BC92AE92129781E09FEF15969C93C6
:10B1E0008E9314978FEF90E017969C938E931697FB
:10B1F00019961C921E92189758961C925897CD013A
:10B200000E94887E8EED95E0EB81FC8191838083A6
:10B21000E0919E06F0919F06D08C00914011109114
:10B22000411116950795E0903E11F0903F11F6946C
:10B23000E79467E675E1A0C08CE190E00E9428B732
:10B240009C838B838AEE95E0AB81BC8111969C93A5
:10B250008E931396BC92AE92129781E09FEF159653
:10B260009C938E9314978FEF90E017969C938E93F8
:10B27000169719961C921E92189758961C925897DA
:10B28000CD010E94887E8EED95E0EB81FC8191835B
:10B290008083009116111091171116950795E09073
:10B2A0001411F0901511F694E7948091E40E8C50EF
:10B2B000823040F4E091B006F091B106D08C67EA9C
:10B2C00075E15AC08091230F823009F07AC08091D5
:10B2D000E20E8C3009F075C0E0919E06F0919F0659
:10B2E000D08C67E875E18091B2069091B3060E9418
:10B2F000B08C8824839466C08CE190E00E9428B7CB
:10B300009C838B838AEE95E0AB81BC8111969C93E4
:10B310008E931396BC92AE92129781E09FEF159692
:10B320009C938E9314978FEF90E017969C938E9337
:10B33000169719961C921E92189758961C92589719
:10B34000CD010E94887E8EED95E0EB81FC8191839A
:10B350008083E091AC06F091AD06D08C00912B116A
:10B3600010912C1116950795E0902911F0902A1153
:10B37000F694E79467E475E18091B2069091B30684
:10B380000E94B08C1EC06BE175E18091B206909175
:10B39000B3060F900F900F900F90DF91CF911F91F8
:10B3A0000F91FF90EF90DF90CF90BF90AF909F9064
:10B3B0008F907F906F905F904F903F902F900C9464
:10B3C000B08C812C912C0E947B6E6EE075E1809197
:10B3D000B2069091B3060E94B08C62E075E1809154
:10B3E000B2069091B3060E943F8BB8018091B206DD
:10B3F0009091B3060E94E93B66EF74E18091B2063A
:10B400009091B3060E943F8BB7018091B206909154
:10B41000B3060E94E93B6AEE74E18091B206909116
:10B42000B3060E943F8B8D2D0E94576E8091B2060D
:10B430009091B3060E949D8CAB81BC81ED91FC91F3
:10B4400011970280F381E02DCD011995CA2C8A2D28
:10B450000E94A57D8D3D9540A8F464E378E08A2D97
:10B460000E949D7DEB81FC81F78AE68AB70182818B
:10B470000E94B57D6CED75E08A2D0E94A17DDD20D6
:10B48000C1F01AC064E873E08A2D0E94A17DAB81EF
:10B49000BC8157961C930E935697B80112968C91C7
:10B4A0000E94B57D6CED75E08A2D0E949D7DDD20AA
:10B4B00019F03324339401C0312C21E02983212C4D
:10B4C0002A830E94FE4F8091AA10882359F1AB81F4
:10B4D000BC81ED91FC9111976091AF107091B0100B
:10B4E0000190F081E02DCD0119958C2D0E94A57D54
:10B4F0008D3DB5E09B075CF48438E3E09E0784F063
:10B500008C018D3D954074F00CED15E00BC07C0175
:10B51000853398403CF064E3E62E68E0F62E02C0E6
:10B5200004E813E02A8121111FC08091A010882314
:10B53000C9F1E091A710F091A81085819681409102
:10B54000A3105091A4109C012153310942175307B5
:10B550004CF1C196841795072CF10E948B4A641513
:10B56000750586059705F0F08091A0108823C1F03D
:10B570004091A3105091A410E091A710F091A81051
:10B58000858196819C01285C3109421753072CF074
:10B5900088539F4F841795071CF481E0382605C017
:10B5A00021E02A83222009F47CC0332009F445C01D
:10B5B000DD20F9F064E873E08C2D0E94A17D9920D4
:10B5C00009F458C06091FE0E7091FF0E41E08C2D81
:10B5D0000E945C7D0E940291AB81BC8112968C918D
:10B5E0000E94A57D08171907ACF38C2D0E942E7DB3
:10B5F00041C064E378E08C2D0E949D7D9920B1F0DC
:10B600006091FE0E7091FF0E40E08C2D0E945C7DDB
:10B610000E940291AB81BC8112968C910E94A57D03
:10B620008E159F05ACF38C2D0E942E7DEB81FC8145
:10B63000F78AE68AB701828110C0DD20B1F064E3A9
:10B6400078E08C2D0E949D7DAB81BC815796FC9249
:10B65000EE925697B70112968C910E94B57D6CEDD3
:10B6600075E08C2D0E94A17D12C064E873E08C2DE2
:10B670000E94A17DEB81FC81178B068BB801828132
:10B680000E94B57D6CED75E08C2D0E949D7D0E9421
:10B690008B4A2B013C01F8EC4F0E511C611C711CB4
:10B6A0001A8229812223D9F1809196108823A9F149
:10B6B0004091991050919A10E0919D10F0919E1038
:10B6C000858196819C01285C3109421753072CF033
:10B6D00088539F4F8417950704F581E0D826809101
:10B6E000B2069091B306DD2039F06BED74E10E9453
:10B6F000B08C82E090E006C069EC74E10E94B08CEE
:10B7000081E090E00E940A840E948B4AAB81BC8158
:10B710005896DC922224239403C0212C1EC0212C95
:10B7200080919610882309F472C2E0919D10F091E7
:10B730009E10858196814091991050919A109C019C
:10B7400021533109421753070CF461C2C19621E01D
:10B750002983841795070CF45AC20E9486800E94A0
:10B76000313B8BE69BE00E94DD7B8091F80A8823C9
:10B7700009F4A7CE8091FA0A882309F4A2CE0E9488
:10B78000313B0E94A73E8823D1F384E0A816B10480
:10B79000D9F134F4B3E0AB16B10409F438C1C4C133
:10B7A000E5E0AE16B10409F4CDC0F6E0AF16B10481
:10B7B00009F0BAC11093F20E0093F10EF092F40E5C
:10B7C000E092F30ED092F50EB8018CE291E00E9467
:10B7D000C23AB7018EE291E00E94C23A6D2D80E339
:10B7E00091E00E941E3CB80186E00E94D37CB70124
:10B7F00086E00E94B87CE0919E06F0919F06D08E74
:10B800006CED75E086E091C08820C1F01093F20ED7
:10B810000093F10EF092F40EE092F30ED092F50E3A
:10B82000B8018CE291E00E94C23AB7018EE291E049
:10B830000E94C23A6D2D80E391E017C01093E60E8E
:10B840000093E50EF092E80EE092E70ED092E90E3A
:10B85000B80180E291E00E94C23AB70182E291E031
:10B860000E94C23A6D2D84E291E00E941E3CB80114
:10B8700084E00E94D37CB70184E00E94B87C8820D9
:10B8800049F0E0919E06F0919F06D08E6CED75E038
:10B8900084E04BC0E091B006F091B106D08E80916B
:10B8A000E40E8D3029F4E0912812F0912912D08E07
:10B8B0006CED75E084E00E94B57D66E970E080E0A3
:10B8C00090E00E94534A8091E40E8D3011F584E09F
:10B8D0000E94A57DA091B006B091B1068D3D954026
:10B8E0004CF0ED91FC9111970190F081E02D6FEFFC
:10B8F0007FEF08C0ED91FC9111970190F081E02D50
:10B9000061E070E0CD0119958091B0069091B1068B
:10B910006FC08091B0069091B106DC01ED91FC9171
:10B920000480F581E02D1995FFC00E94B57D66E980
:10B9300070E080E090E00E94534A80919E069091D2
:10B940009F06EBCF1093ED0E0093EC0EF092EF0EEE
:10B95000E092EE0ED092F00EB80187E291E00E94E4
:10B96000C23AB70189E291E00E94C23A6D2D8BE2A2
:10B9700091E00E941E3CB80185E00E94D37CB70193
:10B9800085E00E94B87CE091AC06F091AD06D08EC7
:10B990006CED75E085E00E94B57D66E970E080E0C1
:10B9A00090E00E94534A8091E30E8D3059F585E076
:10B9B0000E94A57DA091AC06B091AD068D3D95404D
:10B9C0004CF0ED91FC9111970190F081E02D6FEF1B
:10B9D0007FEF08C0ED91FC9111970190F081E02D6F
:10B9E00061E070E0CD0119958091AC069091AD06B3
:10B9F000DC01ED91FC910190F081E02D60E070E0C0
:10BA0000199592C08091AC069091AD0686CF1093A7
:10BA1000010F0093000FF092030FE092020FD092FB
:10BA2000FA0EB8018BE391E00E94C23AB7018DE3B0
:10BA300091E00E94C23A6D2D85E391E00E941E3C88
:10BA4000B80183E00E94D37CB70183E00E94B87CF8
:10BA50008091FA0EE0911B12F0911C12808F809160
:10BA6000FA0E0E948D3A83E00E94A57D2091FA0E85
:10BA7000222369F1B9E0BC1538F020910111309111
:10BA800002113695279502C02EEE32E082179307F9
:10BA900009F44AC06091FE0E7091FF0E41E083E010
:10BAA0000E945C7D0E940291EB81FC8182810E9458
:10BAB000A57D08171907B4F383E00E942E7DAB81A2
:10BAC000BC8157961C930E935697B80129C029E064
:10BAD0002C1508F49EC02091FF103091001136956E
:10BAE00027958217930701F16091FE0E7091FF0E6A
:10BAF00040E083E00E945C7D0E940291EB81FC812A
:10BB000082810E94A57D8E159F05B4F383E00E947B
:10BB10002E7DAB81BC815796FC92EE925697B70171
:10BB200012968C910E94B57D8091B2069091B306D9
:10BB30000E949D8C0E947B6EB4E0AB16B10459F05C
:10BB4000E5E0AE16B10451F0F3E0AF16B10471F4C4
:10BB50006FE774E105C06FEA74E102C066E974E161
:10BB60008091B2069091B3060E94B08C0E947B6EC9
:10BB700064E774E18091B2069091B3060E94B08CA4
:10BB800068E674E18091B2069091B3060E943F8B03
:10BB9000B8018091B2069091B3060E94E93B6CE532
:10BBA00074E18091B2069091B3060E943F8BB70179
:10BBB0008091B2069091B3060E94E93B60E574E182
:10BBC0008091B2069091B3060E943F8B8D2D0E940A
:10BBD000576E8091B2069091B3060E949D8C0F9093
:10BBE0000F900F900F90DF91CF911F910F91FF90C9
:10BBF000EF90DF90CF90BF90AF909F908F907F900D
:10BC00006F905F904F903F902F900C9435841982E5
:10BC1000A4CD2AEC38E065CFCF93DF93CDB7DEB764
:10BC200028970FB6F894DEBF0FBECDBF80912712C4
:10BC30008823E1F1109227120E94AD8381E0809366
:10BC400003028091B506882389F161E474E1809153
:10BC5000B2069091B3060E943F8BE091F40AE43063
:10BC60000CF0E0E08AEB95E09A83898386EB95E01F
:10BC70009C838B8381EB95E09E838D838CEA95E09A
:10BC800098878F83EE0FFF0BEC0FFD1F6181728190
:10BC90008091B2069091B30628960FB6F894DEBF55
:10BCA0000FBECDBFDF91CF910C94B08C28960FB60C
:10BCB000F894DEBF0FBECDBFDF91CF910895809184
:10BCC0002712811113C00E94394381E0809327120B
:10BCD0000E94C9838091B406882341F062E374E135
:10BCE0008091B2069091B3060C94B08C0895809127
:10BCF00035129091361291609093361280933512DE
:10BD00000895809135129091361280689093361282
:10BD1000809335120895809135129091361280618A
:10BD200090933612809335120895FC018281882306
:10BD300071F08381882359F013828091351290919C
:10BD4000361224E08227909336128093351208959C
:10BD5000FC018281882371F0838181110BC081E015
:10BD600083838091351290913612846090933612BD
:10BD7000809335120895FC018481882371F08581B8
:10BD8000882359F01582809135129091361228E05F
:10BD9000822790933612809335120895FC01848196
:10BDA000882371F0858181110BC081E085838091AA
:10BDB0003512909136128860909336128093351226
:10BDC0000895809135129091361220E28227909347
:10BDD0003612809335120895809135129091361263
:10BDE000806290933612809335120895DC01ED91B4
:10BDF000FC910680F781E02D60E070E0199477FFF8
:10BE000003C07195619571096F3F710519F014F0C8
:10BE10006FEF70E080913512909136128C7B9170AB
:10BE2000909336128093351280913512909136128C
:10BE30006F30710514F480641FC06733710514F40A
:10BE400081641AC06F3571051CF48164906114C05F
:10BE5000673871051CF4816490630EC06F3A7105F8
:10BE60001CF48164906408C0673D71051CF4816412
:10BE7000906502C08164906690933612809335126B
:10BE8000089580E094E090933612809335120895DF
:10BE90008091351290913612926090933612809371
:10BEA000351280913512909136128064909336123B
:10BEB000809335120895089508950895089508957A
:10BEC0000895089508950895089580E008950895C7
:10BED000089508950895089508950895089508957A
:10BEE000089508950895089508950895089508956A
:10BEF0000895089580E0089508950895FC016483ED
:10BF00000895FC0162830895FC0113821482158256
:10BF1000168217821086118608950895089508954F
:10BF2000FC0183810895FC0165830895FC0164830D
:10BF30000895FC0160870895FC0166830895FC0163
:10BF40008281089581E080932D126CED75E00C9450
:10BF5000EE7C6CED75E080E00C94EE7CFC011282CE
:10BF600013821482158261E086E10E94C74761E076
:10BF700086E10E945D46E2E7F0E080818160808397
:10BF800010923612109235120895FF920F931F935C
:10BF9000CF93DF938C01C62FF42ED22F6AED70E081
:10BFA000DC011A968D919C911B970E94127AF801E0
:10BFB00082859385DC01ED91FC910190F081E02D6B
:10BFC0006C2F1995F80182859385DC01ED91FC9128
:10BFD0000190F081E02D6F2D1995F80182859385F0
:10BFE000DC01ED91FC910190F081E02D6D2F199510
:10BFF000EC2FF0E0BF0166527F4F6F0D711D6D0F8A
:10C00000711D6F777727F80182859385DF91CF9136
:10C010001F910F91FF900C94127A242F462F6CE4FD
:10C02000B4CF77FF03C071956195710920E0462F69
:10C030006EE2ABCF462F20E067E4A7CF462F20E08B
:10C0400066E4A3CF262F64E4A0CFCF92DF92FF92C5
:10C050000F931F93CF93DF938C01F62E443F81E023
:10C06000580738F0413187E2580728F040E157E29D
:10C0700002C044EF51E0243F81E0380738F0E90185
:10C080002131374228F0C0E1D7E202C0C4EFD1E04D
:10C09000CA01845F914022E3C22ED12CB6010E94D6
:10C0A00064B5462F2F2D62E4C8016FDFCE01845F97
:10C0B0009140B6010E9464B5462F2F2D63E4C8015C
:10C0C000DF91CF911F910F91FF90DF90CF905DCFC7
:10C0D000242F462F62E559CF242F462F61E555CFF7
:10C0E000262F40E06FE351CF262F40E06EE34DCF87
:10C0F000262F40E06DE349CF462F20E06FE445CF87
:10C10000462F20E06DE441CFFC016283611104C041
:10C1100020E040E06BE439CF089577FF03C07195CC
:10C120006195710920E0462F6BE42FCF10922D12FC
:10C1300022EA3FE544EF51E060E070E08091731245
:10C14000909174120E94CD7B90932C1280932B12AD
:10C15000089580917A1281110AC080912D1288234E
:10C1600031F060ED77E081E00E94EE7CDFCF089552
:10C170000F931F93CF93DF93EC017093741260932E
:10C18000731240937A1281E090E00E9428B78C01EC
:10C190000E94887E109338120093371291E090939A
:10C1A0002D1290935B1210922C1210922B1210925F
:10C1B0005E1210925D1210925F1210925C1224EFC8
:10C1C00031E0309366122093651228EB3BE0309308
:10C1D00068122093671220E233E030936D122093AF
:10C1E0006C122CEA3DE030936F1220936E1228E01F
:10C1F00037E0309376122093751224E931E13093C1
:10C20000781220937712109262121092611210929B
:10C21000601210926912109270121092791210929C
:10C220002A12109264121092631210926B121092E2
:10C230006A121092721210927112988399839A83E3
:10C24000DF91CF911F910F9108951F920F920FB61A
:10C250000F9211240BB60F922F933F934F935F933E
:10C260006F937F938F939F93AF93BF93EF93FF93BE
:10C27000809134128F5F809334129091331289171A
:10C2800008F401C1109234128091321290E087308C
:10C29000910508F0F8C0FC018827ED55FE4F8F4F3F
:10C2A0000C948BB560E086E10E945D4680E480934B
:10C2B000331281E048C061E086E10E945D4688E07B
:10C2C0008093331236C060E086E10E945D46809123
:10C2D00030129091311297FF05C088E1809333129C
:10C2E00084E031C088E08093331283E02CC061E0A9
:10C2F00086E10E945D4688E18093331280912F127F
:10C300008F5F80932F12803150F010922F1285E0B2
:10C310001AC061E086E10E945D4688E0EDCF809121
:10C32000301290913112880F991F9093311280939F
:10C33000301282E008C060E086E10E945D4688E03D
:10C340008093331286E0809332129DC061E086E1D3
:10C350000E945D4680EC809333128091351290915B
:10C360003612909331128093301280913512909151
:10C37000361291FF1DC080912E128823B1F080915A
:10C3800035129091361222E09227909336128093C4
:10C390003512809135129091361280649093361246
:10C3A0008093351210922E1203C081E080932E12DA
:10C3B000809135129091361292FF0EC080912E120C
:10C3C000882339F0109236121092351210922E12E4
:10C3D00003C081E080932E12809135129091361225
:10C3E00084FF14C080912E12882369F08091351249
:10C3F0009091361220E18227909336128093351265
:10C4000010922E1203C081E080932E12809135127B
:10C410009091361287FF13C080912E12882361F00D
:10C4200080913512909136128058909336128093F5
:10C43000351210922E1203C081E080932E1280914B
:10C4400035129091361290FF14C080912E128823DD
:10C4500069F0809135129091361221E092279093E5
:10C4600036128093351210922E1203C081E0809311
:10C470002E12809135129091361290933112809342
:10C48000301210923212FF91EF91BF91AF919F91B4
:10C490008F917F916F915F914F913F912F910F906D
:10C4A0000BBE0F900FBE0F901F90189520E040E03C
:10C4B0006CCD65E4FBCF68E4F9CFCF93DF93FC014B
:10C4C0002381222321F0EC0161E4F0DF1B82DF9164
:10C4D000CF910895CF93DF93FC012381211105C0F3
:10C4E000EC0160E4E3DF81E08B83DF91CF9108957D
:10C4F000FC012581222311F060E5D8CF0895FC01CD
:10C500002481222311F06CE3D1CF0895FC01208512
:10C51000222331F02185222319F011866BE3C6CF47
:10C520000895FC012085222339F02185211104C0C2
:10C5300021E021876AE3BACF0895FC0126812223F6
:10C5400031F02781222319F0178269E3AFCF0895D4
:10C55000FC012681222339F02781211104C021E02A
:10C56000278368E3A3CF089567E3A0CF6AE49ECF53
:10C5700069E49CCF66E39ACF65E398CF6EE496CFEB
:10C5800064E394CF63E392CF62E390CF61E38ECF15
:10C5900060E38CCF6FE28ACF6DE288CFFC0112821C
:10C5A000138214821582168217821286089580E003
:10C5B00008950F931F93CF938C0168E776E187ED81
:10C5C00098E00E943F8BD8011896ED91FC91199745
:10C5D0006081718187ED98E00E94C937C1E0D80180
:10C5E0001A968C91C81710F563E776E187ED98E00D
:10C5F0000E943F8B6C2F87ED98E00E94863A60E79F
:10C6000076E187ED98E00E943F8BF8019085818567
:10C61000E92FF82FEC0FF11DEC0FF11D60817181F6
:10C6200087ED98E00E94C937CF5FD9CFCF911F9196
:10C630000F910895CF93DF93CDB7DEB7A0970FB6D4
:10C64000F894DEBF0FBECDBF80310CF080E028E64D
:10C6500036E13A83298321E636E13C832B8323E5C7
:10C6600036E13E832D8327E436E138872F832DE39F
:10C6700036E13A87298723E336E13C872B872FE28F
:10C6800036E13E872D8728E236E1388B2F872DE172
:10C6900036E13A8B298B20E136E13C8B2B8B25E070
:10C6A00036E13E8B2D8B29EF35E1388F2F8B27EE2E
:10C6B00035E13A8F298F26ED35E13C8F2B8F21ED27
:10C6C00035E13E8F2D8F24EC35E138A32F8FE82FF5
:10C6D000EE0FFF0BEC0FFD1F81819281A0960FB62C
:10C6E000F894DEBF0FBECDBFDF91CF910895AF921A
:10C6F000BF92CF92DF92EF92FF920F931F93CF934F
:10C70000DF938BE392E17EE1D72ED80ECC24C39445
:10C7100002E010E0C3E0D0E0E2E0BE2EEE24E394BD
:10C72000F12C8091D0119091D111DC01ED91FC910F
:10C730000480F581E02D1995892B09F4ADC0A090F6
:10C7400030018091D0119091D111DC01ED91FC91DB
:10C750000680F781E02D199596B3B39A2091840055
:10C7600030918500285A344E30938D0020938C00F0
:10C770002A2D2C7119F01092CD114BC093FB9927E3
:10C7800090F9E091CD11E11116C0992351F2803258
:10C7900041F6C092CD1180933B128091131390917A
:10C7A0001413892B09F0BDCFF0921413E0921313E8
:10C7B0001092CF11B6CF9111DECFE13041F4803429
:10C7C00009F0AFCFB092CD1180933C12E6CF91E04B
:10C7D0009E0F9093CD11F0E0E55CFD4E808390328A
:10C7E00009F09FCF1092CD11EBE3F2E12FEF3FEF75
:10C7F0008191281B3109DE12FBCF409159128091A3
:10C800005A1290E0982F8827840F911D2817390716
:10C8100029F0D0931413C093131383CF8091131373
:10C8200090911413019739F48091CF118F5F809309
:10C83000CF11843020F010931413009313138091C0
:10C84000CE118F5F8093CE119091CC11981708F57F
:10C85000C092151320E030E0F901E55CFD4E428105
:10C86000838190E0982F8827840F911DAC014F5E43
:10C8700052404B3D554028F4F901EE52FE4E918353
:10C8800080832E5F3F4F2C31310531F71092CE114E
:10C8900048CF1092151345CFDF91CF911F910F9183
:10C8A000FF90EF90DF90CF90BF90AF900895EF9200
:10C8B000FF920F931F93CF93DF931092C50D82E0E9
:10C8C0008093C60D68EE73E07093C80D6093C70D3A
:10C8D00040ED57E05093CA0D4093C90D2CED35E063
:10C8E0003093CC0D2093CB0D8FE08093CD0D109223
:10C8F000CE0D94E09093CF0D7093D10D6093D00D39
:10C900005093D30D4093D20D3093D50D2093D40D79
:10C910008093D60D1092D70D93E09093D80D70931D
:10C92000DA0D6093D90D5093DC0D4093DB0D3093FD
:10C93000DE0D2093DD0D8093DF0D1092E00D91E070
:10C940009093E10D7093E30D6093E20D5093E50D2C
:10C950004093E40D3093E70D2093E60D8093E80DAE
:10C960001092E90DEAEEFDE0A3EFBDE080E008EEF5
:10C9700013E060ED77E04CED55E031E022E095E02A
:10C98000980F908312830183748363835683458356
:10C99000ED01229791E03883219628831C928F5FC6
:10C9A0003A961A968C3059F71092620E9093630E55
:10C9B0001092640E9093650E8AE892E09093670E51
:10C9C0008093660E9093690E8093680E80E090E0ED
:10C9D0009C012B53324FF901EB55FF4F118210820E
:10C9E0003296108203968837910591F784E290E0A1
:10C9F00090936B0E80936A0E81E080936C0E2CE016
:10CA000030E030936E0E20936D0E94E090936F0E95
:10CA100021E230E03093710E2093700E27E02093D6
:10CA2000720E29E030E03093740E2093730E20E1F3
:10CA30002093750E7AE07093E20E2BE02093E30EC4
:10CA40002093E40E48EE53E05093E60E4093E50E3B
:10CA500020ED37E03093E80E2093E70E1092E90EB8
:10CA600064E66093EA0E6093EB0E5093ED0E4093F4
:10CA7000EC0E3093EF0E2093EE0E1092F00E5093CA
:10CA8000F20E4093F10E3093F40E2093F30E1092B9
:10CA9000F50E1092F60E8093F70E1092F90E10928A
:10CAA000F80E8093FA0E8093FB0EE8ECF0E0F09322
:10CAB000FD0EE093FC0EE0E2F3E0F093FF0EE09356
:10CAC000FE0E5093010F4093000F3093030F2093FD
:10CAD000020F8093040FE9E5F0E0F093060FE09376
:10CAE000050FE0E8F0E0F093080FE093070FEFEF99
:10CAF000F0E0F0930A0FE093090FF0930C0FE0932E
:10CB00000B0F80930D0F90930E0F10920F0F8093C9
:10CB1000100F9093110F1092120F1092130F809319
:10CB2000140F1092150F1092160F8093170F10927A
:10CB3000180F98E29093190F50931B0F40931A0F00
:10CB400050931D0F40931C0F30931F0F20931E0F07
:10CB50008093200F92E39093210FE2E0E093220F65
:10CB60008093230F6093240FE6E4E093250F9093C6
:10CB7000260F1092270F1092280F1092290F109253
:10CB80002A0F10922B0F10922C0FEAEFF0E0F09387
:10CB90002E0FE0932D0F10922F0F1092300F6093F5
:10CBA000310F61E46093320F1092330F9093340F82
:10CBB0001092350F9093360FEEE5F1E0F093380FB9
:10CBC000E093370F1092390FACEDB5E0B0933B0F07
:10CBD000A0933A0F00EA1FE010933D0F00933C0F23
:10CBE00030933F0F20933E0FC8E8D3E1D093410F1D
:10CBF000C093400F68EBE62E6BE0F62EF092430FE9
:10CC0000E092420FE0E4FFE1F093450FE093440F20
:10CC10001092460F1092470F1092480F69E16093EF
:10CC2000490F80934A0F80934B0F80934C0F509382
:10CC30004E0F40934D0F3093500F20934F0FF092B3
:10CC4000520FE092510F1093540F0093530FD09353
:10CC5000560FC093550F20E737E13093580F2093BC
:10CC6000570F1092590F10925A0F10925B0F90931A
:10CC70005C0F90935D0F90935E0F10925F0F109278
:10CC8000600F1092610F8093620F1092720F1092DA
:10CC9000630F99E09093640F1092650F1092660FE6
:10CCA0001092670F1092680FB0936A0FA093690FEC
:10CCB000F0936C0FE0936B0F80936D0F70936E0F7A
:10CCC00010926F0F21E030E03093710F2093700FBE
:10CCD00040E052EC61E070E04093730F5093740FAA
:10CCE0006093750F7093760F4093770F5093780F82
:10CCF0006093790F70937A0F40E056E960E070E03E
:10CD000040937B0F50937C0F60937D0F70937E0F49
:10CD100040937F0F5093800F6093810F7093820F29
:10CD20001092830F20E039E13093850F2093840F18
:10CD30001092860F9EE19093870F1092880F2EE13C
:10CD400030E030938A0F2093890F30938C0F20931B
:10CD50008B0F30938E0F20938D0F90938F0F9093A6
:10CD6000900F8093910F8093920F1092930F909356
:10CD7000940F8093950F9CE09093960F8093970F5C
:10CD800083E891EFA0E0B0E08093980F9093990F23
:10CD9000A0939A0FB0939B0F05EC1DE0C0E0D0E08C
:10CDA000CE010E9451BBF80161918F01861719F0E5
:10CDB000CE010E9463BB2196C73DF1E0DF0781F7FA
:10CDC000DF91CF911F910F91FF90EF9008954F92B7
:10CDD0005F926F927F928F929F92AF92BF92CF920B
:10CDE000DF92EF92FF92CF93DF93EB01A091391284
:10CDF000B0913A129D012F5F3F4F45E0429F2001C5
:10CE0000439F500C1124052C000C66087708812CD8
:10CE1000912C54012434E1E03E07ECF446E053E960
:10CE200061E0772775016401C40CD51CE61CF71C72
:10CE30004C0D5D1D6E1D7F1D6BBFFA014791569114
:10CE400065E0860E911CA11CB11CC417D50729F101
:10CE50002F5F3F4FDFCF25E0822E912CA12CB12CEC
:10CE600021E030E0A217B30708F44CC046E053E9D4
:10CE700061E07727480D591D6A1D7B1D6BBFFA01C4
:10CE800047915691F5E08F0E911CA11CB11CC4175F
:10CE9000D50719F02F5F3F4FE5CF46E053E961E03A
:10CEA0007727E5E0E29F6001E39FD00C11240D2C71
:10CEB000000CEE08FF084E5F5F4F6F4F7F4F4C0D29
:10CEC0005D1D6E1D7F1D6BBFFA0147915691FC01E0
:10CED0005383428346E053E961E077274C5F5F4F1D
:10CEE0006F4F7F4FC40ED51EE61EF71EEBBEF60138
:10CEF000C790FC01C48230933A1220933912C901C1
:10CF0000019606C010923A121092391280E090E019
:10CF1000DF91CF91FF90EF90DF90CF90BF90AF90D7
:10CF20009F908F907F906F905F904F900895809129
:10CF30000E02882311F0729801C0729A90910E022D
:10CF400081E0892780930E0208951092E00A4091B3
:10CF50002C0650912D0660E070E027EC37E68091BA
:10CF60001A0690911B060C94CD7B8091370688237E
:10CF700069F08091DF0A882349F081E08093DC0A20
:10CF8000809136060E94DF370C94C6450895CF93F2
:10CF9000DF93CDB7DEB765970FB6F894DEBF0FBE4F
:10CFA000CDBF81E08093E00A80918412882371F1E3
:10CFB00082E390E09A83898388E290E09C838B836C
:10CFC0008EE690E09E838D8384EF91E098878F8337
:10CFD0001D8A84E08F938DB79EB745970FB6F8945E
:10CFE0009EBF0FBE8DBFADB7BEB7119685E1FE01E6
:10CFF000319601900D928A95E1F78EEE99E00E94AC
:10D0000048920FB6F894DEBF0FBECDBF65960FB63F
:10D01000F894DEBF0FBECDBFDF91CF910895809110
:10D020007A12811112C08AE599E9A1E0BB27ABBF52
:10D03000FC016791769182E00E94EE7C81E0809312
:10D040005B1210925F1210925C12089561E08BE205
:10D050000E945D46EE9A25EA37E448E853E160E035
:10D0600070E080911A0690911B060E94CD7B9093F0
:10D07000A5118093A411089561E08BE20E945D46A2
:10D08000EE9A25EA37E448E853E160E070E08091E9
:10D090001A0690911B060E94CD7B9093A511809358
:10D0A000A411089581E20E948F8E21E0892B09F45A
:10D0B00020E0822F089580913206882309F44CC025
:10D0C0008091DF0A882309F447C081E08093DC0A5D
:10D0D000E9DF882329F0809135068823D9F106C03D
:10D0E00080913306811105C0809132060E94DF379E
:10D0F00031C090913206963069F5823081F08330EC
:10D10000D1F0813039F5E091480AF091490A7497DD
:10D110008081918145E550E060E070E017C0E091CA
:10D12000480AF091490A7497808191814AE550E05C
:10D1300060E070E00BC0E091480AF091490A7497F2
:10D14000808191814FE550E060E070E0885B954F11
:10D150000E94FC860C94C64508958091A7118823EF
:10D1600039F08091A611882319F081E08093D90AC3
:10D1700080911C0690911D06DC01ED91FC910688C2
:10D18000F789E02D19958091801281110E94974CAA
:10D1900080917F12882391F061E088E00E945D46D3
:10D1A00040917D1250917E1260E070E02FE937E4EB
:10D1B00080911A0690911B060E94CD7B8091A71149
:10D1C000882321F08091A611811101C074DF809124
:10D1D000A611882379F08091A711882359F08091B6
:10D1E0008312882339F0E0918112F09182128281BA
:10D1F0000E943C7DAACE8091DE0A811156C052DF8A
:10D200008823F1F081E08093DE0A80911C069091E2
:10D210001D06DC01ED91FC910288F389E02D199542
:10D220000E9409472DE237E448E95AE360E070E0E4
:10D2300080911A0690911B060E94CD7B86DE09C064
:10D240008091A611882329F18091A711882311F0DC
:10D2500013DF31CFFBDE80918312882339F0E09118
:10D260008112F091821282810E943C7D40917B125A
:10D2700050917C1214161506BCF4052E000C660B9A
:10D28000770B2DEA38E680911A0690911B060C94D4
:10D29000CD7B80918312882339F0E0918112F09147
:10D2A000821282810E943C7D58CF08950F931F9374
:10D2B00020917A12211135C04AE559E961E07727BA
:10D2C0009C01220F331F820F931F092E000CAA0B03
:10D2D000BB0B0296A11DB11D840F951FA61FB71F82
:10D2E000ABBFFC0187910AE519E921E033274091A2
:10D2F0005F1293E0499FA0011124052E000C660BDC
:10D30000770B4E5F5F4F6F4F7F4F040F151F261F28
:10D31000371F2BBFF8010791801718F01F910F914D
:10D320007ECE1F910F9108958F929F92AF92BF92E0
:10D33000CF92DF92EF92FF920F931F93CF93DF93E1
:10D34000EC01A62E80917A1281116BC04AE559E951
:10D3500061E077276E01CC0CDD1CCC0EDD1E0D2CA0
:10D36000000CEE08FF08D701C6010296A11DB11DF1
:10D37000480F591F6A1F7B1F6BBFFA0187914AE54F
:10D3800059E961E07727B0905F1293E0B99E800180
:10D390001124012E000C220B330B0E5F1F4F2F4F59
:10D3A0003F4F400F511F621F731F6BBFFA01479120
:10D3B000481708F036C080905D1290905E12009180
:10D3C000731210917412B401C8010E94667B882305
:10D3D00021F0B401C8010E947E7B8AE599E9A1E0B1
:10D3E000BB278C0D9D1DAE1DBF1DABBFFC01679102
:10D3F000769182E00E94EE7CB0925C12C0935F1244
:10D40000AA2079F010925B122FE038E642E350E058
:10D4100060E070E0C8010E94CD7B90935E12809323
:10D420005D12DF91CF911F910F91FF90EF90DF90F0
:10D43000CF90BF90AF909F908F900895CF92DF9242
:10D44000EF92FF9280917A12811134C0809179120B
:10D45000882381F161E08EE090E066DF60917712D1
:10D4600070917812CB01A0E0B0E0C0907512D0901E
:10D470007612E12CF12CC816D906EA06FB0664F4F4
:10D48000BC01CD016C197D098E099F090E94148B86
:10D49000C60ED71EE81EF91E2EE13AE6B701A60118
:10D4A00080917312909174120E94CD7B90937212AE
:10D4B00080937112FF90EF90DF90CF900895CF92FC
:10D4C000DF92EF92FF9280917A12811134C08091A5
:10D4D0007012882381F161E08DE090E025DF60919A
:10D4E0006E1270916F12CB01A0E0B0E0C0906C1290
:10D4F000D0906D12E12CF12CC816D906EA06FB0675
:10D5000064F4BC01CD016C197D098E099F090E944C
:10D51000148BC60ED71EE81EF91E2FE53AE6B7019A
:10D52000A60180917312909174120E94CD7B90930A
:10D530006B1280936A12FF90EF90DF90CF90089566
:10D54000CF92DF92EF92FF9280917A12811134C0D4
:10D5500080916912882381F161E08CE090E0E4DE43
:10D560006091671270916812CB01A0E0B0E0C090AA
:10D570006512D0906612E12CF12CC816D906EA0685
:10D58000FB0664F4BC01CD016C197D098E099F096D
:10D590000E94148BC60ED71EE81EF91E20EA3AE63A
:10D5A000B701A60180917312909174120E94CD7BF5
:10D5B0009093641280936312FF90EF90DF90CF906E
:10D5C000089580917A1281112CC080916212882373
:10D5D00041F080916912811104C081E08093691249
:10D5E000AFDF80916112882361F080917A128111FE
:10D5F00008C080917012811104C081E08093701284
:10D600005EDF80916012882361F080917A1281112F
:10D6100008C080917912811104C081E08093791251
:10D620000DCF08958091B5068093B406089580913A
:10D63000AD12882359F08091AB129091AC12DC01AD
:10D64000ED91FC910480F581E02D1994089580916D
:10D65000AD12882369F08091AB129091AC12DC017D
:10D66000ED91FC910190F081E02D6FEF73E0199442
:10D6700008958091AD12882389F08091AF1288239C
:10D6800021F080E090E0D3DF03C080E090E0DFDFB6
:10D690009091AF1281E089278093AF120895209175
:10D6A000AD12222369F0A091AB12B091AC12ED91B2
:10D6B000FC9111970190F081E02DBC01CD011994EE
:10D6C00008958091AA12882359F08091A812909110
:10D6D000A912DC01ED91FC910480F581E02D1994F3
:10D6E00008958091AA12882369F08091A8129091E0
:10D6F000A912DC01ED91FC910190F081E02D6FEF1A
:10D7000073E0199408958091AA12882389F080917A
:10D71000AE12882321F080E090E0D3DF03C080E0E8
:10D7200090E0DFDF9091AE1281E089278093AE1206
:10D7300008952091AA12222369F0A091A812B09115
:10D74000A912ED91FC9111970190F081E02DBC019F
:10D75000CD01199408952091A712222369F0A09178
:10D76000A512B091A612ED91FC9111970190F08154
:10D77000E02DBC01CD01199408952091A41222231B
:10D7800069F0A091A212B091A312ED91FC911197B2
:10D790000190F081E02DBC01CD01199408952091F4
:10D7A000A112222369F0A0919F12B091A012ED91D5
:10D7B000FC9111970190F081E02DBC01CD011994ED
:10D7C000089520919E12222369F0A0919C12B0919D
:10D7D0009D12ED91FC9111970190F081E02DBC011B
:10D7E000CD011994089520919B12222369F0A091F4
:10D7F0009912B0919A12ED91FC9111970190F081DC
:10D80000E02DBC01CD011994089520919812222396
:10D8100069F0A0919612B0919712ED91FC91119739
:10D820000190F081E02DBC01CD0119940895209163
:10D830009512222369F0A0919312B0919412ED9168
:10D84000FC9111970190F081E02DBC01CD0119945C
:10D8500008958091AE069091AF06DC01ED91FC91A8
:10D86000E25AFF4F0190F081E02D19948091AE06AD
:10D870009091AF06DC01ED91FC91E45AFF4F0190CD
:10D88000F081E02D19948091AE069091AF06DC01F5
:10D89000ED91FC91E65AFF4F0190F081E02D199433
:10D8A0008091040F81110DC08091290690912A0664
:10D8B000DC01ED91FC910190F081E02D60E070E0E1
:10D8C000199408958091040F81110DC0809129064B
:10D8D00090912A06DC01ED91FC910190F081E02D00
:10D8E0006FEF70E0199408958091B506882361F078
:10D8F0000E94C880029741F06CE377E18091B20604
:10D900009091B3060C94B08C08958091B40688234E
:10D9100041F06EE876E18091B2069091B3060C94E6
:10D92000B08C08958091B406882341F06EE776E1CB
:10D930008091B2069091B3060C94B08C0895CF9369
:10D94000DF932091B2123091B31228173907D1F02A
:10D950009093B3128093B2122091B406222391F0D7
:10D96000EC016DE077E18091B2069091B3060E94E0
:10D970003F8BBE018091B2069091B306DF91CF91AB
:10D980000C94C937DF91CF910895CF93DF93209105
:10D99000B0123091B11228173907D1F09093B1121B
:10D9A0008093B0122091B406222391F0EC0163EF32
:10D9B00076E18091B2069091B3060E943F8BBE0142
:10D9C0008091B2069091B306DF91CF910C94C93744
:10D9D000DF91CF9108952091A712222339F0BC0145
:10D9E00080919112909192120C94197A089520913D
:10D9F000A412222339F0BC0180918F1290919012D1
:10DA00000C94197A08952091A112222339F0BC01B7
:10DA100080918D1290918E120C94197A0895209114
:10DA20009E12222339F0BC0180918B1290918C12AE
:10DA30000C94197A089520919B12222339F0BC018D
:10DA40008091891290918A120C94197A08952091EC
:10DA50009812222339F0BC0180918712909188128C
:10DA60000C94197A089520919512222339F0BC0163
:10DA700080918512909186120C94197A0895CF9214
:10DA8000DF92EF92FF9220910002213019F4209151
:10DA9000100F04C02230C9F52091160F2223A9F1DE
:10DAA0009C01211584E0380710F02FEF33E0ADE042
:10DAB000B0E00E94BFBB2FEF33E040E050E00E9497
:10DAC00071BB69017A018FEFC81AD80AE80AF80A0F
:10DAD00080918A138C15C9F0C0928A138091B40684
:10DAE000882399F06CED76E18091B2069091B306AF
:10DAF0000E943F8B6C2D8091B2069091B306FF90EF
:10DB0000EF90DF90CF900C946F3AFF90EF90DF9002
:10DB1000CF900895CF92DF92EF92FF922091000272
:10DB2000213019F420910D0F04C02230C9F5209145
:10DB3000130F2223A9F19C01211584E0380710F06E
:10DB40002FEF33E0ADE0B0E00E94BFBB2FEF33E03A
:10DB500040E050E00E9471BB69017A018FEFC81A62
:10DB6000D80AE80AF80A809188138C15C9F0C09287
:10DB700088138091B406882399F065EC76E1809152
:10DB8000B2069091B3060E943F8B6C2D8091B20635
:10DB90009091B306FF90EF90DF90CF900C946F3A86
:10DBA000FF90EF90DF90CF90089581E08093AB06D7
:10DBB0000E9449428091B406882341F06BEA76E1E5
:10DBC0008091B2069091B3060C94B08C089583E0D6
:10DBD0008093AB060E945F418091B406882341F098
:10DBE00068EB76E18091B2069091B3060C94B08C0C
:10DBF000089582E08093AB060E945F418091B40655
:10DC0000882341F06EE976E18091B2069091B306E7
:10DC10000C94B08C08950C94E590809101028111D0
:10DC20000C94CB900C94E5900C94CB9084E60C94DF
:10DC3000DF4389E10C94DF4382E30C94DF438BE400
:10DC40000C94DF4380910002813011F482E001C026
:10DC500081E00C94824482E00C94824481E00C9434
:10DC600082440C94A10D682F8091B2069091B30666
:10DC70000E94863A6AE377E18091B2069091B306FA
:10DC80000C943F8B2091B2063091B306882319F093
:10DC900062EB77E002C066EB77E0C9010C943F8B42
:10DCA000F1DF8091B2069091B3060C949D8C209187
:10DCB000B2063091B306882319F06FE277E102C013
:10DCC00064E377E1C9010E943F8B8091B206909195
:10DCD000B3060C949D8C6DE277E18091B206909131
:10DCE000B3060C943F8B69E277E18091B206909184
:10DCF000B3060C943F8BCF93CDE267E277E180913E
:10DD0000B2069091B3060E943F8BC150B1F780914B
:10DD1000B2069091B3060E949D8C8091B2069091BC
:10DD2000B306DC01ED91FC910284F385E02DCF91E7
:10DD3000199408950895089508950895623039F06A
:10DD4000633041F0613041F4409362120895409392
:10DD500061120895409360120895623069F0633053
:10DD6000A1F06130D1F45093661240936512309364
:10DD7000681220936712089550936D1240936C12AD
:10DD800030936F1220936E12089550937612409341
:10DD9000751230937812209377120895FC018581D3
:10DDA0000895089508950895089520917A122111F3
:10DDB00002C0FC016283089520917A12211102C0F1
:10DDC000FC016483089520917A12211102C0FC01A4
:10DDD000638308950895089580917A12811102C095
:10DDE0000C94A25F0895089580E008950895089521
:10DDF000089508950895089580917A12811103C0BD
:10DE00008FE090E053CA089580917A12811120C06A
:10DE1000633091F028F4613049F0623051F0089598
:10DE2000653081F060F0663081F0089589E090E01F
:10DE30000EC08AE090E00BC08BE090E008C08CE060
:10DE400090E005C08DE090E002C08EE090E02ECA28
:10DE5000089520917A12211107C0FC018481882342
:10DE600019F082E090E022CA089520917A122111DF
:10DE700007C0FC018381882319F081E090E016CA75
:10DE8000089580917A12811103C08BE090E00ECA50
:10DE9000089580917A12811104C060E080E190E0E1
:10DEA00043CA089580917A12811104C060E08FE026
:10DEB00090E03ACA089580917A12811126C06330A9
:10DEC000A1F028F4613049F0623059F008956530CE
:10DED000A1F078F06630A9F0089560E089E090E064
:10DEE00013C060E08AE090E00FC060E08BE090E05B
:10DEF0000BC060E08CE090E007C060E08DE090E057
:10DF000003C060E08EE090E00FCA089580917A121D
:10DF1000811126C06330A1F028F4613049F06230ED
:10DF200059F008956530A1F078F06630A9F00895B1
:10DF300061E089E090E013C061E08AE090E00FC00A
:10DF400061E08BE090E00BC061E08CE090E007C006
:10DF500061E08DE090E003C061E08EE090E0E4C914
:10DF6000089520917A12211108C0FC018281882332
:10DF700021F061E088E090E0D7C9089520917A12FD
:10DF8000211108C0FC018481882321F061E082E036
:10DF900090E0CAC9089520917A12211108C0FC01AD
:10DFA0008381882321F061E081E090E0BDC908957C
:10DFB00080917A12811104C061E086E090E0B4C9DA
:10DFC000089580917A12811104C060E08BE090E0A6
:10DFD000ABC9089580917A12811104C061E087E095
:10DFE00090E0A2C9089580917A12811104C061E085
:10DFF00085E090E099C90895CF93DF93FC012581D6
:10E000002223A1F1EC0180917A1281112EC060913E
:10E0100063127091641280917312909174120E9435
:10E020007E7B1092691280917A1281110CC06091EE
:10E030006A1270916B1280917312909174120E9407
:10E040007E7B1092701280917A1281110CC06091C7
:10E0500071127091721280917312909174120E94D9
:10E060007E7B1092791210922A121D82DF91CF913D
:10E070000895CF93DF93FC01258121111EC0EC018F
:10E0800080917A12811117C080912A12811113C0D8
:10E0900021EE3AE648EB5BE060E070E080917312BD
:10E0A000909174120E94CD7B9093641280936312BE
:10E0B00081E080932A1281E08D83DF91CF910895D2
:10E0C00080917A12882329F06CED75E081E00C9440
:10E0D000EE7C84E090E0EAC880917A12882329F0EF
:10E0E00068EE73E081E00C94EE7C60E084E090E008
:10E0F0001BC980917A1281111BC080912D12882337
:10E10000B9F068EE73E081E00E94EE7C10922D126F
:10E1100022EA3FE548E95AE360E070E0809173123B
:10E12000909174120E94CD7B90932C1280932B12AD
:10E1300008956CED75E080E00C94EE7C24EF31E006
:10E14000DB010E9499B52FEF30E040E050E00E94E3
:10E1500071BBCA01B90164527A4F8F4F9F4F80E063
:10E160000C94EE7C80917A12882339F060ED77E090
:10E1700081E00E94EE7C0C94966061E083E090E088
:10E18000D3C820917A12211103C002960C94A96081
:10E19000089520917A12222389F06FE676E080E0DC
:10E1A0000E94EE7C29EA3FE542E350E060E070E047
:10E1B00080917312909174120C94CD7B02960C9402
:10E1C000A96080E00E94157D81E00E94157D80910C
:10E1D0007A12811103C082E00E94157D6CED75E01A
:10E1E00080E00E94EE7C6CED75E081E00E94EE7CA8
:10E1F00080917A1281110DC08AE599E9A1E0BB27CF
:10E20000ABBFFC016791769182E00E94EE7C0C949A
:10E210000F680895FC01808991899387828782899C
:10E2200093899587848784899589978786870895B8
:10E2300026E00C942A8E0895089508950895CF93AA
:10E24000DF93EC018091B512811109C06A8D7B8D3D
:10E25000CE0149960E94003B81E08093B51221E8EF
:10E260003FEF3B872A878FE790E09D878C871F864B
:10E270001E86398B288B9B8B8A8B1D8A1C8ADF918B
:10E28000CF9108950F931F93CF93DF93EC011F8AD3
:10E290001E8A8C01075E1F4F40E060E0C8010E94AB
:10E2A000427F40E064E0C8010E94427F0E948B4AA6
:10E2B0006C8F7D8F8E8F9F8FDF91CF911F910F91EC
:10E2C00008950F931F93CF93DF93EC018091B412C5
:10E2D000811112C00A8D1B8D6AEA70E0C8010E948C
:10E2E000127AD801ED91FC910284F385E02DC801EA
:10E2F000199581E08093B4124AE06EE0CE01499610
:10E300000E94427F21E83FEF3B872A878FE790E01A
:10E310009D878C871F861E86398B288B9B8B8A8BCB
:10E320001D8A1C8ADF91CF911F910F9108950F9341
:10E330001F93CF93DF93EC011F8A1E8A8C01075E27
:10E340001F4F40E060E0C8010E94067F40E064E0AB
:10E35000C8010E94067F0E948B4A6C8F7D8F8E8F32
:10E360009F8FDF91CF911F910F9108950F931F936E
:10E37000CF93DF93EC01E8A1F9A180819181A28183
:10E38000B3818E01075E1F4F81159649A105B10526
:10E3900009F450C040E056E960E070E08DE997E094
:10E3A00047DF64E170E080E090E00E94534AE8A11A
:10E3B000F9A180819181A281B38181152BE492071B
:10E3C000A105B105E9F068F4803629E09207A105BE
:10E3D000B105A1F080389542A105B105C1F442E034
:10E3E00012C0811521EE9207A105B10559F08115E2
:10E3F000924CA140B10559F445E005C041E003C08D
:10E4000043E001C046E06FE0C8010E94067F8DE94D
:10E4100097E00E94AA89E8A1F9A140815181628117
:10E4200073818DE997E004DF64E170E080E090E0C3
:10E430000E94534A4AE06EE0C8010E94067F41E014
:10E4400067E1C8010E94067F4AA168E1C8010E94F5
:10E45000067F4BA18FEF840F8E3108F04CE066E110
:10E46000C8010E94067F21E83FEF3B872A878FE79C
:10E4700090E09D878C871F861E86398B288B9B8B0F
:10E480008A8B1D8A1C8ADF91CF911F910F9108956D
:10E49000D0C7EF92FF920F931F93CF93DF93EC01BE
:10E4A0006623E1F0262F653608F024E60A891B89E9
:10E4B000E888F988D801AE19BF0930E00E9499B503
:10E4C00028EC30E040E050E00E949DBBE20EF31EDD
:10E4D000FB86EA86021B130B1D870C87DF91CF9109
:10E4E0001F910F91FF90EF900895CF93DF93CDB7D9
:10E4F000DEB7A2970FB6F894DEBF0FBECDBF803156
:10E500000CF080E121E138E13A83298329E038E108
:10E510003C832B8321E038E13E832D8329EF37E1D3
:10E5200038872F8321EF37E13A87298729EE37E1B2
:10E530003C872B8721EE37E13E872D8729ED37E198
:10E54000388B2F872BEC37E13A8B298B29EB37E17E
:10E550003C8B2B8B2CE937E13E8B2D8B27E837E169
:10E56000388F2F8B2DE737E13A8F298F23E737E15B
:10E570003C8F2B8F26E637E13E8F2D8F2AE537E142
:10E5800038A32F8F22E537E13AA329A3E82FEE0F16
:10E59000FF0BEC0FFD1F81819281A2960FB6F894BC
:10E5A000DEBF0FBECDBFDF91CF9108958F929F92B6
:10E5B000AF92BF92CF92DF92EF92FF920F931F9391
:10E5C000DC0118968D919C9119971E96CD90DC9048
:10E5D0001F976817790709F456C05896FC9058970A
:10E5E0004C01092E000CAA08BB088B01072E000C59
:10E5F000220B330B861797073CF41696ED91FC918E
:10E600001797FF2039F015C01496ED91FC911597DE
:10E61000FF2079F00D2C000CEE08FF08A9019801ED
:10E62000281939094A095B091C966D917C911D973F
:10E630000EC00D2C000CEE08FF08A9019801281946
:10E6400039094A095B091A966D917C911B97CB0198
:10E65000770FAA0BBB0BBC01CD016C197D098E098C
:10E660009F090E9455B58F01FF0F220B330BA901A3
:10E670009801281939094A095B090E9471BBC20E29
:10E68000D31EE41EF51EC6011F910F91FF90EF905F
:10E69000DF90CF90BF90AF909F908F900895EF92B2
:10E6A000FF920F931F93CF93DF938C01FC01778B25
:10E6B000668B7CDFEC01F8018281938188309105C3
:10E6C00031F57801F9E1EF0EF11CD7FF06C06AE0E1
:10E6D000C1388FEFD80754F001C068E02C2F9D2F70
:10E6E000C038D1052CF02FE790E002C021E89FEF61
:10E6F000422F592F57FF03C0519541955109C7012A
:10E700000E94C54FCD2B69F54FE766E027C00997FA
:10E7100041F57801E9E1EE0EF11CD7FF06C06EE08D
:10E72000C138FFEFDF0754F001C06CE02C2F9D2FA4
:10E73000C038D1052CF02FE790E002C021E89FEF10
:10E74000422F592F57FF03C0519541955109C701D9
:10E750000E94C54FCD2B29F44FE767E0C7010E9407
:10E76000C54F0E948B4AF801648F758F868F978FF3
:10E77000DF91CF911F910F91FF90EF900895CF936C
:10E78000DF93EC017F8B6E8B11DF9C018A819B8173
:10E7900088309105C1F437FF06C061E021388FEF62
:10E7A00038074CF001C060E0A901203831052CF099
:10E7B0004FE750E002C041E85FEF57FF1FC051959F
:10E7C000419551091BC00997E9F4922F832F2038F6
:10E7D000310514F09FE780E0492F582F41388FEF23
:10E7E000580714F441E85FEF57FF03C05195419576
:10E7F0005109632F661F6627661F6C5FCE0149961D
:10E800000E94427F0E948B4A6C8F7D8F8E8F9F8FDC
:10E81000DF91CF9108950F931F93CF93DF93EC0176
:10E820000E948B4A0C8D1D8D2E8D3F8DDC01CB01FE
:10E83000801B910BA20BB30B853F9140A105B10545
:10E8400040F06E897F89CE01DF91CF911F910F91AA
:10E8500096CFDF91CF911F910F910895CF93DF93C2
:10E86000EC017F8B6E8BA2DE9C018A819B818830BC
:10E870009105C1F437FF06C061E021388FEF3807FA
:10E880004CF001C060E0A901203831052CF04FE7C1
:10E8900050E002C041E85FEF57FF1FC0519541951E
:10E8A00051091BC00997E9F4922F832F20383105B5
:10E8B00014F09FE780E0492F582F41388FEF580719
:10E8C00014F441E85FEF57FF03C05195419551099A
:10E8D000632F661F6627661F6C5FCE0149960E94F4
:10E8E000067F0E948B4A6C8F7D8F8E8F9F8FDF916A
:10E8F000CF9108950F931F93CF93DF93EC010E9464
:10E900008B4A0C8D1D8D2E8D3F8DDC01CB01801B24
:10E91000910BA20BB30B853F9140A105B10540F0CF
:10E920006E897F89CE01DF91CF911F910F9196CF94
:10E93000DF91CF911F910F9108954F925F926F9247
:10E940007F928F929F92AF92BF92CF92DF92EF927F
:10E95000FF928AE18093DD092093DE0988E28093AB
:10E96000E00981E08093E3098093E4098EE08093DD
:10E97000E20980EC92E1A0E0B0E08093740990930A
:10E980007509A0937609B093770980EB94E0A0E035
:10E99000B0E08093780990937909A0937A09B093B5
:10E9A0007B09A4E1440F551F661F771FAA95D1F775
:10E9B00022E030E0B0EBCB2EB4E0DB2EE12CF12CEA
:10E9C00080E6482E89E0582E612C712C90E4892E27
:10E9D0009CE9992EA12CB12CC901880F991F880F91
:10E9E000991FFC01EC58F64F77FF05C04082518219
:10E9F0006282738204C0C082D182E282F382C90142
:10EA00000196880F991F880F991FFC01EC58F64F4B
:10EA1000283129F0C082D182E282F38204C0808250
:10EA20009182A282B382440F551F661F771F2E5F0B
:10EA30003F4F2A31310581F6FF90EF90DF90CF9064
:10EA4000BF90AF909F908F907F906F905F904F900E
:10EA50000C94A086CF93DF93EC0161E089E00E94E3
:10EA6000C74760E089E00E945D461092E1098CE2B0
:10EA700095E099838883DF91CF9108950895089553
:10EA8000FC01828193818830910529F410922B0139
:10EA900010922A010895099721F4109229011092E9
:10EAA00028010895FC01178A168A6CED75E08281B1
:10EAB0000C94B57DCF93DF93EC011F8A1E8A8A8167
:10EAC000CDD78B8D882331F08A810E94A57D9A8FC6
:10EAD000898F1B8EDF91CF910895DF92EF92FF9285
:10EAE0000F931F93CF93DF93EC018A81893008F451
:10EAF0009CD7DD8C6B8D7C8D098D1A8DEA80FB8017
:10EB000089E08E1508F466C00F30110538F0013623
:10EB10009DE6190728F000E61DE602C00FE010E0B0
:10EB20006F30710538F061368DE6780728F060E6C1
:10EB30007DE602C06FE070E080E090E00E942CBAB9
:10EB400020E030E04AE754E40E9404B620E030E0E0
:10EB50004CE852E40E948DBA9B01AC0160E070E089
:10EB60008AEF94E40E9404B60E946CB6FF2425E16B
:10EB70002E9DF0012F9DF00D1124E354FF4EDD205A
:10EB800071F023813481AB0177FF04C044275527FE
:10EB9000461B570B88279927841B950B0AC0258194
:10EBA0003681AB0177FF04C044275527461B570B1E
:10EBB000CA014FB7F89455E15E9DF0015F9DF00DDD
:10EBC0001124E354FF4E108B0787328B218B948BDB
:10EBD000838B4FBF9D8D6B8D7C8D8A819923E9F04E
:10EBE0008A3058F495E1899FF0011124E354FF4ED7
:10EBF000058116811695079502C00EEE12E041E0E0
:10EC00005BD761E070E080E090E00E94534A8A8127
:10EC10009CD708171907A8F31CC08A3058F495E14F
:10EC2000899FF0011124E354FF4E0381148116954E
:10EC3000079502C00AEC18E040E03ED761E070E0C2
:10EC400080E090E00E94534A8A817FD78017910725
:10EC5000A8F38A8103D7B8018A81DF91CF911F91F0
:10EC60000F91FF90EF90DF9080C7CF93DF93EC017F
:10EC70008A81893008F4D9D648EE53E05B874A8709
:10EC800020ED37E03D872C878CED95E09F878E87C0
:10EC9000598B488B3B8B2A8B9D8B8C8BDF91CF9133
:10ECA0000895CF93DF93EC017F8B6E8B88859985D8
:10ECB0006817790759F48A81D1D68B8D882319F189
:10ECC0008A8143D79A8F898F1B8E1DC0CE016EDC3F
:10ECD000EA81EA30B0F49C01C39714F022E330E0FB
:10ECE0002E3C8FEF380714F42EEC3FEF8FB7F894DB
:10ECF00095E1E99FF0011124E354FF4E318720870D
:10ED00008FBF81E08B8FDF91CF910895CF93DF93F9
:10ED1000EC018BA19CA1892B11F01CA21BA29B01D1
:10ED200077FF03C0319521953109B901CE013EDC51
:10ED300090932D0180932C019F8B8E8B0E948B4A88
:10ED40006F8F78A389A39AA3DF91CF9108950F9332
:10ED50001F93CF93DF938C01FC01778B668B26DCAE
:10ED6000EC01F8018281938188309105D1F4D7FFBD
:10ED700006C060E08AE00E945D4661E005C061E097
:10ED80008AE00E945D4660E086E00E945D46D7FF13
:10ED900003C0D195C195D109D0932B01C0932A010D
:10EDA0001BC00997C9F4D7FF06C060E08DE00E9440
:10EDB0005D4661E005C061E08DE00E945D4660E077
:10EDC0008BE00E945D46D7FF03C0D195C195D10964
:10EDD000D0932901C0932801DF91CF911F910F910A
:10EDE0000895CF93DF93EC018A81893008F41DD612
:10EDF0002EEC3FEF3B872A8782E390E09D878C874C
:10EE00001F861E86398B288B9B8B8A8B1D8A1C8ABA
:10EE10006EEE72E08A8195D66AEC78E08A818DD6B2
:10EE20008CED95E09A8F898F1B8EDF91CF9108959D
:10EE3000CF93DF93EC018BA19CA1892B11F01CA235
:10EE40001BA2CE01E7D910922D0110922C011F8A2E
:10EE50001E8A0E948B4A6F8F78A389A39AA3DF91A1
:10EE6000CF9108950F931F93CF93DF93FC0123A1BC
:10EE700034A1232B89F1EC010E948B4A0F8D18A13C
:10EE800029A13AA1DC01CB01801B910BA20BB30B92
:10EE90004097A105B10500F18BA19CA10197E1F478
:10EEA0006E897F89615071097F8B6E8BCE0116163A
:10EEB00017062CF0DF91CF911F910F91B9CF76DB20
:10EEC00090932D0180932C019F8B8E8B0E948B4AF7
:10EED0006F8F78A389A39AA3DF91CF911F910F9190
:10EEE0000895CF93DF93EC018D8D9E8D1B861A863E
:10EEF0009D878C871F861E86198A188A9B8B8A8B12
:10EF00001D8A1C8A61E08CE20E94C7478A819B812E
:10EF1000089721F410922D0110922C011CA21BA223
:10EF2000DF91CF910895CF93DF93EC0121E03FEF84
:10EF30003B872A878FEF90E09D878C871F861E86F0
:10EF4000398B288B9B8B8A8B1D8A1C8A61E08AE017
:10EF50000E94C74761E086E00E94C74761E08DE2FA
:10EF60000E94C74761E08DE00E94C74761E08BE0E7
:10EF70000E94C74761E08EE20E94C7478A819B8159
:10EF80008830910529F410922B0110922A0106C0B5
:10EF9000099721F41092290110922801DF91CF9155
:10EFA00008950F931F93CF93DF93EC010E948B4A38
:10EFB0000C8D1D8D2E8D3F8DDC01CB01801B910BA7
:10EFC000A20BB30B853F9140A105B10540F06E89BE
:10EFD0007F89CE01DF91CF911F910F9160CBDF919F
:10EFE000CF911F910F9108950F931F93CF93DF93AC
:10EFF0008C01FC01178A168AEC01699640E068E0F2
:10F00000CE010E94C54F4FE766E0CE010E94C54F7A
:10F0100040E06CE0CE010E94C54F4FE767E0CE01B3
:10F020000E94C54F0E948B4AF801648F758F868FAE
:10F03000978FDF91CF911F910F9108956F927F92DB
:10F040008F929F92AF92BF92CF92DF92EF92FF92F8
:10F050000F931F93CF93DF9380919A1390919B13FB
:10F06000DC01ED91FC910480F581E02D1995B12C26
:10F07000181619060CF0D5C0AA24A39480919A13EF
:10F0800090919B13DC01ED91FC910480F581E02DC2
:10F090001995892B09F4C5C0C091101381E08C0F1C
:10F0A0008093101380919A1390919B13DC01ED9142
:10F0B000FC910680F781E02D1995EC2FF0E0E053EC
:10F0C000FD4E80838A30D1F6E0901013F12C10921F
:10F0D000B70D1092B60D1092B20D1092B30D1092A2
:10F0E000B40D1092B50D1092B10D1092B00D10929A
:10F0F000AF0D80EDC82E82E1D82E00E010E0D0E008
:10F10000C0E00E151F050CF06FC0F60191916F0164
:10F110009D3009F466C09C37A1F19A3009F055C0C2
:10F12000CC2359F16C2E712CC30101970E945C3ED7
:10F130007093B70D6093B60D0E948B4A6093C8110F
:10F140007093C9118093CA119093CB118091B6121C
:10F15000882309F462C08090B60D9090B70DB80175
:10F160006619770980ED92E10E94C65388169906C8
:10F1700009F453C01092CF1252C01092CF12D0E0B7
:10F1800030C08C2F90E0FC01E654F24F1082D13059
:10F1900099F068F0D230B1F40E945C3E6093B20DF9
:10F1A0007093B30D8093B40D9093B50D0BC00E9476
:10F1B0005C3E6093AF0D06C00E945C3E7093B10D43
:10F1C0006093B00DDF5FC0E00CC00F3311053CF45D
:10F1D000EC2FF0E0E654F24F9083CF5F02C0109224
:10F1E000CF120F5F1F4F8DCF8091CF1281110EC0B4
:10F1F0008091AC0D9091AD0D01969093AD0D8093E3
:10F20000AC0D60E087E80E94359702C0BB24B39440
:10F210001092D0121092101331CFA092CF12D1E0E1
:10F22000E0CF8B2DDF91CF911F910F91FF90EF9049
:10F23000DF90CF90BF90AF909F908F907F906F9016
:10F240000895CF931092AE0D1092AB0D1092AD0DAC
:10F250001092AC0D61E089E30E945D460E94695303
:10F2600080919A1390919B13DC01ED91FC910480A5
:10F27000F581E02D1995892B61F080919A13909179
:10F280009B13DC01ED91FC910680F781E02D19952F
:10F29000E7CF0E94B19780919A1390919B13DC0164
:10F2A000ED91FC910284F385E02D19951092C71120
:10F2B0000E948B4A6093C8117093C9118093CA1140
:10F2C0009093CB11C1E0BADE81110E94C5300E943B
:10F2D000A9531CD78091AC0D9091AD0D0A9724F4E1
:10F2E0008091C711882331F060E08AE80E94359749
:10F2F000C093AE0D8091AE0D882329F38091AB0DA4
:10F30000882341F047ED51E060E070E085EC9DE03E
:10F310000E9441BB60E089E30E945D4660E08AE3B1
:10F32000CF910C945D46EF92FF920F931F93CF9372
:10F33000DF9300D000D0CDB7DEB76CEF75E0CE0123
:10F3400001960E94008B0D811E81F02EEE24E39425
:10F3500080919A1390919B13DC01ED91FC910480B4
:10F36000F581E02D1995892B21F180919A139091C7
:10F370009B13DC01ED91FC910680F781E02D19953E
:10F380008F3439F4E092CE128093C312E092C2120D
:10F39000DFCF9091CE129923D9F2E091C21291E081
:10F3A0009E0F9093C212F0E0ED53FD4E80839F15A7
:10F3B00078F28091C2128F1510F4F12C21C04BE02D
:10F3C00050E067EB72E1CE0101960E94BC3DA3ECD8
:10F3D000B2E1ECEFF5E0FF24F3941127CF018C5F4D
:10F3E00095408017910734F49D9181919817B1F35E
:10F3F000F12CF4CF1092C3121092CE121092C212BE
:10F40000CE0101960E94D08A8F2D26960FB6F894D1
:10F41000DEBF0FBECDBFDF91CF911F910F91FF9047
:10F42000EF900895DC01ED91FC910190F081E02DC9
:10F430001994CF93DF93EC017F8B6E8BB7D8BC010F
:10F440008A81DF91CF9191C3482F50E095E1899F48
:10F45000F0011124E354FF4E218132818085918592
:10F46000280F391F838194818217930728F08581A3
:10F47000968128173907E8F485E1849FF001859F7C
:10F48000F00D1124E354FF4E85819681281739072A
:10F4900028F52581368185E1849FF001859FF00D57
:10F4A0001124E354FF4E8285823019F411861086B0
:10F4B000128685E1849FF001859FF00D1124E354AD
:10F4C000FF4E328321838091840090918500280F24
:10F4D000391F309389002093880008958381948197
:10F4E00082179307C0F623813481D5CF8091EE0A2D
:10F4F000811157C0E0919D10F0919E1085819681F9
:10F5000090939A108093991010929C1010929B10D7
:10F51000E091A710F091A810858196819093A41096
:10F520008093A3101092A6101092A510E091B11034
:10F53000F091B210858196819093AE108093AD10BA
:10F540001092B0101092AF10E091BB10F091BC106F
:10F55000858196819093B8108093B7101092BA105D
:10F560001092B91082E190E09093911080939010E6
:10F5700081E0809396108093A0108093AA108093CE
:10F58000B4108093921080E090E021E0FC01E45CF4
:10F59000FF4E2183079684359105C1F781E0809362
:10F5A000EE0A08951092B61008951092AC100895C6
:10F5B0006CE20C9456624F925F926F927F928F92A0
:10F5C0009F92AF92BF92CF92DF92EF92FF920F93F2
:10F5D0001F93CF93DF936C01A4ECCA1AADEFDA0A44
:10F5E000D601ED91FC917E970CF05DC0FC01E858CE
:10F5F000FF4F812C912CA191B191AB2B21F42115BE
:10F60000310549F450C0BFEF8B1A9B0AAEE18A1650
:10F61000910489F748C0EC015401AA0CBB1CAA0C48
:10F62000BB1CAC0EBD1EF501EC54FF4F4083518353
:10F63000628373837401EE0CFF1CEC0EFD1EF70158
:10F64000E858FF4F31832083EC54FF4F1183008330
:10F65000BE01680D791DFB01EC55FE4F81E08083F2
:10F660000E948B4AF5016083718382839383C65C19
:10F67000DD4F88819981F701E250FE4F91838083AD
:10F68000D6012D913C9111972F5F3F4F2D933C93C5
:10F690009C012F5F3F4F1216130614F021E030E05B
:10F6A0003983288302C08FEF9FEFDF91CF911F91A5
:10F6B0000F91FF90EF90DF90CF90BF90AF909F9011
:10F6C0008F907F906F905F904F900895DC01A250D3
:10F6D000BE4F20E030E04D915D914617570739F459
:10F6E000280F391FF901EC55FE4F808108952F5FD7
:10F6F0003F4F2E31310579F780E00895CF93DF93A6
:10F70000EC01C45CDD4FA881B981109709F442C0B7
:10F71000FC01E250FE4F20E030E04191519146174C
:10F72000570799F5A901440F551F480F591FFA01B2
:10F73000E858FF4F60817181672B61F1118210825F
:10F74000FC01E20FF31FEC55FE4F1082FA01EE535D
:10F75000FE4F11821082235D3F4F220F331F220F75
:10F76000331FFC01E20FF31F1082118212821382F9
:10F77000FA01E859FE4F11821082EA56FF4F1182BA
:10F7800010821197B983A88305C02F5F3F4F2E3198
:10F79000310519F6DF91CF9108950F931F9301E082
:10F7A00010E009DF1F910F9108950F931F9300E060
:10F7B00010E001DF1F910F9108952F923F924F9219
:10F7C0005F926F927F928F929F92AF92BF92CF92F1
:10F7D000DF92EF92FF920F931F93CF93DF9300D0AE
:10F7E00000D0CDB7DEB78C010E948B4A98012E5312
:10F7F0003E4F3C832B831E830D83D801AC55BE4FF7
:10F80000BA83A9831801B2E02B1ABEEF3B0AF901B3
:10F81000AA24A394B12C32E0832E912C1182108261
:10F820009F012A543140D9012D913C91232B09F499
:10F830004DC0AD81BE812D913D914D915C9113974D
:10F840007D01B4EBEB0EF11CD701CD90DD90ED9076
:10F85000FC902B013C01421A530A640A750A4C14AD
:10F860005D046E047F0490F1C20ED31EE41EF51EEB
:10F87000AD81BE81CD92DD92ED92FC921397A9816C
:10F88000BA812C91222311F19F0126593109D90106
:10F890002D913C912115310519F4B182A08216C039
:10F8A0007F01BAE5EB1AF108D7014D915C911197F0
:10F8B000421753075CF4B182A0824F5F5F4F4D93B4
:10F8C0005C934217530714F09182808232962D8107
:10F8D0003E812C5F3F4F3E832D83A981BA811196D3
:10F8E000BA83A983E215F30509F098CFEB81FC8177
:10F8F00081919191FC83EB838130910599F002977E
:10F90000C9F4EB81FC81EC54F1400190F081E02DD1
:10F910001995AB81BC81DA966D917C91DB97C8011A
:10F92000EDDE08C0EB81FC81EC54F1400190F081E8
:10F93000E02D19952B813C8122153305B9F62696C9
:10F940000FB6F894DEBF0FBECDBFDF91CF911F91F0
:10F950000F91FF90EF90DF90CF90BF90AF909F906E
:10F960008F907F906F905F904F903F902F90089571
:10F970006E3E22E0720738F06B3C98E0790728F081
:10F980006AEC78E002C06EEE72E0660F771F9FB7F8
:10F99000F89425E1829FF0011124E354FF4E748313
:10F9A00063839FBF08956E3E22E0720738F06B3C80
:10F9B00098E0790728F06AEC78E002C06EEE72E019
:10F9C000660F771F9FB7F89425E1829FF0011124FD
:10F9D000E354FF4E768365839FBF0895660F771FBC
:10F9E000282F30E095E1899FF0011124E354FF4E68
:10F9F000858196816817790718F46581768107C03B
:10FA0000838194818617970710F4638174818FB77F
:10FA1000F89495E1929FF001939FF00D1124E35427
:10FA2000FF4E728361838FBF0895982F8FB7F8942C
:10FA300025E1929FF0011124E354FF4E21E027833A
:10FA40008FBF41B121E030E0B90102C0660F771FDE
:10FA50009A95E2F7CB01842B81B908958A3058F446
:10FA60009FB7F89425E1829FF0011124E354FF4EE3
:10FA7000118610869FBF08951F93CF93DF9325E1D2
:10FA8000829FC0011124EC01C354DF4E8A8581118D
:10FA90000FC01FB7F89481E08A8789899A899A8371
:10FAA00089830E948B4A6B877C878D879E871FBFC7
:10FAB000DF91CF911F910895CF93DF938A30D0F5D6
:10FAC0006233710538F061369DE6790728F060E60B
:10FAD0007DE602C062E370E0D42FC82F80E090E0A2
:10FAE0000E942CBA20E030E04AE754E40E9404B6B9
:10FAF00020E030E04CE852E40E948DBA9B01AC015A
:10FB000060E070E08AEF94E40E9404B60E946CB654
:10FB10009B01DD2321F022273327261B370B8FB7CC
:10FB2000F89495E1C99FF0011124E354FF4E318709
:10FB300020878FBFDF91CF9108958A3008F418CFC6
:10FB400008958A3008F42FCF08958A3058F495E14B
:10FB5000899FF0011124E354FF4E81819281969593
:10FB60008795089580E090E008958A3008F436CFB4
:10FB700008951F920F920FB60F9211240BB60F9299
:10FB80000F931F932F933F934F935F936F937F93A5
:10FB90008F939F93AF93BF93CF93EF93FF938091F6
:10FBA0006113893048F01092611380916C118823A1
:10FBB00099F0809165110DC0E0916113E15025E14C
:10FBC000E29FF0011124E354FF4E8781882321F046
:10FBD000808192B1892782B9E091611385E1E89F24
:10FBE000F0011124E354FF4E8781882321F08081A6
:10FBF00092B1892B82B9E0916113C5E1CE9FF001EA
:10FC00001124E354FF4E80859185892B09F04DC066
:10FC1000E0916113CE9FF0011124E354FF4E8285E1
:10FC2000813009F060C00E948B4AE0916113CE9F41
:10FC3000F0011124E354FF4E038514852585368594
:10FC4000E0916113CE9FF0011124E354FF4E07842D
:10FC5000F089E02DAB01BC01401B510B620B730B13
:10FC6000CF01A0E0B0E084179507A607B707D8F545
:10FC7000E0916113A0916113CA9FD0011124A35494
:10FC8000BF4E53968D919C915497CE9FF0011124B5
:10FC9000E354FF4E91878087E0916113CE9FF0017E
:10FCA0001124E354FF4E82E0828780916113CCDB04
:10FCB000809161138F5F80936113FF91EF91CF91DA
:10FCC000BF91AF919F918F917F916F915F914F9174
:10FCD0003F912F911F910F910F900BBE0F900FBE70
:10FCE0000F901F901895E09161138091840090917E
:10FCF000850025E1E29FF0011124E354FF4E2181AC
:10FD00003281820F931F9093890080938800D0CF17
:10FD10001F93CF93DF9380916013811173C0109272
:10FD200061139FB7F89485E128EB3BE04CED55E07B
:10FD300064E971E1A1E0B0E0E0916113E93008F01D
:10FD400052C0E09161138E9FF0011124E354FF4EE5
:10FD500032832183E09161138E9FF0011124E354DB
:10FD6000FF4E56834583E09161138E9FF00111246D
:10FD7000E354FF4E74836383E0916113F091611348
:10FD8000ED0101C0CC0FFA95EAF78E9FF001112426
:10FD9000E354FF4EC083E09161138E9FF001112464
:10FDA000E354FF4E1782E09161138E9FF0011124FE
:10FDB000E354FF4E11861086E09161138E9FF0018F
:10FDC0001124E354FF4E1286E09161138E9FF001DF
:10FDD0001124E354FF4E148A138AE0916113EF5FFC
:10FDE000E0936113A9CF9FBF8FB7F89420EA3FE05B
:10FDF0003093671120936611109265118FBF81E0D7
:10FE000080936013DF91CF911F9108950F931F93FB
:10FE1000CF93DF938C01C62FD42FDC0111968D91E7
:10FE20009C911297DC01ED91FC910190F081E02D05
:10FE3000D8016C911995F80181819281DC01ED91D5
:10FE4000FC910190F081E02D6C2F1995F8018181D2
:10FE50009281DC01ED91FC910190F081E02D6D2FFC
:10FE60001995F80180816C2F70E0680F711D6D0F7E
:10FE7000711D6F77772781819281DF91CF911F91DB
:10FE80000F91D0CA0F931F93CF93DF938C01C62F8E
:10FE9000D42FDC0111968D919C911297DC01ED918C
:10FEA000FC910190F081E02DD8016C911995F80139
:10FEB00081819281DC01ED91FC910190F081E02D36
:10FEC0006C2F1995F80181819281DC01ED91FC91F3
:10FED0000190F081E02D6D2F1995F80180816C2F34
:10FEE00070E0680F711D6D0F711D6F77772781812D
:10FEF0009281DF91CF911F910F9194CA4F925F929F
:10FF00006F927F92AF92BF92CF92DF92EF92FF9269
:10FF10001F93CF93DF93DD24D39445E0C42E52E0AA
:10FF2000A52EB12CC3E0D0E0EE24E394F12C809117
:10FF3000441390914513DC01ED91FC910480F5810F
:10FF4000E02D1995892B09F4BEC0109130018091E4
:10FF5000441390914513DC01ED91FC910680F781EB
:10FF6000E02D199596B3B39A2091840030918500C5
:10FF70002059384E30938D0020938C00212F2C7106
:10FF800039F010925F13D0934313C0934213CFCF35
:10FF900093FB992790F9E0915F13E11116C0992323
:10FFA00031F28F3021F6D0925F1380934613809107
:10FFB000421390914313892B09F0B9CFF092431368
:10FFC000E092421310924113B2CF9111DACF91E037
:10FFD0009E0F90935F13F0E0EA5BFC4E80839931B3
:10FFE00009F0A5CF81116CC080915D1382FF05C01F
:10FFF000D0934313C093421363C083FDF9CF809124
:020000021000EC
:10000000421390914313019739F4809141138F5F0C
:1000100080934113843020F0B0924313A092421396
:10002000809140138F5F8093401390913F139817F6
:1000300008F044C0D0923E13AEE1B3E1E7E4F3E14F
:1000400040E050E0BA0110E0CF01FC011B3098F411
:1000500001964080512C612C712C012E04C0440C5F
:10006000551C661C771C0A94D2F744295529662929
:100070007729185FEACF9A013770205E3340C29E1D
:10008000C001C39E900D112497FD079623E095951E
:1000900087952A95E1F784529A4F8D939D931B5033
:1000A0003BE076956795579547953A95D1F783E16B
:1000B000AE33B80749F61092401302C010923E13B7
:1000C00010925F1334CFDF91CF911F91FF90EF908B
:1000D000DF90CF90BF90AF907F906F905F904F90E8
:1000E00008958091F40A833031F480911C1390912B
:1000F0001D130C94776308958091F40A823029F4DB
:1001000080911A1390911B13F9CE0895F5DFE9CF72
:10011000109296101092A0101092AA101092B41083
:100120001092921080E090E0FC01E45CFF4E11829E
:10013000079684359105C1F708958091F40A8230BD
:1001400039F0833049F0813049F48091171301C0B0
:1001500080E18093F00A04C08EE0FBCF1092F00A99
:100160008091F00A08958091F40A823039F083304A
:1001700049F0813059F4809116130895BDDF8091C4
:100180003E130895AEDF80911513089580E0089521
:100190008091F40A823049F0833069F0813089F42B
:1001A00080911113909112130895A6DF809142134C
:1001B00090914313089595DF809113139091141338
:1001C000089581E090E008958F929F92AF92BF9240
:1001D000CF92DF92EF92FF921F93CF93DF93EC01C8
:1001E00011E08E819F81892B09F410E02C813D81E3
:1001F000E885F985C580D680878190E0A601480F03
:10020000591F2417350764F180850D2C000CEE086A
:10021000FF08A901330F660B770B0380F481E02DF3
:100220009A01AB012C193D094E095F09882329F079
:10023000A1E0BFEF0E9499BB04C0AFEFB0E00E9405
:100240008DBB4F01FF0FAA08BB08A50194012C1913
:100250003D094E095F090E9471BB3F832E834BC04D
:10026000A601481B590B421753070CF43FC0808569
:100270000D2C000CEE08FF08A901330F660B770B5D
:1002800081809280092C000CAA08BB089A01AB015E
:10029000281939094A095B09882399F0A1E0BFEFC1
:1002A0000E9499BBA7019601281939094A095B09DF
:1002B0000E9471BBDA01C90181509F4FAF4FBF4F00
:1002C00012C0AFEFB0E00E948DBBA70196012819C4
:1002D00039094A095B090E9471BBDA01C9018F5FC4
:1002E0009109A109B1099F838E8305C01F821E82D7
:1002F000111101C019828E819F81009789F08F3F73
:10030000910519F014F08FEF90E081305FEF9507C1
:1003100014F481E09FEF9F838E8381E018271A8376
:10032000DF91CF911F91FF90EF90DF90CF90BF9022
:10033000AF909F908F90089560E089E30E945D46A2
:1003400060E08AE30E945D4660E085E30E945D46CE
:1003500060E085E00E945D4660E084E00E945D46CA
:1003600060E087E00E945D4672980895CF93C09147
:1003700013026C2F89E30E945D4681E0C8276C2F31
:100380008AE30E945D46C0931302CF910895CF93F4
:10039000DF93C09112026C2F89E30E945D46D1E089
:1003A000DC276D2F8AE30E945D466C2F85E30E9457
:1003B0005D466D2F85E00E945D466D2F84E00E94B2
:1003C0005D466C2F87E00E945D46CC2311F0729849
:1003D00001C0729A9091120281E0892780931202E3
:1003E000DF91CF910895CF93DF938091771381119F
:1003F0000DC0109276131092751381E090E09093E7
:100400007413809373138093771336C080917513A0
:1004100090917613863191057CF18F38910534F4F3
:100420008091731390917413019609C08D3521E06A
:10043000920754F4809173139091741302969093E1
:1004400074138093731318C0863222E0920734F439
:1004500080917313909174130496F1CF883E93406A
:100460003CF480917313909174138A5B9F4FE7CF94
:1004700010927413109273138ADFC0917513D09188
:100480007613C93E83E0D80754F01092771354DFF7
:100490002AE632E848EE53E060E070E007C023EF60
:1004A00031E8AE010D2E000C660B770B8BE69BE05E
:1004B00074D99093721380937113809173139091F8
:1004C00074138C0F9D1F9093761380937513DF9197
:1004D000CF910895CF93DF938091B706882319F0C9
:1004E000DF91CF9180CFC0917113D0917213BE0173
:1004F0008BE69BE0EBD8882321F0BE018BE69BE0E6
:10050000FDD8DF91CF9118CFCF93C0916E136C2F90
:1005100070E088E00E94034889E180936D13909118
:100520001102992311F0CD5F01C0C350C0936E1327
:1005300080916E13873970F0992321F08FEF8093AB
:100540006E1308C08D3D30F086E980936E1388E706
:1005500080936D1380916E138F3F19F410921102E6
:1005600005C08A3118F481E08093110240916D1327
:1005700050E060E070E024E832E88BE69BE00DD9C3
:1005800090937B1380937A13CF910895CF92DF924B
:10059000EF92FF92CF93DF93EC019C01AFEFB0E0BD
:1005A0000E94BFBBCC24CA9423E0D22EE12CF12CB4
:1005B000A70196010E9471BBB90188E00E9403481F
:1005C0009E01A4E6B0E00E94BFBBA70196010E9475
:1005D00071BB80918F0F821320938F0FDF91CF918A
:1005E000FF90EF90DF90CF900895CF93DF93C0916D
:1005F0007A13D0917B13BE018BE69BE067D88823EA
:1006000021F0BE018BE69BE079D860E088E00E9493
:100610005D468091B4068823D1F080917C138823B5
:1006200019F063EF78E10DC080917913882319F0F8
:100630006AED78E106C080912712811108C06BEC49
:1006400078E18091B2069091B3060E94B08C10922E
:100650007C1310927913DF91CF91089561E088E0C7
:100660000E945D468091B406882361F080917C13DE
:10067000811108C06DEB78E18091B2069091B306CC
:100680000C94B08C089580917C13811110C0ADDF63
:1006900081E080937C138091B406882341F062E26C
:1006A00079E18091B2069091B3060E94B08C80915E
:1006B0006C13882329F060E088E00E945D4601C049
:1006C000CDDF90916C1381E0892780936C13882390
:1006D00029F040918B0F50918C0F04C040918D0FE9
:1006E00050918E0F60E070E023E433E88BE69BE0EE
:1006F00054D890937B1380937A130895CF9380916D
:100700006A1381110FC081E080936A138091B4064F
:10071000882341F06BE878E18091B2069091B306AE
:100720000E94B08CC09169136C2F85E00E945D46D9
:100730004091940F50E060E070E02EE733E88BE6E4
:100740009BE02BD8909368138093671381E06C2F04
:10075000682760936913CF910895CF93DF93C09179
:100760006F13D0917013BE018BE69BE00E94667BF5
:10077000882361F0BE018BE69BE00E947E7B109295
:10078000701310926F13DF91CF91D6CDDF91CF917F
:10079000089560916F13709170138BE69BE00E9437
:1007A000667B81112EC060E089E30E945D4660E0B7
:1007B0008AE30E945D4660E085E30E945D4660E05A
:1007C00085E00E945D4660E084E00E945D4660E056
:1007D00087E00E945D4672988091910F882319F0FE
:1007E00027EC31E802C026EB31E842E350E060E05C
:1007F00070E08BE69BE00E94D57B90937013809312
:100800006F13089560E08AE30C945D4661E08AE32B
:100810000C945D460F931F93CF93DF938C01C1E03F
:10082000D0E00C171D079CF0F1DF64E670E080E07B
:1008300090E00E94534AE6DFC017D10734F46AE51E
:1008400070E080E090E00E94534A2196EACFDF9169
:10085000CF911F910F91089583E090E0DBCF82E06C
:1008600090E0D8CF81E090E0D5CF60E089E30C94B0
:100870005D4661E089E30C945D460F931F93CF932F
:10088000DF938C01C1E0D0E00C171D079CF0F1DF75
:1008900064E670E080E090E00E94534AE6DFC01713
:1008A000D10734F46AE570E080E090E00E94534A9A
:1008B0002196EACFDF91CF911F910F91089583E0A8
:1008C00090E0DBCF82E090E0D8CF81E090E0D5CF20
:1008D00060918F0F70E088E00E9403488091B40619
:1008E000882341F06CE079E18091B2069091B306E3
:1008F0000C94B08C089510926B138091A006811116
:1009000004C060E084E00E945D468091B4068823C4
:1009100041F06AEA78E18091B2069091B3060C94B6
:10092000B08C089581E080936B138091A0068111B3
:1009300006C06091621370E084E00E9403488091D9
:10094000B406882341F068E978E18091B20690917D
:10095000B3060C94B08C08951092A00680916B138E
:10096000811104C060E084E00C945D4660916213E4
:1009700070E084E00C940348CF93DF9360E085E05F
:100980000E945D4680916A1381110BC08091AE0672
:100990009091AF06DC01ED91FC9102ACF3ADE02D3E
:1009A0001995C0916713D0916813BE018BE69BE047
:1009B0000E94667B882329F0BE018BE69BE00E94A3
:1009C0007E7B8091B406882371F020916A13809118
:1009D000B2069091B306222319F06FE778E102C0C6
:1009E00063E778E1BDD710926A13DF91CF91089544
:1009F00061E085E00E945D468091AE069091AF0671
:100A0000DC01ED91FC9102ACF3ADE02D19958091E4
:100A1000B406882339F068E678E18091B2069091B7
:100A2000B3069EC7089560E085E30E945D4680910D
:100A3000AE069091AF06DC01ED91FC9106A8F7A9F6
:100A4000E02D19958091B406882339F06CE578E1A2
:100A50008091B2069091B30683C7089561E085E363
:100A60000E945D468091AE069091AF06DC01ED914B
:100A7000FC9106A8F7A9E02D19958091B40688236A
:100A800039F061E578E18091B2069091B30668C7CC
:100A900008958F929F92AF92BF92CF92DF92EF9282
:100AA000FF9285E40E940F4ABC01990F880B990BB5
:100AB0000E942EBA20E030E040E85AE30E948DBA4E
:100AC00020E030E040EA50E40E948DBA6B017C01E6
:100AD00080911002882351F0C0926313D092641366
:100AE000E0926513F09266131092100226E636E645
:100AF00046E65FE360916313709164138091651320
:100B0000909166130E948DBA4B015C0120ED3CEC84
:100B10004CEC5DE3C701B6010E948DBA9B01AC01AC
:100B2000C501B4010E94A0B5609363137093641370
:100B300080936513909366132DE33CE248E450E400
:100B40000E948DBA2AE939E949E95EE30E94A0B51D
:100B5000FF90EF90DF90CF90BF90AF909F908F90DD
:100B6000089580910F02882351F093DF20E030E058
:100B700040E050E40E9428BA87FF38C0089589DF1A
:100B800020E030E04AE754E40E948DBA0E9471B63A
:100B90002091840F3091850F4091B706621773073B
:100BA00010F4442349F1442309F442C072DF20E0E9
:100BB00030E04AE754E40E948DBA0E9471B6209159
:100BC000840F3091850F6217730790F11092B7066A
:100BD00081E08093B6068091B406882349F169E1EB
:100BE00078E18091B2069091B306BAC610920F02D6
:100BF00081E08093B606089581E08093B706109255
:100C0000B6068091B406882381F068E378E180918C
:100C1000B2069091B30633D50E94489465E378E11B
:100C20008091B2069091B3069BD60E94394352CC74
:100C300008951092D80A0895CF93DF93CAE6DAE0B8
:100C400081E090E09A8389831092D80A0E942E4A0C
:100C50006C837D838E839F83E49AEC9ADF91CF919E
:100C60000895CF92DF92EF92FF928091E209833054
:100C700009F061C08091E3098130D1F488EE93E0FE
:100C8000A0E0B0E08093740990937509A093760971
:100C9000B093770980E797E1A0E0B0E0809378090E
:100CA00090937909A0937A09B0937B0932E001C04F
:100CB00030E0E091E309F0E0EC51F64F2081A0E153
:100CC000A30F48EE53E060E070E088EBC82E8BE0A5
:100CD000D82EE12CF12C832F90E0FC01EE0FFF1FAA
:100CE000EE0FFF1FEC58F64F27FF10C0C082D182D5
:100CF000E282F382880F991F880F991FFC01E85840
:100D0000F64F40835183628373830FC040835183C6
:100D100062837383880F991F880F991FFC01E8581D
:100D2000F64FC082D182E282F3823E5F220F3A13F5
:100D3000D2CF3093DD09FF90EF90DF90CF900895F0
:100D4000CF93DF938091E109811153C01092DF09A5
:100D50001092DC09C1E0C093E109D091E00961E0A3
:100D600089E00E94C74760E089E00E945D462D2F20
:100D700030E040E050E060E47FE180E090E00E94FD
:100D800071BBC093B00089E08093B1002093B300A1
:100D90008BEA289F212D112426952093B400809161
:100DA0006F008B7F80936F008091B0008062809392
:100DB000B0002091840030918500E091DC0981E051
:100DC0008E0F8093DC0984E0E89FF0011124EC5839
:100DD000F64F80819181A281B381820F931F9093FE
:100DE0008B0080938A00B29A80916F008460809318
:100DF0006F00DF91CF9108958F929F92AF92BF9233
:100E0000CF92DF92EF92FF9282E18093DD0986E03C
:100E10008093DE0996E29093E00991E09093E309D4
:100E20009093E4098093E20988ED90E4A0E0B0E0BB
:100E30008093740990937509A0937609B09377090C
:100E40008CE19CE0A0E0B0E0809378099093790970
:100E5000A0937A09B0937B09742F662755274427FE
:100E600022E030E0ACE1CA2EACE0DA2EE12CF12C2D
:100E7000B8E38B2EB8E19B2EA12CB12CC901880FB1
:100E8000991F880F991FFC01EC58F64F77FF05C09A
:100E900080829182A282B38204C0C082D182E28227
:100EA000F382F901EE0FFF1FEE0FFF1FE858F64F18
:100EB000C082D182E282F382440F551F661F771FE2
:100EC0002E5F3F4F22313105C9F68CE199E8A0E051
:100ED000B0E08093B8099093B909A093BA09B09390
:100EE000BB09FF90EF90DF90CF90BF90AF909F90A5
:100EF0008F9026CF1F920F920FB60F9211240BB630
:100F00000F922F933F934F935F936F937F938F93A2
:100F10009F93AF93BF93EF93FF939091DC098091E0
:100F2000DD09981316C01092DC098091E3098F5FE8
:100F30008093E3099091E3098091E409891740F4D3
:100F400081E08093E3098091DF098F5F8093DF095F
:100F500088DE9091DF098091DE0998130DC08091A1
:100F6000B0008F7D8093B00080916F008B7F809365
:100F70006F001092E10927C08091B00085FF04C086
:100F80008091B0008F7D03C08091B000806280931B
:100F9000B0002091840030918500E091DC0981E06F
:100FA0008E0F8093DC0984E0E89FF0011124EC5857
:100FB000F64F80819181A281B381820F931F90931C
:100FC0008B0080938A00FF91EF91BF91AF919F9129
:100FD0008F917F916F915F914F913F912F910F90E2
:100FE0000BBE0F900FBE0F901F9018951F920F927F
:100FF0000FB60F9211240BB60F921F932F933F93AE
:101000004F935F936F937F938F939F93AF93BF9310
:10101000EF93FF93CF93DF9300D01F92CDB7DEB74E
:1010200080916A0A7CD611E0892B09F010E00E94B9
:101030002E4A69837A838B839C8389819A81AB81D1
:10104000BC8140916E0A50916F0A6091700A709154
:10105000710A841B950BA60BB70B20916B0A30917C
:101060006C0A2430310509F44CC02530310521F0DB
:1010700021303105E9F414C020916D0A222339F0A2
:101080002091D80A20FF02C0289A01C02898112375
:1010900079F0813E2EE29207A105B10548F02BC000
:1010A000112379F125E030E030936C0A20936B0A2C
:1010B00020916B0A30916C0A2530310511F5E091D1
:1010C000D80AF0E0EE0FFF1FEE58F54F91838083B2
:1010D00089819A81AB81BC8180936E0A90936F0A5B
:1010E000A093700AB093710A8091D80A8F5F8093A1
:1010F000D80A833330F084E090E090936C0A8093B8
:101100006B0A0F900F900F900F90DF91CF91FF918E
:10111000EF91BF91AF919F918F917F916F915F916F
:101120004F913F912F911F910F900BBE0F900FBECB
:101130000F901F901895CF93DF93EC0180916A0A6E
:1011400062E00E94C747E881F9810190F081E02DBB
:10115000CE01DF91CF9119940895CF92DF92EF9253
:10116000FF920F931F93CF93DF936C017A018B0152
:10117000C0E0D0E0CE15DF0589F0D8016D918D017A
:10118000D601ED91FC910190F081E02DC6011995F9
:10119000892B11F47E0102C02196ECCFC701DF91AB
:1011A000CF911F910F91FF90EF90DF90CF90089516
:1011B000FC01A089B1898C91A689B78982FD0FC0F5
:1011C0009C91818D8F5F8F73228D821749F0218DC5
:1011D000DF01A20FB11D5D969C93818F08958C91C4
:1011E0000895FC01918D828D981761F0828DDF0149
:1011F000A80FB11D5D968C91928D9F5F9F73928F0A
:1012000090E008958FEF9FEF0895FC01918D828DFE
:10121000981731F0828DE80FF11D858D90E00895CB
:101220008FEF9FEF0895FC01918D228D892F90E023
:10123000805C9F4F821B91098F739927089580E0EE
:1012400097E0F1DF21E0892B09F420E0822F089557
:101250008DE997E0E8DF21E0892B09F420E0822F77
:1012600008958AE398E0DFDF21E0892B09F420E08C
:10127000822F089587ED98E0D6DF21E0892B09F4CD
:1012800020E0822F0895FC01848DDF01A80FB11D9D
:10129000A35ABF4F2C91848D90E001968F739927AC
:1012A000848FA689B7892C93A089B1898C91806499
:1012B0008C93938D848D981306C00288F389E02D5A
:1012C00080818F7D80830895EF92FF920F931F930B
:1012D000CF93DF93EC0181E0888F9B8D8C8D9813E9
:1012E00005C0E889F989808185FD23C0F62E0B8D24
:1012F00010E00F5F1F4F0F731127E02E8C8DE81247
:101300000BC00FB607FCFACFE889F989808185FF09
:10131000F5CFCE01B8DFF2CF8B8DFE01E80FF11DC6
:10132000E35AFF4FF0820B8FEA89FB89808180624C
:1013300007C0EE89FF896083E889F989808180642C
:10134000808381E090E0DF91CF911F910F91FF901A
:10135000EF900895CF93DF93EC01888D8823C1F03F
:10136000EA89FB89808185FD05C0A889B9898C91AE
:1013700086FD0EC00FB607FCF5CF808185FFF2CF4A
:10138000A889B9898C9185FFEDCFCE017CDFE8CFAC
:10139000DF91CF91089580E090E0892B19F06ADF0A
:1013A000811116C080E090E0892B19F05ADF81117D
:1013B00012C080E090E0892B19F04ADF81110EC045
:1013C00080E090E0892B79F03ADF81110AC008951E
:1013D0000E940000E7CF0E940000EBCF0E940000B7
:1013E000EFCF0C94000008950E9439B90F931F931A
:1013F000CF93DF938C01EB01FC01808191810097F9
:10140000B1F0688179816115710579F0428153816C
:101410002C813D814217530740F00E9451B98C81C5
:101420009D81F8019583848313C00E94BDB7888194
:101430009981F801918380838A819B819383828340
:101440008C819D8195838483198218821B821A82E4
:101450001D821C82DF91CF911F910F9108950F93F0
:101460001F93CF93DF93EC0188819981009729F036
:101470002A813B812617370788F48B016F5F7F4FE6
:101480000E9455B8009761F0998388831B830A8373
:101490002C813D81232B11F4FC01108281E001C0DD
:1014A00080E0DF91CF911F910F910895EF92FF920D
:1014B0000F931F93CF93DF93FB0124813581E0804D
:1014C000F180FC0104811581E114F10411F480E044
:1014D00016C02115310591F0EC01020F131FB80160
:1014E000BEDF8823A1F3288139818C819D81B701DA
:1014F000820F931F0E9451B91D830C8381E0DF91FD
:10150000CF911F910F91FF90EF900895EF92FF926E
:101510000F931F93CF93DF93EC017B018A01BA01F4
:101520009EDF2881398181110DC02115310519F007
:10153000C9010E94BDB7198218821D821C821B82BC
:101540001A8206C01D830C83B701C9010E9451B9DC
:10155000CE01DF91CF911F910F91FF90EF900895F1
:10156000CF93DF93EC016115710551F0FB01019000
:101570000020E9F73197AF01461B570BC7DF0CC0BE
:1015800088819981009711F00E94BDB71982188255
:101590001D821C821B821A82CE01DF91CF91089599
:1015A000FC01808191810C94BDB70F931F93CF9361
:1015B000DF93CDB7DEB762970FB6F894DEBF0FBEEC
:1015C000CDBF8C01CB01F8011182108213821282EF
:1015D0001582148250E0BE016F5F7F4F0E94BCB93C
:1015E000BE016F5F7F4FC801BBDF62960FB6F894F4
:1015F000DEBF0FBECDBFDF91CF911F910F91089538
:10160000FC011182108213821282158214826115EC
:10161000710549F0FB0101900020E9F73197AF0116
:10162000461B570B73CF0895CF93DF9300D01F92C3
:10163000CDB7DEB7611571058105910579F09B0184
:10164000AC0169833A834B835C830E94B0B92981E2
:101650003A814B815C810E9471BB03C060E070E005
:10166000CB010F900F900F900F90DF91CF910895C5
:10167000DC01ED91FC910190F081E02D1994EF9245
:10168000FF920F931F93CF93DF938C017B01C0E0F8
:10169000D0E0F701EC0FFD1F6491662361F0D801E3
:1016A000ED91FC910190F081E02DC8011995892BF5
:1016B00011F02196EECFCE01DF91CF911F910F91C6
:1016C000FF90EF9008956115710579F0FB0101908D
:1016D0000020E9F73197AF01461B570BDC01ED9174
:1016E000FC910280F381E02D199480E090E0089550
:1016F0004F925F926F927F92EF92FF920F931F93A0
:10170000CF93DF93CDB7DEB7A1970FB6F894DEBFC6
:101710000FBECDBF7C01FA01CB0119A2223008F423
:101720002AE08E010F5D1F4F422E512C612C712C2F
:10173000BF01A30192010E949DBBF901CA010150A2
:1017400011096A3014F4605D01C0695CD8016C93C2
:10175000232B242B252B61F7B801C701B4DFA196F9
:101760000FB6F894DEBF0FBECDBFDF91CF911F91B2
:101770000F91FF90EF907F906F905F904F90089542
:101780004F925F926F927F928F929F92AF92BF9291
:10179000CF92DF92EF92FF92CF93DF93EC016A0139
:1017A0007B01B22E9A01AB01C701B6010E94A7B618
:1017B000882319F060E076E027C026013701E8941D
:1017C00077F82FEF3FEF4FE75FE7C301B2010E94C9
:1017D000A7B681110DC02FEF3FEF4FE75FE7C301C1
:1017E000B2010E9428BA18161CF464E076E00CC01E
:1017F0002FEF3FEF4FE75FE4C701B6010E949DB6B0
:10180000181694F468E076E0CE01DF91CF91FF9056
:10181000EF90DF90CF90BF90AF909F908F907F9090
:101820006F905F904F904FCF2FEF3FEF4FE75FEC00
:10183000C701B6010E9428BA87FDE4CF20E030E05E
:10184000A901C701B6010E9428BA87FF09C06DE24D
:10185000CE010EDF4C01F7FAF094F7F8F09402C0D5
:10186000812C912CA12C60E070E080E09FE3AB1410
:1018700041F020E030E040E251E40E9404B6A3943D
:10188000F6CF9B01AC01C701B6010E94A0B52B01A8
:101890003C010E9471B66B017C010E942CBA9B0135
:1018A000AC01C301B2010E949FB52B013C012AE0AB
:1018B000B701A601CE011CDF7C01E80CF91CBB209E
:1018C00029F06EE2CE01D4DEE80EF91EDB2CDD201D
:1018D00021F120E030E040E251E4C301B2010E9476
:1018E0008DBA2B013C010E9471B64B01A12CB12C89
:1018F0002AE0B501A401CE01FBDEE80EF91EC50108
:10190000B4010E942CBA9B01AC01C301B2010E9438
:101910009FB52B013C01DA94DACFC701DF91CF915B
:10192000FF90EF90DF90CF90BF90AF909F908F90FF
:101930007F906F905F904F9008956CE076E0C3CEFB
:101940000F931F93CF93DF93EC01BDDE8C01CE018B
:10195000F4DF800F911FDF91CF911F910F910895B8
:101960000F931F93CF93DF93EC0189DE8C01CE019F
:10197000E4DF800F911FDF91CF911F910F910895A8
:101980001F920F920FB60F9211240BB60F922F9346
:101990003F934F935F936F937F938F939F93AF93F7
:1019A000BF93EF93FF9380E097E06DDCFF91EF91A1
:1019B000BF91AF919F918F917F916F915F914F9167
:1019C0003F912F910F900BBE0F900FBE0F901F9065
:1019D00018951F920F920FB60F9211240BB60F920B
:1019E0002F933F934F935F936F937F938F939F9327
:1019F000AF93BF93EF93FF9380E097E0D9DBFF9124
:101A0000EF91BF91AF919F918F917F916F915F9176
:101A10004F913F912F910F900BBE0F900FBE0F90E3
:101A20001F9018951F920F920FB60F9211240BB6AC
:101A30000F922F933F934F935F936F937F938F9367
:101A40009F93AF93BF93EF93FF938DE997E01BDCD8
:101A5000FF91EF91BF91AF919F918F917F916F9186
:101A60005F914F913F912F910F900BBE0F900FBE42
:101A70000F901F9018951F920F920FB60F9211247E
:101A80000BB60F922F933F934F935F936F937F9378
:101A90008F939F93AF93BF93EF93FF938DE997E05D
:101AA00087DBFF91EF91BF91AF919F918F917F91D4
:101AB0006F915F914F913F912F910F900BBE0F90BF
:101AC0000FBE0F901F9018951F920F920FB60F9296
:101AD00011240BB60F922F933F934F935F936F9305
:101AE0007F938F939F93AF93BF93EF93FF938AE37B
:101AF00098E0C9DBFF91EF91BF91AF919F918F91DA
:101B00007F916F915F914F913F912F910F900BBEFD
:101B10000F900FBE0F901F9018951F920F920FB647
:101B20000F9211240BB60F922F933F934F935F9315
:101B30006F937F938F939F93AF93BF93EF93FF9395
:101B40008AE398E035DBFF91EF91BF91AF919F91D0
:101B50008F917F916F915F914F913F912F910F9056
:101B60000BBE0F900FBE0F901F9018951F920F92F3
:101B70000FB60F9211240BB60F922F933F934F93F2
:101B80005F936F937F938F939F93AF93BF93EF93E5
:101B9000FF9387ED98E077DBFF91EF91BF91AF91D5
:101BA0009F918F917F916F915F914F913F912F9175
:101BB0000F900BBE0F900FBE0F901F9018951F92A5
:101BC0000F920FB60F9211240BB60F922F933F93E3
:101BD0004F935F936F937F938F939F93AF93BF9335
:101BE000EF93FF9387ED98E0E3DAFF91EF91BF91D8
:101BF000AF919F918F917F916F915F914F913F91A5
:101C00002F910F900BBE0F900FBE0F901F90189545
